
LED_Blink.elf:     file format elf32-littlearm

Sections:
Idx Name          Size      VMA       LMA       File off  Algn
  0 .isr_vector   000000c0  08000000  08000000  00010000  2**0
                  CONTENTS, ALLOC, LOAD, READONLY, DATA
  1 .text         00001818  080000c0  080000c0  000100c0  2**2
                  CONTENTS, ALLOC, LOAD, READONLY, CODE
  2 .rodata       0000001c  080018d8  080018d8  000118d8  2**2
                  CONTENTS, ALLOC, LOAD, READONLY, DATA
  3 .ARM.extab    00000000  080018f4  080018f4  0002000c  2**0
                  CONTENTS
  4 .ARM          00000008  080018f4  080018f4  000118f4  2**2
                  CONTENTS, ALLOC, LOAD, READONLY, DATA
  5 .preinit_array 00000000  080018fc  080018fc  0002000c  2**0
                  CONTENTS, ALLOC, LOAD, DATA
  6 .init_array   00000004  080018fc  080018fc  000118fc  2**2
                  CONTENTS, ALLOC, LOAD, DATA
  7 .fini_array   00000004  08001900  08001900  00011900  2**2
                  CONTENTS, ALLOC, LOAD, DATA
  8 .data         0000000c  20000000  08001904  00020000  2**2
                  CONTENTS, ALLOC, LOAD, DATA
  9 .bss          00000020  2000000c  08001910  0002000c  2**2
                  ALLOC
 10 ._user_heap_stack 00000604  2000002c  08001910  0002002c  2**0
                  ALLOC
 11 .ARM.attributes 00000028  00000000  00000000  0002000c  2**0
                  CONTENTS, READONLY
 12 .debug_info   00002f71  00000000  00000000  00020034  2**0
                  CONTENTS, READONLY, DEBUGGING, OCTETS
 13 .debug_abbrev 00000d76  00000000  00000000  00022fa5  2**0
                  CONTENTS, READONLY, DEBUGGING, OCTETS
 14 .debug_aranges 000003a8  00000000  00000000  00023d20  2**3
                  CONTENTS, READONLY, DEBUGGING, OCTETS
 15 .debug_ranges 00000320  00000000  00000000  000240c8  2**3
                  CONTENTS, READONLY, DEBUGGING, OCTETS
 16 .debug_macro  00012770  00000000  00000000  000243e8  2**0
                  CONTENTS, READONLY, DEBUGGING, OCTETS
 17 .debug_line   00004938  00000000  00000000  00036b58  2**0
                  CONTENTS, READONLY, DEBUGGING, OCTETS
 18 .debug_str    000728c6  00000000  00000000  0003b490  2**0
                  CONTENTS, READONLY, DEBUGGING, OCTETS
 19 .comment      00000050  00000000  00000000  000add56  2**0
                  CONTENTS, READONLY
 20 .debug_frame  00000bc0  00000000  00000000  000adda8  2**2
                  CONTENTS, READONLY, DEBUGGING, OCTETS

Disassembly of section .text:

080000c0 <__do_global_dtors_aux>:
 80000c0:	b510      	push	{r4, lr}
 80000c2:	4c06      	ldr	r4, [pc, #24]	; (80000dc <__do_global_dtors_aux+0x1c>)
 80000c4:	7823      	ldrb	r3, [r4, #0]
 80000c6:	2b00      	cmp	r3, #0
 80000c8:	d107      	bne.n	80000da <__do_global_dtors_aux+0x1a>
 80000ca:	4b05      	ldr	r3, [pc, #20]	; (80000e0 <__do_global_dtors_aux+0x20>)
 80000cc:	2b00      	cmp	r3, #0
 80000ce:	d002      	beq.n	80000d6 <__do_global_dtors_aux+0x16>
 80000d0:	4804      	ldr	r0, [pc, #16]	; (80000e4 <__do_global_dtors_aux+0x24>)
 80000d2:	e000      	b.n	80000d6 <__do_global_dtors_aux+0x16>
 80000d4:	bf00      	nop
 80000d6:	2301      	movs	r3, #1
 80000d8:	7023      	strb	r3, [r4, #0]
 80000da:	bd10      	pop	{r4, pc}
 80000dc:	2000000c 	.word	0x2000000c
 80000e0:	00000000 	.word	0x00000000
 80000e4:	080018c0 	.word	0x080018c0

080000e8 <frame_dummy>:
 80000e8:	4b04      	ldr	r3, [pc, #16]	; (80000fc <frame_dummy+0x14>)
 80000ea:	b510      	push	{r4, lr}
 80000ec:	2b00      	cmp	r3, #0
 80000ee:	d003      	beq.n	80000f8 <frame_dummy+0x10>
 80000f0:	4903      	ldr	r1, [pc, #12]	; (8000100 <frame_dummy+0x18>)
 80000f2:	4804      	ldr	r0, [pc, #16]	; (8000104 <frame_dummy+0x1c>)
 80000f4:	e000      	b.n	80000f8 <frame_dummy+0x10>
 80000f6:	bf00      	nop
 80000f8:	bd10      	pop	{r4, pc}
 80000fa:	46c0      	nop			; (mov r8, r8)
 80000fc:	00000000 	.word	0x00000000
 8000100:	20000010 	.word	0x20000010
 8000104:	080018c0 	.word	0x080018c0

08000108 <__udivsi3>:
 8000108:	2200      	movs	r2, #0
 800010a:	0843      	lsrs	r3, r0, #1
 800010c:	428b      	cmp	r3, r1
 800010e:	d374      	bcc.n	80001fa <__udivsi3+0xf2>
 8000110:	0903      	lsrs	r3, r0, #4
 8000112:	428b      	cmp	r3, r1
 8000114:	d35f      	bcc.n	80001d6 <__udivsi3+0xce>
 8000116:	0a03      	lsrs	r3, r0, #8
 8000118:	428b      	cmp	r3, r1
 800011a:	d344      	bcc.n	80001a6 <__udivsi3+0x9e>
 800011c:	0b03      	lsrs	r3, r0, #12
 800011e:	428b      	cmp	r3, r1
 8000120:	d328      	bcc.n	8000174 <__udivsi3+0x6c>
 8000122:	0c03      	lsrs	r3, r0, #16
 8000124:	428b      	cmp	r3, r1
 8000126:	d30d      	bcc.n	8000144 <__udivsi3+0x3c>
 8000128:	22ff      	movs	r2, #255	; 0xff
 800012a:	0209      	lsls	r1, r1, #8
 800012c:	ba12      	rev	r2, r2
 800012e:	0c03      	lsrs	r3, r0, #16
 8000130:	428b      	cmp	r3, r1
 8000132:	d302      	bcc.n	800013a <__udivsi3+0x32>
 8000134:	1212      	asrs	r2, r2, #8
 8000136:	0209      	lsls	r1, r1, #8
 8000138:	d065      	beq.n	8000206 <__udivsi3+0xfe>
 800013a:	0b03      	lsrs	r3, r0, #12
 800013c:	428b      	cmp	r3, r1
 800013e:	d319      	bcc.n	8000174 <__udivsi3+0x6c>
 8000140:	e000      	b.n	8000144 <__udivsi3+0x3c>
 8000142:	0a09      	lsrs	r1, r1, #8
 8000144:	0bc3      	lsrs	r3, r0, #15
 8000146:	428b      	cmp	r3, r1
 8000148:	d301      	bcc.n	800014e <__udivsi3+0x46>
 800014a:	03cb      	lsls	r3, r1, #15
 800014c:	1ac0      	subs	r0, r0, r3
 800014e:	4152      	adcs	r2, r2
 8000150:	0b83      	lsrs	r3, r0, #14
 8000152:	428b      	cmp	r3, r1
 8000154:	d301      	bcc.n	800015a <__udivsi3+0x52>
 8000156:	038b      	lsls	r3, r1, #14
 8000158:	1ac0      	subs	r0, r0, r3
 800015a:	4152      	adcs	r2, r2
 800015c:	0b43      	lsrs	r3, r0, #13
 800015e:	428b      	cmp	r3, r1
 8000160:	d301      	bcc.n	8000166 <__udivsi3+0x5e>
 8000162:	034b      	lsls	r3, r1, #13
 8000164:	1ac0      	subs	r0, r0, r3
 8000166:	4152      	adcs	r2, r2
 8000168:	0b03      	lsrs	r3, r0, #12
 800016a:	428b      	cmp	r3, r1
 800016c:	d301      	bcc.n	8000172 <__udivsi3+0x6a>
 800016e:	030b      	lsls	r3, r1, #12
 8000170:	1ac0      	subs	r0, r0, r3
 8000172:	4152      	adcs	r2, r2
 8000174:	0ac3      	lsrs	r3, r0, #11
 8000176:	428b      	cmp	r3, r1
 8000178:	d301      	bcc.n	800017e <__udivsi3+0x76>
 800017a:	02cb      	lsls	r3, r1, #11
 800017c:	1ac0      	subs	r0, r0, r3
 800017e:	4152      	adcs	r2, r2
 8000180:	0a83      	lsrs	r3, r0, #10
 8000182:	428b      	cmp	r3, r1
 8000184:	d301      	bcc.n	800018a <__udivsi3+0x82>
 8000186:	028b      	lsls	r3, r1, #10
 8000188:	1ac0      	subs	r0, r0, r3
 800018a:	4152      	adcs	r2, r2
 800018c:	0a43      	lsrs	r3, r0, #9
 800018e:	428b      	cmp	r3, r1
 8000190:	d301      	bcc.n	8000196 <__udivsi3+0x8e>
 8000192:	024b      	lsls	r3, r1, #9
 8000194:	1ac0      	subs	r0, r0, r3
 8000196:	4152      	adcs	r2, r2
 8000198:	0a03      	lsrs	r3, r0, #8
 800019a:	428b      	cmp	r3, r1
 800019c:	d301      	bcc.n	80001a2 <__udivsi3+0x9a>
 800019e:	020b      	lsls	r3, r1, #8
 80001a0:	1ac0      	subs	r0, r0, r3
 80001a2:	4152      	adcs	r2, r2
 80001a4:	d2cd      	bcs.n	8000142 <__udivsi3+0x3a>
 80001a6:	09c3      	lsrs	r3, r0, #7
 80001a8:	428b      	cmp	r3, r1
 80001aa:	d301      	bcc.n	80001b0 <__udivsi3+0xa8>
 80001ac:	01cb      	lsls	r3, r1, #7
 80001ae:	1ac0      	subs	r0, r0, r3
 80001b0:	4152      	adcs	r2, r2
 80001b2:	0983      	lsrs	r3, r0, #6
 80001b4:	428b      	cmp	r3, r1
 80001b6:	d301      	bcc.n	80001bc <__udivsi3+0xb4>
 80001b8:	018b      	lsls	r3, r1, #6
 80001ba:	1ac0      	subs	r0, r0, r3
 80001bc:	4152      	adcs	r2, r2
 80001be:	0943      	lsrs	r3, r0, #5
 80001c0:	428b      	cmp	r3, r1
 80001c2:	d301      	bcc.n	80001c8 <__udivsi3+0xc0>
 80001c4:	014b      	lsls	r3, r1, #5
 80001c6:	1ac0      	subs	r0, r0, r3
 80001c8:	4152      	adcs	r2, r2
 80001ca:	0903      	lsrs	r3, r0, #4
 80001cc:	428b      	cmp	r3, r1
 80001ce:	d301      	bcc.n	80001d4 <__udivsi3+0xcc>
 80001d0:	010b      	lsls	r3, r1, #4
 80001d2:	1ac0      	subs	r0, r0, r3
 80001d4:	4152      	adcs	r2, r2
 80001d6:	08c3      	lsrs	r3, r0, #3
 80001d8:	428b      	cmp	r3, r1
 80001da:	d301      	bcc.n	80001e0 <__udivsi3+0xd8>
 80001dc:	00cb      	lsls	r3, r1, #3
 80001de:	1ac0      	subs	r0, r0, r3
 80001e0:	4152      	adcs	r2, r2
 80001e2:	0883      	lsrs	r3, r0, #2
 80001e4:	428b      	cmp	r3, r1
 80001e6:	d301      	bcc.n	80001ec <__udivsi3+0xe4>
 80001e8:	008b      	lsls	r3, r1, #2
 80001ea:	1ac0      	subs	r0, r0, r3
 80001ec:	4152      	adcs	r2, r2
 80001ee:	0843      	lsrs	r3, r0, #1
 80001f0:	428b      	cmp	r3, r1
 80001f2:	d301      	bcc.n	80001f8 <__udivsi3+0xf0>
 80001f4:	004b      	lsls	r3, r1, #1
 80001f6:	1ac0      	subs	r0, r0, r3
 80001f8:	4152      	adcs	r2, r2
 80001fa:	1a41      	subs	r1, r0, r1
 80001fc:	d200      	bcs.n	8000200 <__udivsi3+0xf8>
 80001fe:	4601      	mov	r1, r0
 8000200:	4152      	adcs	r2, r2
 8000202:	4610      	mov	r0, r2
 8000204:	4770      	bx	lr
 8000206:	e7ff      	b.n	8000208 <__udivsi3+0x100>
 8000208:	b501      	push	{r0, lr}
 800020a:	2000      	movs	r0, #0
 800020c:	f000 f806 	bl	800021c <__aeabi_idiv0>
 8000210:	bd02      	pop	{r1, pc}
 8000212:	46c0      	nop			; (mov r8, r8)

08000214 <__aeabi_uidivmod>:
 8000214:	2900      	cmp	r1, #0
 8000216:	d0f7      	beq.n	8000208 <__udivsi3+0x100>
 8000218:	e776      	b.n	8000108 <__udivsi3>
 800021a:	4770      	bx	lr

0800021c <__aeabi_idiv0>:
 800021c:	4770      	bx	lr
 800021e:	46c0      	nop			; (mov r8, r8)

08000220 <__aeabi_uldivmod>:
 8000220:	2b00      	cmp	r3, #0
 8000222:	d111      	bne.n	8000248 <__aeabi_uldivmod+0x28>
 8000224:	2a00      	cmp	r2, #0
 8000226:	d10f      	bne.n	8000248 <__aeabi_uldivmod+0x28>
 8000228:	2900      	cmp	r1, #0
 800022a:	d100      	bne.n	800022e <__aeabi_uldivmod+0xe>
 800022c:	2800      	cmp	r0, #0
 800022e:	d002      	beq.n	8000236 <__aeabi_uldivmod+0x16>
 8000230:	2100      	movs	r1, #0
 8000232:	43c9      	mvns	r1, r1
 8000234:	0008      	movs	r0, r1
 8000236:	b407      	push	{r0, r1, r2}
 8000238:	4802      	ldr	r0, [pc, #8]	; (8000244 <__aeabi_uldivmod+0x24>)
 800023a:	a102      	add	r1, pc, #8	; (adr r1, 8000244 <__aeabi_uldivmod+0x24>)
 800023c:	1840      	adds	r0, r0, r1
 800023e:	9002      	str	r0, [sp, #8]
 8000240:	bd03      	pop	{r0, r1, pc}
 8000242:	46c0      	nop			; (mov r8, r8)
 8000244:	ffffffd9 	.word	0xffffffd9
 8000248:	b403      	push	{r0, r1}
 800024a:	4668      	mov	r0, sp
 800024c:	b501      	push	{r0, lr}
 800024e:	9802      	ldr	r0, [sp, #8]
 8000250:	f000 f834 	bl	80002bc <__udivmoddi4>
 8000254:	9b01      	ldr	r3, [sp, #4]
 8000256:	469e      	mov	lr, r3
 8000258:	b002      	add	sp, #8
 800025a:	bc0c      	pop	{r2, r3}
 800025c:	4770      	bx	lr
 800025e:	46c0      	nop			; (mov r8, r8)

08000260 <__aeabi_lmul>:
 8000260:	b5f0      	push	{r4, r5, r6, r7, lr}
 8000262:	46ce      	mov	lr, r9
 8000264:	4647      	mov	r7, r8
 8000266:	b580      	push	{r7, lr}
 8000268:	0007      	movs	r7, r0
 800026a:	4699      	mov	r9, r3
 800026c:	0c3b      	lsrs	r3, r7, #16
 800026e:	469c      	mov	ip, r3
 8000270:	0413      	lsls	r3, r2, #16
 8000272:	0c1b      	lsrs	r3, r3, #16
 8000274:	001d      	movs	r5, r3
 8000276:	000e      	movs	r6, r1
 8000278:	4661      	mov	r1, ip
 800027a:	0400      	lsls	r0, r0, #16
 800027c:	0c14      	lsrs	r4, r2, #16
 800027e:	0c00      	lsrs	r0, r0, #16
 8000280:	4345      	muls	r5, r0
 8000282:	434b      	muls	r3, r1
 8000284:	4360      	muls	r0, r4
 8000286:	4361      	muls	r1, r4
 8000288:	18c0      	adds	r0, r0, r3
 800028a:	0c2c      	lsrs	r4, r5, #16
 800028c:	1820      	adds	r0, r4, r0
 800028e:	468c      	mov	ip, r1
 8000290:	4283      	cmp	r3, r0
 8000292:	d903      	bls.n	800029c <__aeabi_lmul+0x3c>
 8000294:	2380      	movs	r3, #128	; 0x80
 8000296:	025b      	lsls	r3, r3, #9
 8000298:	4698      	mov	r8, r3
 800029a:	44c4      	add	ip, r8
 800029c:	4649      	mov	r1, r9
 800029e:	4379      	muls	r1, r7
 80002a0:	4372      	muls	r2, r6
 80002a2:	0c03      	lsrs	r3, r0, #16
 80002a4:	4463      	add	r3, ip
 80002a6:	042d      	lsls	r5, r5, #16
 80002a8:	0c2d      	lsrs	r5, r5, #16
 80002aa:	18c9      	adds	r1, r1, r3
 80002ac:	0400      	lsls	r0, r0, #16
 80002ae:	1940      	adds	r0, r0, r5
 80002b0:	1889      	adds	r1, r1, r2
 80002b2:	bcc0      	pop	{r6, r7}
 80002b4:	46b9      	mov	r9, r7
 80002b6:	46b0      	mov	r8, r6
 80002b8:	bdf0      	pop	{r4, r5, r6, r7, pc}
 80002ba:	46c0      	nop			; (mov r8, r8)

080002bc <__udivmoddi4>:
 80002bc:	b5f0      	push	{r4, r5, r6, r7, lr}
 80002be:	4657      	mov	r7, sl
 80002c0:	464e      	mov	r6, r9
 80002c2:	4645      	mov	r5, r8
 80002c4:	46de      	mov	lr, fp
 80002c6:	b5e0      	push	{r5, r6, r7, lr}
 80002c8:	0004      	movs	r4, r0
 80002ca:	000d      	movs	r5, r1
 80002cc:	4692      	mov	sl, r2
 80002ce:	4699      	mov	r9, r3
 80002d0:	b083      	sub	sp, #12
 80002d2:	428b      	cmp	r3, r1
 80002d4:	d830      	bhi.n	8000338 <__udivmoddi4+0x7c>
 80002d6:	d02d      	beq.n	8000334 <__udivmoddi4+0x78>
 80002d8:	4649      	mov	r1, r9
 80002da:	4650      	mov	r0, sl
 80002dc:	f000 f8ba 	bl	8000454 <__clzdi2>
 80002e0:	0029      	movs	r1, r5
 80002e2:	0006      	movs	r6, r0
 80002e4:	0020      	movs	r0, r4
 80002e6:	f000 f8b5 	bl	8000454 <__clzdi2>
 80002ea:	1a33      	subs	r3, r6, r0
 80002ec:	4698      	mov	r8, r3
 80002ee:	3b20      	subs	r3, #32
 80002f0:	469b      	mov	fp, r3
 80002f2:	d433      	bmi.n	800035c <__udivmoddi4+0xa0>
 80002f4:	465a      	mov	r2, fp
 80002f6:	4653      	mov	r3, sl
 80002f8:	4093      	lsls	r3, r2
 80002fa:	4642      	mov	r2, r8
 80002fc:	001f      	movs	r7, r3
 80002fe:	4653      	mov	r3, sl
 8000300:	4093      	lsls	r3, r2
 8000302:	001e      	movs	r6, r3
 8000304:	42af      	cmp	r7, r5
 8000306:	d83a      	bhi.n	800037e <__udivmoddi4+0xc2>
 8000308:	42af      	cmp	r7, r5
 800030a:	d100      	bne.n	800030e <__udivmoddi4+0x52>
 800030c:	e078      	b.n	8000400 <__udivmoddi4+0x144>
 800030e:	465b      	mov	r3, fp
 8000310:	1ba4      	subs	r4, r4, r6
 8000312:	41bd      	sbcs	r5, r7
 8000314:	2b00      	cmp	r3, #0
 8000316:	da00      	bge.n	800031a <__udivmoddi4+0x5e>
 8000318:	e075      	b.n	8000406 <__udivmoddi4+0x14a>
 800031a:	2200      	movs	r2, #0
 800031c:	2300      	movs	r3, #0
 800031e:	9200      	str	r2, [sp, #0]
 8000320:	9301      	str	r3, [sp, #4]
 8000322:	2301      	movs	r3, #1
 8000324:	465a      	mov	r2, fp
 8000326:	4093      	lsls	r3, r2
 8000328:	9301      	str	r3, [sp, #4]
 800032a:	2301      	movs	r3, #1
 800032c:	4642      	mov	r2, r8
 800032e:	4093      	lsls	r3, r2
 8000330:	9300      	str	r3, [sp, #0]
 8000332:	e028      	b.n	8000386 <__udivmoddi4+0xca>
 8000334:	4282      	cmp	r2, r0
 8000336:	d9cf      	bls.n	80002d8 <__udivmoddi4+0x1c>
 8000338:	2200      	movs	r2, #0
 800033a:	2300      	movs	r3, #0
 800033c:	9200      	str	r2, [sp, #0]
 800033e:	9301      	str	r3, [sp, #4]
 8000340:	9b0c      	ldr	r3, [sp, #48]	; 0x30
 8000342:	2b00      	cmp	r3, #0
 8000344:	d001      	beq.n	800034a <__udivmoddi4+0x8e>
 8000346:	601c      	str	r4, [r3, #0]
 8000348:	605d      	str	r5, [r3, #4]
 800034a:	9800      	ldr	r0, [sp, #0]
 800034c:	9901      	ldr	r1, [sp, #4]
 800034e:	b003      	add	sp, #12
 8000350:	bcf0      	pop	{r4, r5, r6, r7}
 8000352:	46bb      	mov	fp, r7
 8000354:	46b2      	mov	sl, r6
 8000356:	46a9      	mov	r9, r5
 8000358:	46a0      	mov	r8, r4
 800035a:	bdf0      	pop	{r4, r5, r6, r7, pc}
 800035c:	4642      	mov	r2, r8
 800035e:	2320      	movs	r3, #32
 8000360:	1a9b      	subs	r3, r3, r2
 8000362:	4652      	mov	r2, sl
 8000364:	40da      	lsrs	r2, r3
 8000366:	4641      	mov	r1, r8
 8000368:	0013      	movs	r3, r2
 800036a:	464a      	mov	r2, r9
 800036c:	408a      	lsls	r2, r1
 800036e:	0017      	movs	r7, r2
 8000370:	4642      	mov	r2, r8
 8000372:	431f      	orrs	r7, r3
 8000374:	4653      	mov	r3, sl
 8000376:	4093      	lsls	r3, r2
 8000378:	001e      	movs	r6, r3
 800037a:	42af      	cmp	r7, r5
 800037c:	d9c4      	bls.n	8000308 <__udivmoddi4+0x4c>
 800037e:	2200      	movs	r2, #0
 8000380:	2300      	movs	r3, #0
 8000382:	9200      	str	r2, [sp, #0]
 8000384:	9301      	str	r3, [sp, #4]
 8000386:	4643      	mov	r3, r8
 8000388:	2b00      	cmp	r3, #0
 800038a:	d0d9      	beq.n	8000340 <__udivmoddi4+0x84>
 800038c:	07fb      	lsls	r3, r7, #31
 800038e:	0872      	lsrs	r2, r6, #1
 8000390:	431a      	orrs	r2, r3
 8000392:	4646      	mov	r6, r8
 8000394:	087b      	lsrs	r3, r7, #1
 8000396:	e00e      	b.n	80003b6 <__udivmoddi4+0xfa>
 8000398:	42ab      	cmp	r3, r5
 800039a:	d101      	bne.n	80003a0 <__udivmoddi4+0xe4>
 800039c:	42a2      	cmp	r2, r4
 800039e:	d80c      	bhi.n	80003ba <__udivmoddi4+0xfe>
 80003a0:	1aa4      	subs	r4, r4, r2
 80003a2:	419d      	sbcs	r5, r3
 80003a4:	2001      	movs	r0, #1
 80003a6:	1924      	adds	r4, r4, r4
 80003a8:	416d      	adcs	r5, r5
 80003aa:	2100      	movs	r1, #0
 80003ac:	3e01      	subs	r6, #1
 80003ae:	1824      	adds	r4, r4, r0
 80003b0:	414d      	adcs	r5, r1
 80003b2:	2e00      	cmp	r6, #0
 80003b4:	d006      	beq.n	80003c4 <__udivmoddi4+0x108>
 80003b6:	42ab      	cmp	r3, r5
 80003b8:	d9ee      	bls.n	8000398 <__udivmoddi4+0xdc>
 80003ba:	3e01      	subs	r6, #1
 80003bc:	1924      	adds	r4, r4, r4
 80003be:	416d      	adcs	r5, r5
 80003c0:	2e00      	cmp	r6, #0
 80003c2:	d1f8      	bne.n	80003b6 <__udivmoddi4+0xfa>
 80003c4:	9800      	ldr	r0, [sp, #0]
 80003c6:	9901      	ldr	r1, [sp, #4]
 80003c8:	465b      	mov	r3, fp
 80003ca:	1900      	adds	r0, r0, r4
 80003cc:	4169      	adcs	r1, r5
 80003ce:	2b00      	cmp	r3, #0
 80003d0:	db24      	blt.n	800041c <__udivmoddi4+0x160>
 80003d2:	002b      	movs	r3, r5
 80003d4:	465a      	mov	r2, fp
 80003d6:	4644      	mov	r4, r8
 80003d8:	40d3      	lsrs	r3, r2
 80003da:	002a      	movs	r2, r5
 80003dc:	40e2      	lsrs	r2, r4
 80003de:	001c      	movs	r4, r3
 80003e0:	465b      	mov	r3, fp
 80003e2:	0015      	movs	r5, r2
 80003e4:	2b00      	cmp	r3, #0
 80003e6:	db2a      	blt.n	800043e <__udivmoddi4+0x182>
 80003e8:	0026      	movs	r6, r4
 80003ea:	409e      	lsls	r6, r3
 80003ec:	0033      	movs	r3, r6
 80003ee:	0026      	movs	r6, r4
 80003f0:	4647      	mov	r7, r8
 80003f2:	40be      	lsls	r6, r7
 80003f4:	0032      	movs	r2, r6
 80003f6:	1a80      	subs	r0, r0, r2
 80003f8:	4199      	sbcs	r1, r3
 80003fa:	9000      	str	r0, [sp, #0]
 80003fc:	9101      	str	r1, [sp, #4]
 80003fe:	e79f      	b.n	8000340 <__udivmoddi4+0x84>
 8000400:	42a3      	cmp	r3, r4
 8000402:	d8bc      	bhi.n	800037e <__udivmoddi4+0xc2>
 8000404:	e783      	b.n	800030e <__udivmoddi4+0x52>
 8000406:	4642      	mov	r2, r8
 8000408:	2320      	movs	r3, #32
 800040a:	2100      	movs	r1, #0
 800040c:	1a9b      	subs	r3, r3, r2
 800040e:	2200      	movs	r2, #0
 8000410:	9100      	str	r1, [sp, #0]
 8000412:	9201      	str	r2, [sp, #4]
 8000414:	2201      	movs	r2, #1
 8000416:	40da      	lsrs	r2, r3
 8000418:	9201      	str	r2, [sp, #4]
 800041a:	e786      	b.n	800032a <__udivmoddi4+0x6e>
 800041c:	4642      	mov	r2, r8
 800041e:	2320      	movs	r3, #32
 8000420:	1a9b      	subs	r3, r3, r2
 8000422:	002a      	movs	r2, r5
 8000424:	4646      	mov	r6, r8
 8000426:	409a      	lsls	r2, r3
 8000428:	0023      	movs	r3, r4
 800042a:	40f3      	lsrs	r3, r6
 800042c:	4644      	mov	r4, r8
 800042e:	4313      	orrs	r3, r2
 8000430:	002a      	movs	r2, r5
 8000432:	40e2      	lsrs	r2, r4
 8000434:	001c      	movs	r4, r3
 8000436:	465b      	mov	r3, fp
 8000438:	0015      	movs	r5, r2
 800043a:	2b00      	cmp	r3, #0
 800043c:	dad4      	bge.n	80003e8 <__udivmoddi4+0x12c>
 800043e:	4642      	mov	r2, r8
 8000440:	002f      	movs	r7, r5
 8000442:	2320      	movs	r3, #32
 8000444:	0026      	movs	r6, r4
 8000446:	4097      	lsls	r7, r2
 8000448:	1a9b      	subs	r3, r3, r2
 800044a:	40de      	lsrs	r6, r3
 800044c:	003b      	movs	r3, r7
 800044e:	4333      	orrs	r3, r6
 8000450:	e7cd      	b.n	80003ee <__udivmoddi4+0x132>
 8000452:	46c0      	nop			; (mov r8, r8)

08000454 <__clzdi2>:
 8000454:	b510      	push	{r4, lr}
 8000456:	2900      	cmp	r1, #0
 8000458:	d103      	bne.n	8000462 <__clzdi2+0xe>
 800045a:	f000 f807 	bl	800046c <__clzsi2>
 800045e:	3020      	adds	r0, #32
 8000460:	e002      	b.n	8000468 <__clzdi2+0x14>
 8000462:	0008      	movs	r0, r1
 8000464:	f000 f802 	bl	800046c <__clzsi2>
 8000468:	bd10      	pop	{r4, pc}
 800046a:	46c0      	nop			; (mov r8, r8)

0800046c <__clzsi2>:
 800046c:	211c      	movs	r1, #28
 800046e:	2301      	movs	r3, #1
 8000470:	041b      	lsls	r3, r3, #16
 8000472:	4298      	cmp	r0, r3
 8000474:	d301      	bcc.n	800047a <__clzsi2+0xe>
 8000476:	0c00      	lsrs	r0, r0, #16
 8000478:	3910      	subs	r1, #16
 800047a:	0a1b      	lsrs	r3, r3, #8
 800047c:	4298      	cmp	r0, r3
 800047e:	d301      	bcc.n	8000484 <__clzsi2+0x18>
 8000480:	0a00      	lsrs	r0, r0, #8
 8000482:	3908      	subs	r1, #8
 8000484:	091b      	lsrs	r3, r3, #4
 8000486:	4298      	cmp	r0, r3
 8000488:	d301      	bcc.n	800048e <__clzsi2+0x22>
 800048a:	0900      	lsrs	r0, r0, #4
 800048c:	3904      	subs	r1, #4
 800048e:	a202      	add	r2, pc, #8	; (adr r2, 8000498 <__clzsi2+0x2c>)
 8000490:	5c10      	ldrb	r0, [r2, r0]
 8000492:	1840      	adds	r0, r0, r1
 8000494:	4770      	bx	lr
 8000496:	46c0      	nop			; (mov r8, r8)
 8000498:	02020304 	.word	0x02020304
 800049c:	01010101 	.word	0x01010101
	...

080004a8 <main>:
/**
  * @brief  The application entry point.
  * @retval int
  */
int main(void)
{
 80004a8:	b580      	push	{r7, lr}
 80004aa:	af00      	add	r7, sp, #0
  /* USER CODE END 1 */

  /* MCU Configuration--------------------------------------------------------*/

  /* Reset of all peripherals, Initializes the Flash interface and the Systick. */
  HAL_Init();
 80004ac:	f000 f936 	bl	800071c <HAL_Init>
  /* USER CODE BEGIN Init */

  /* USER CODE END Init */

  /* Configure the system clock */
  SystemClock_Config();
 80004b0:	f000 f804 	bl	80004bc <SystemClock_Config>
  /* USER CODE BEGIN SysInit */

  /* USER CODE END SysInit */

  /* Initialize all configured peripherals */
  MX_GPIO_Init();
 80004b4:	f000 f85e 	bl	8000574 <MX_GPIO_Init>

  /* USER CODE END 2 */

  /* Infinite loop */
  /* USER CODE BEGIN WHILE */
  while (1)
 80004b8:	e7fe      	b.n	80004b8 <main+0x10>
	...

080004bc <SystemClock_Config>:
/**
  * @brief System Clock Configuration
  * @retval None
  */
void SystemClock_Config(void)
{
 80004bc:	b590      	push	{r4, r7, lr}
 80004be:	b095      	sub	sp, #84	; 0x54
 80004c0:	af00      	add	r7, sp, #0
  RCC_OscInitTypeDef RCC_OscInitStruct = {0};
 80004c2:	2418      	movs	r4, #24
 80004c4:	193b      	adds	r3, r7, r4
 80004c6:	0018      	movs	r0, r3
 80004c8:	2338      	movs	r3, #56	; 0x38
 80004ca:	001a      	movs	r2, r3
 80004cc:	2100      	movs	r1, #0
 80004ce:	f001 f9ef 	bl	80018b0 <memset>
  RCC_ClkInitTypeDef RCC_ClkInitStruct = {0};
 80004d2:	1d3b      	adds	r3, r7, #4
 80004d4:	0018      	movs	r0, r3
 80004d6:	2314      	movs	r3, #20
 80004d8:	001a      	movs	r2, r3
 80004da:	2100      	movs	r1, #0
 80004dc:	f001 f9e8 	bl	80018b0 <memset>

  /** Configure the main internal regulator output voltage
  */
  __HAL_PWR_VOLTAGESCALING_CONFIG(PWR_REGULATOR_VOLTAGE_SCALE1);
 80004e0:	4b22      	ldr	r3, [pc, #136]	; (800056c <SystemClock_Config+0xb0>)
 80004e2:	681b      	ldr	r3, [r3, #0]
 80004e4:	4a22      	ldr	r2, [pc, #136]	; (8000570 <SystemClock_Config+0xb4>)
 80004e6:	401a      	ands	r2, r3
 80004e8:	4b20      	ldr	r3, [pc, #128]	; (800056c <SystemClock_Config+0xb0>)
 80004ea:	2180      	movs	r1, #128	; 0x80
 80004ec:	0109      	lsls	r1, r1, #4
 80004ee:	430a      	orrs	r2, r1
 80004f0:	601a      	str	r2, [r3, #0]

  /** Initializes the RCC Oscillators according to the specified parameters
  * in the RCC_OscInitTypeDef structure.
  */
  RCC_OscInitStruct.OscillatorType = RCC_OSCILLATORTYPE_HSI;
 80004f2:	0021      	movs	r1, r4
 80004f4:	187b      	adds	r3, r7, r1
 80004f6:	2202      	movs	r2, #2
 80004f8:	601a      	str	r2, [r3, #0]
  RCC_OscInitStruct.HSIState = RCC_HSI_ON;
 80004fa:	187b      	adds	r3, r7, r1
 80004fc:	2201      	movs	r2, #1
 80004fe:	60da      	str	r2, [r3, #12]
  RCC_OscInitStruct.HSICalibrationValue = RCC_HSICALIBRATION_DEFAULT;
 8000500:	187b      	adds	r3, r7, r1
 8000502:	2210      	movs	r2, #16
 8000504:	611a      	str	r2, [r3, #16]
  RCC_OscInitStruct.PLL.PLLState = RCC_PLL_ON;
 8000506:	187b      	adds	r3, r7, r1
 8000508:	2202      	movs	r2, #2
 800050a:	629a      	str	r2, [r3, #40]	; 0x28
  RCC_OscInitStruct.PLL.PLLSource = RCC_PLLSOURCE_HSI;
 800050c:	187b      	adds	r3, r7, r1
 800050e:	2200      	movs	r2, #0
 8000510:	62da      	str	r2, [r3, #44]	; 0x2c
  RCC_OscInitStruct.PLL.PLLMUL = RCC_PLLMUL_6;
 8000512:	187b      	adds	r3, r7, r1
 8000514:	2280      	movs	r2, #128	; 0x80
 8000516:	0312      	lsls	r2, r2, #12
 8000518:	631a      	str	r2, [r3, #48]	; 0x30
  RCC_OscInitStruct.PLL.PLLDIV = RCC_PLLDIV_3;
 800051a:	187b      	adds	r3, r7, r1
 800051c:	2280      	movs	r2, #128	; 0x80
 800051e:	0412      	lsls	r2, r2, #16
 8000520:	635a      	str	r2, [r3, #52]	; 0x34
  if (HAL_RCC_OscConfig(&RCC_OscInitStruct) != HAL_OK)
 8000522:	187b      	adds	r3, r7, r1
 8000524:	0018      	movs	r0, r3
 8000526:	f000 fbdd 	bl	8000ce4 <HAL_RCC_OscConfig>
 800052a:	1e03      	subs	r3, r0, #0
 800052c:	d001      	beq.n	8000532 <SystemClock_Config+0x76>
  {
    Error_Handler();
 800052e:	f000 f87d 	bl	800062c <Error_Handler>
  }

  /** Initializes the CPU, AHB and APB buses clocks
  */
  RCC_ClkInitStruct.ClockType = RCC_CLOCKTYPE_HCLK|RCC_CLOCKTYPE_SYSCLK
 8000532:	1d3b      	adds	r3, r7, #4
 8000534:	220f      	movs	r2, #15
 8000536:	601a      	str	r2, [r3, #0]
                              |RCC_CLOCKTYPE_PCLK1|RCC_CLOCKTYPE_PCLK2;
  RCC_ClkInitStruct.SYSCLKSource = RCC_SYSCLKSOURCE_PLLCLK;
 8000538:	1d3b      	adds	r3, r7, #4
 800053a:	2203      	movs	r2, #3
 800053c:	605a      	str	r2, [r3, #4]
  RCC_ClkInitStruct.AHBCLKDivider = RCC_SYSCLK_DIV1;
 800053e:	1d3b      	adds	r3, r7, #4
 8000540:	2200      	movs	r2, #0
 8000542:	609a      	str	r2, [r3, #8]
  RCC_ClkInitStruct.APB1CLKDivider = RCC_HCLK_DIV1;
 8000544:	1d3b      	adds	r3, r7, #4
 8000546:	2200      	movs	r2, #0
 8000548:	60da      	str	r2, [r3, #12]
  RCC_ClkInitStruct.APB2CLKDivider = RCC_HCLK_DIV1;
 800054a:	1d3b      	adds	r3, r7, #4
 800054c:	2200      	movs	r2, #0
 800054e:	611a      	str	r2, [r3, #16]

  if (HAL_RCC_ClockConfig(&RCC_ClkInitStruct, FLASH_LATENCY_1) != HAL_OK)
 8000550:	1d3b      	adds	r3, r7, #4
 8000552:	2101      	movs	r1, #1
 8000554:	0018      	movs	r0, r3
 8000556:	f000 ff99 	bl	800148c <HAL_RCC_ClockConfig>
 800055a:	1e03      	subs	r3, r0, #0
 800055c:	d001      	beq.n	8000562 <SystemClock_Config+0xa6>
  {
    Error_Handler();
 800055e:	f000 f865 	bl	800062c <Error_Handler>
  }
}
 8000562:	46c0      	nop			; (mov r8, r8)
 8000564:	46bd      	mov	sp, r7
 8000566:	b015      	add	sp, #84	; 0x54
 8000568:	bd90      	pop	{r4, r7, pc}
 800056a:	46c0      	nop			; (mov r8, r8)
 800056c:	40007000 	.word	0x40007000
 8000570:	ffffe7ff 	.word	0xffffe7ff

08000574 <MX_GPIO_Init>:
  * @brief GPIO Initialization Function
  * @param None
  * @retval None
  */
static void MX_GPIO_Init(void)
{
 8000574:	b590      	push	{r4, r7, lr}
 8000576:	b08b      	sub	sp, #44	; 0x2c
 8000578:	af00      	add	r7, sp, #0
  GPIO_InitTypeDef GPIO_InitStruct = {0};
 800057a:	2414      	movs	r4, #20
 800057c:	193b      	adds	r3, r7, r4
 800057e:	0018      	movs	r0, r3
 8000580:	2314      	movs	r3, #20
 8000582:	001a      	movs	r2, r3
 8000584:	2100      	movs	r1, #0
 8000586:	f001 f993 	bl	80018b0 <memset>
/* USER CODE BEGIN MX_GPIO_Init_1 */
/* USER CODE END MX_GPIO_Init_1 */

  /* GPIO Ports Clock Enable */
  __HAL_RCC_GPIOB_CLK_ENABLE();
 800058a:	4b26      	ldr	r3, [pc, #152]	; (8000624 <MX_GPIO_Init+0xb0>)
 800058c:	6ada      	ldr	r2, [r3, #44]	; 0x2c
 800058e:	4b25      	ldr	r3, [pc, #148]	; (8000624 <MX_GPIO_Init+0xb0>)
 8000590:	2102      	movs	r1, #2
 8000592:	430a      	orrs	r2, r1
 8000594:	62da      	str	r2, [r3, #44]	; 0x2c
 8000596:	4b23      	ldr	r3, [pc, #140]	; (8000624 <MX_GPIO_Init+0xb0>)
 8000598:	6adb      	ldr	r3, [r3, #44]	; 0x2c
 800059a:	2202      	movs	r2, #2
 800059c:	4013      	ands	r3, r2
 800059e:	613b      	str	r3, [r7, #16]
 80005a0:	693b      	ldr	r3, [r7, #16]
  __HAL_RCC_GPIOA_CLK_ENABLE();
 80005a2:	4b20      	ldr	r3, [pc, #128]	; (8000624 <MX_GPIO_Init+0xb0>)
 80005a4:	6ada      	ldr	r2, [r3, #44]	; 0x2c
 80005a6:	4b1f      	ldr	r3, [pc, #124]	; (8000624 <MX_GPIO_Init+0xb0>)
 80005a8:	2101      	movs	r1, #1
 80005aa:	430a      	orrs	r2, r1
 80005ac:	62da      	str	r2, [r3, #44]	; 0x2c
 80005ae:	4b1d      	ldr	r3, [pc, #116]	; (8000624 <MX_GPIO_Init+0xb0>)
 80005b0:	6adb      	ldr	r3, [r3, #44]	; 0x2c
 80005b2:	2201      	movs	r2, #1
 80005b4:	4013      	ands	r3, r2
 80005b6:	60fb      	str	r3, [r7, #12]
 80005b8:	68fb      	ldr	r3, [r7, #12]
  __HAL_RCC_GPIOC_CLK_ENABLE();
 80005ba:	4b1a      	ldr	r3, [pc, #104]	; (8000624 <MX_GPIO_Init+0xb0>)
 80005bc:	6ada      	ldr	r2, [r3, #44]	; 0x2c
 80005be:	4b19      	ldr	r3, [pc, #100]	; (8000624 <MX_GPIO_Init+0xb0>)
 80005c0:	2104      	movs	r1, #4
 80005c2:	430a      	orrs	r2, r1
 80005c4:	62da      	str	r2, [r3, #44]	; 0x2c
 80005c6:	4b17      	ldr	r3, [pc, #92]	; (8000624 <MX_GPIO_Init+0xb0>)
 80005c8:	6adb      	ldr	r3, [r3, #44]	; 0x2c
 80005ca:	2204      	movs	r2, #4
 80005cc:	4013      	ands	r3, r2
 80005ce:	60bb      	str	r3, [r7, #8]
 80005d0:	68bb      	ldr	r3, [r7, #8]
  __HAL_RCC_GPIOH_CLK_ENABLE();
 80005d2:	4b14      	ldr	r3, [pc, #80]	; (8000624 <MX_GPIO_Init+0xb0>)
 80005d4:	6ada      	ldr	r2, [r3, #44]	; 0x2c
 80005d6:	4b13      	ldr	r3, [pc, #76]	; (8000624 <MX_GPIO_Init+0xb0>)
 80005d8:	2180      	movs	r1, #128	; 0x80
 80005da:	430a      	orrs	r2, r1
 80005dc:	62da      	str	r2, [r3, #44]	; 0x2c
 80005de:	4b11      	ldr	r3, [pc, #68]	; (8000624 <MX_GPIO_Init+0xb0>)
 80005e0:	6adb      	ldr	r3, [r3, #44]	; 0x2c
 80005e2:	2280      	movs	r2, #128	; 0x80
 80005e4:	4013      	ands	r3, r2
 80005e6:	607b      	str	r3, [r7, #4]
 80005e8:	687b      	ldr	r3, [r7, #4]

  /*Configure GPIO pin Output Level */
  HAL_GPIO_WritePin(GPIOB, GPIO_PIN_5|GPIO_PIN_7, GPIO_PIN_RESET);
 80005ea:	4b0f      	ldr	r3, [pc, #60]	; (8000628 <MX_GPIO_Init+0xb4>)
 80005ec:	2200      	movs	r2, #0
 80005ee:	21a0      	movs	r1, #160	; 0xa0
 80005f0:	0018      	movs	r0, r3
 80005f2:	f000 fb59 	bl	8000ca8 <HAL_GPIO_WritePin>

  /*Configure GPIO pins : PB5 PB7 */
  GPIO_InitStruct.Pin = GPIO_PIN_5|GPIO_PIN_7;
 80005f6:	0021      	movs	r1, r4
 80005f8:	187b      	adds	r3, r7, r1
 80005fa:	22a0      	movs	r2, #160	; 0xa0
 80005fc:	601a      	str	r2, [r3, #0]
  GPIO_InitStruct.Mode = GPIO_MODE_OUTPUT_PP;
 80005fe:	187b      	adds	r3, r7, r1
 8000600:	2201      	movs	r2, #1
 8000602:	605a      	str	r2, [r3, #4]
  GPIO_InitStruct.Pull = GPIO_NOPULL;
 8000604:	187b      	adds	r3, r7, r1
 8000606:	2200      	movs	r2, #0
 8000608:	609a      	str	r2, [r3, #8]
  GPIO_InitStruct.Speed = GPIO_SPEED_FREQ_LOW;
 800060a:	187b      	adds	r3, r7, r1
 800060c:	2200      	movs	r2, #0
 800060e:	60da      	str	r2, [r3, #12]
  HAL_GPIO_Init(GPIOB, &GPIO_InitStruct);
 8000610:	187b      	adds	r3, r7, r1
 8000612:	4a05      	ldr	r2, [pc, #20]	; (8000628 <MX_GPIO_Init+0xb4>)
 8000614:	0019      	movs	r1, r3
 8000616:	0010      	movs	r0, r2
 8000618:	f000 f9c8 	bl	80009ac <HAL_GPIO_Init>

/* USER CODE BEGIN MX_GPIO_Init_2 */
/* USER CODE END MX_GPIO_Init_2 */
}
 800061c:	46c0      	nop			; (mov r8, r8)
 800061e:	46bd      	mov	sp, r7
 8000620:	b00b      	add	sp, #44	; 0x2c
 8000622:	bd90      	pop	{r4, r7, pc}
 8000624:	40021000 	.word	0x40021000
 8000628:	50000400 	.word	0x50000400

0800062c <Error_Handler>:
/**
  * @brief  This function is executed in case of error occurrence.
  * @retval None
  */
void Error_Handler(void)
{
 800062c:	b580      	push	{r7, lr}
 800062e:	af00      	add	r7, sp, #0
  \details Disables IRQ interrupts by setting the I-bit in the CPSR.
           Can only be executed in Privileged modes.
 */
__STATIC_FORCEINLINE void __disable_irq(void)
{
  __ASM volatile ("cpsid i" : : : "memory");
 8000630:	b672      	cpsid	i
}
 8000632:	46c0      	nop			; (mov r8, r8)
  /* USER CODE BEGIN Error_Handler_Debug */
  /* User can add his own implementation to report the HAL error return state */
  __disable_irq();
  while (1)
  {
	  HAL_GPIO_WritePin(GPIOB, GPIO_PIN_5|GPIO_PIN_7, GPIO_PIN_SET);
 8000634:	4b0b      	ldr	r3, [pc, #44]	; (8000664 <Error_Handler+0x38>)
 8000636:	2201      	movs	r2, #1
 8000638:	21a0      	movs	r1, #160	; 0xa0
 800063a:	0018      	movs	r0, r3
 800063c:	f000 fb34 	bl	8000ca8 <HAL_GPIO_WritePin>
	  	  HAL_Delay(1000);
 8000640:	23fa      	movs	r3, #250	; 0xfa
 8000642:	009b      	lsls	r3, r3, #2
 8000644:	0018      	movs	r0, r3
 8000646:	f000 f8d9 	bl	80007fc <HAL_Delay>
	  	  HAL_GPIO_WritePin(GPIOB, GPIO_PIN_5|GPIO_PIN_7, GPIO_PIN_RESET);
 800064a:	4b06      	ldr	r3, [pc, #24]	; (8000664 <Error_Handler+0x38>)
 800064c:	2200      	movs	r2, #0
 800064e:	21a0      	movs	r1, #160	; 0xa0
 8000650:	0018      	movs	r0, r3
 8000652:	f000 fb29 	bl	8000ca8 <HAL_GPIO_WritePin>
	        HAL_Delay(1000);
 8000656:	23fa      	movs	r3, #250	; 0xfa
 8000658:	009b      	lsls	r3, r3, #2
 800065a:	0018      	movs	r0, r3
 800065c:	f000 f8ce 	bl	80007fc <HAL_Delay>
	  HAL_GPIO_WritePin(GPIOB, GPIO_PIN_5|GPIO_PIN_7, GPIO_PIN_SET);
 8000660:	e7e8      	b.n	8000634 <Error_Handler+0x8>
 8000662:	46c0      	nop			; (mov r8, r8)
 8000664:	50000400 	.word	0x50000400

08000668 <HAL_MspInit>:
/* USER CODE END 0 */
/**
  * Initializes the Global MSP.
  */
void HAL_MspInit(void)
{
 8000668:	b580      	push	{r7, lr}
 800066a:	af00      	add	r7, sp, #0
  /* USER CODE BEGIN MspInit 0 */

  /* USER CODE END MspInit 0 */

  __HAL_RCC_SYSCFG_CLK_ENABLE();
 800066c:	4b07      	ldr	r3, [pc, #28]	; (800068c <HAL_MspInit+0x24>)
 800066e:	6b5a      	ldr	r2, [r3, #52]	; 0x34
 8000670:	4b06      	ldr	r3, [pc, #24]	; (800068c <HAL_MspInit+0x24>)
 8000672:	2101      	movs	r1, #1
 8000674:	430a      	orrs	r2, r1
 8000676:	635a      	str	r2, [r3, #52]	; 0x34
  __HAL_RCC_PWR_CLK_ENABLE();
 8000678:	4b04      	ldr	r3, [pc, #16]	; (800068c <HAL_MspInit+0x24>)
 800067a:	6b9a      	ldr	r2, [r3, #56]	; 0x38
 800067c:	4b03      	ldr	r3, [pc, #12]	; (800068c <HAL_MspInit+0x24>)
 800067e:	2180      	movs	r1, #128	; 0x80
 8000680:	0549      	lsls	r1, r1, #21
 8000682:	430a      	orrs	r2, r1
 8000684:	639a      	str	r2, [r3, #56]	; 0x38
  /* System interrupt init*/

  /* USER CODE BEGIN MspInit 1 */

  /* USER CODE END MspInit 1 */
}
 8000686:	46c0      	nop			; (mov r8, r8)
 8000688:	46bd      	mov	sp, r7
 800068a:	bd80      	pop	{r7, pc}
 800068c:	40021000 	.word	0x40021000

08000690 <NMI_Handler>:
/******************************************************************************/
/**
  * @brief This function handles Non maskable Interrupt.
  */
void NMI_Handler(void)
{
 8000690:	b580      	push	{r7, lr}
 8000692:	af00      	add	r7, sp, #0
  /* USER CODE BEGIN NonMaskableInt_IRQn 0 */

  /* USER CODE END NonMaskableInt_IRQn 0 */
  /* USER CODE BEGIN NonMaskableInt_IRQn 1 */
  while (1)
 8000694:	e7fe      	b.n	8000694 <NMI_Handler+0x4>

08000696 <HardFault_Handler>:

/**
  * @brief This function handles Hard fault interrupt.
  */
void HardFault_Handler(void)
{
 8000696:	b580      	push	{r7, lr}
 8000698:	af00      	add	r7, sp, #0
  /* USER CODE BEGIN HardFault_IRQn 0 */

  /* USER CODE END HardFault_IRQn 0 */
  while (1)
 800069a:	e7fe      	b.n	800069a <HardFault_Handler+0x4>

0800069c <SVC_Handler>:

/**
  * @brief This function handles System service call via SWI instruction.
  */
void SVC_Handler(void)
{
 800069c:	b580      	push	{r7, lr}
 800069e:	af00      	add	r7, sp, #0

  /* USER CODE END SVC_IRQn 0 */
  /* USER CODE BEGIN SVC_IRQn 1 */

  /* USER CODE END SVC_IRQn 1 */
}
 80006a0:	46c0      	nop			; (mov r8, r8)
 80006a2:	46bd      	mov	sp, r7
 80006a4:	bd80      	pop	{r7, pc}

080006a6 <PendSV_Handler>:

/**
  * @brief This function handles Pendable request for system service.
  */
void PendSV_Handler(void)
{
 80006a6:	b580      	push	{r7, lr}
 80006a8:	af00      	add	r7, sp, #0

  /* USER CODE END PendSV_IRQn 0 */
  /* USER CODE BEGIN PendSV_IRQn 1 */

  /* USER CODE END PendSV_IRQn 1 */
}
 80006aa:	46c0      	nop			; (mov r8, r8)
 80006ac:	46bd      	mov	sp, r7
 80006ae:	bd80      	pop	{r7, pc}

080006b0 <SysTick_Handler>:

/**
  * @brief This function handles System tick timer.
  */
void SysTick_Handler(void)
{
 80006b0:	b580      	push	{r7, lr}
 80006b2:	af00      	add	r7, sp, #0
  /* USER CODE BEGIN SysTick_IRQn 0 */

  /* USER CODE END SysTick_IRQn 0 */
  HAL_IncTick();
 80006b4:	f000 f886 	bl	80007c4 <HAL_IncTick>
  /* USER CODE BEGIN SysTick_IRQn 1 */

  /* USER CODE END SysTick_IRQn 1 */
}
 80006b8:	46c0      	nop			; (mov r8, r8)
 80006ba:	46bd      	mov	sp, r7
 80006bc:	bd80      	pop	{r7, pc}

080006be <SystemInit>:
  * @brief  Setup the microcontroller system.
  * @param  None
  * @retval None
  */
void SystemInit (void)
{
 80006be:	b580      	push	{r7, lr}
 80006c0:	af00      	add	r7, sp, #0
  /* Configure the Vector Table location add offset address ------------------*/
#if defined (USER_VECT_TAB_ADDRESS)
  SCB->VTOR = VECT_TAB_BASE_ADDRESS | VECT_TAB_OFFSET; /* Vector Table Relocation in Internal SRAM */
#endif /* USER_VECT_TAB_ADDRESS */
}
 80006c2:	46c0      	nop			; (mov r8, r8)
 80006c4:	46bd      	mov	sp, r7
 80006c6:	bd80      	pop	{r7, pc}

080006c8 <Reset_Handler>:

    .section  .text.Reset_Handler
  .weak  Reset_Handler
  .type  Reset_Handler, %function
Reset_Handler:  
   ldr   r0, =_estack
 80006c8:	480d      	ldr	r0, [pc, #52]	; (8000700 <LoopForever+0x2>)
   mov   sp, r0          /* set stack pointer */
 80006ca:	4685      	mov	sp, r0
   
/* Call the clock system initialization function.*/
  bl  SystemInit
 80006cc:	f7ff fff7 	bl	80006be <SystemInit>

/* Copy the data segment initializers from flash to SRAM */
  ldr r0, =_sdata
 80006d0:	480c      	ldr	r0, [pc, #48]	; (8000704 <LoopForever+0x6>)
  ldr r1, =_edata
 80006d2:	490d      	ldr	r1, [pc, #52]	; (8000708 <LoopForever+0xa>)
  ldr r2, =_sidata
 80006d4:	4a0d      	ldr	r2, [pc, #52]	; (800070c <LoopForever+0xe>)
  movs r3, #0
 80006d6:	2300      	movs	r3, #0
  b LoopCopyDataInit
 80006d8:	e002      	b.n	80006e0 <LoopCopyDataInit>

080006da <CopyDataInit>:

CopyDataInit:
  ldr r4, [r2, r3]
 80006da:	58d4      	ldr	r4, [r2, r3]
  str r4, [r0, r3]
 80006dc:	50c4      	str	r4, [r0, r3]
  adds r3, r3, #4
 80006de:	3304      	adds	r3, #4

080006e0 <LoopCopyDataInit>:

LoopCopyDataInit:
  adds r4, r0, r3
 80006e0:	18c4      	adds	r4, r0, r3
  cmp r4, r1
 80006e2:	428c      	cmp	r4, r1
  bcc CopyDataInit
 80006e4:	d3f9      	bcc.n	80006da <CopyDataInit>
  
/* Zero fill the bss segment. */
  ldr r2, =_sbss
 80006e6:	4a0a      	ldr	r2, [pc, #40]	; (8000710 <LoopForever+0x12>)
  ldr r4, =_ebss
 80006e8:	4c0a      	ldr	r4, [pc, #40]	; (8000714 <LoopForever+0x16>)
  movs r3, #0
 80006ea:	2300      	movs	r3, #0
  b LoopFillZerobss
 80006ec:	e001      	b.n	80006f2 <LoopFillZerobss>

080006ee <FillZerobss>:

FillZerobss:
  str  r3, [r2]
 80006ee:	6013      	str	r3, [r2, #0]
  adds r2, r2, #4
 80006f0:	3204      	adds	r2, #4

080006f2 <LoopFillZerobss>:

LoopFillZerobss:
  cmp r2, r4
 80006f2:	42a2      	cmp	r2, r4
  bcc FillZerobss
 80006f4:	d3fb      	bcc.n	80006ee <FillZerobss>

/* Call static constructors */
    bl __libc_init_array
 80006f6:	f001 f8b7 	bl	8001868 <__libc_init_array>
/* Call the application's entry point.*/
  bl  main
 80006fa:	f7ff fed5 	bl	80004a8 <main>

080006fe <LoopForever>:

LoopForever:
    b LoopForever
 80006fe:	e7fe      	b.n	80006fe <LoopForever>
   ldr   r0, =_estack
 8000700:	20005000 	.word	0x20005000
  ldr r0, =_sdata
 8000704:	20000000 	.word	0x20000000
  ldr r1, =_edata
 8000708:	2000000c 	.word	0x2000000c
  ldr r2, =_sidata
 800070c:	08001904 	.word	0x08001904
  ldr r2, =_sbss
 8000710:	2000000c 	.word	0x2000000c
  ldr r4, =_ebss
 8000714:	2000002c 	.word	0x2000002c

08000718 <ADC1_COMP_IRQHandler>:
 * @retval : None
*/
    .section  .text.Default_Handler,"ax",%progbits
Default_Handler:
Infinite_Loop:
  b  Infinite_Loop
 8000718:	e7fe      	b.n	8000718 <ADC1_COMP_IRQHandler>
	...

0800071c <HAL_Init>:
  *        In the default implementation,Systick is used as source of time base.
  *        the tick variable is incremented each 1ms in its ISR.
  * @retval HAL status
  */
HAL_StatusTypeDef HAL_Init(void)
{
 800071c:	b580      	push	{r7, lr}
 800071e:	b082      	sub	sp, #8
 8000720:	af00      	add	r7, sp, #0
  HAL_StatusTypeDef  status = HAL_OK;
 8000722:	1dfb      	adds	r3, r7, #7
 8000724:	2200      	movs	r2, #0
 8000726:	701a      	strb	r2, [r3, #0]
#if (BUFFER_CACHE_DISABLE != 0)
  __HAL_FLASH_BUFFER_CACHE_DISABLE();
#endif /* BUFFER_CACHE_DISABLE */

#if (PREREAD_ENABLE != 0)
  __HAL_FLASH_PREREAD_BUFFER_ENABLE();
 8000728:	4b0b      	ldr	r3, [pc, #44]	; (8000758 <HAL_Init+0x3c>)
 800072a:	681a      	ldr	r2, [r3, #0]
 800072c:	4b0a      	ldr	r3, [pc, #40]	; (8000758 <HAL_Init+0x3c>)
 800072e:	2140      	movs	r1, #64	; 0x40
 8000730:	430a      	orrs	r2, r1
 8000732:	601a      	str	r2, [r3, #0]
#if (PREFETCH_ENABLE != 0)
  __HAL_FLASH_PREFETCH_BUFFER_ENABLE();
#endif /* PREFETCH_ENABLE */

  /* Use SysTick as time base source and configure 1ms tick (default clock after Reset is MSI) */
  if (HAL_InitTick(TICK_INT_PRIORITY) != HAL_OK)
 8000734:	2000      	movs	r0, #0
 8000736:	f000 f811 	bl	800075c <HAL_InitTick>
 800073a:	1e03      	subs	r3, r0, #0
 800073c:	d003      	beq.n	8000746 <HAL_Init+0x2a>
  {
    status = HAL_ERROR;
 800073e:	1dfb      	adds	r3, r7, #7
 8000740:	2201      	movs	r2, #1
 8000742:	701a      	strb	r2, [r3, #0]
 8000744:	e001      	b.n	800074a <HAL_Init+0x2e>
  }
  else
  {
    /* Init the low level hardware */
    HAL_MspInit();
 8000746:	f7ff ff8f 	bl	8000668 <HAL_MspInit>
  }

  /* Return function status */
  return status;
 800074a:	1dfb      	adds	r3, r7, #7
 800074c:	781b      	ldrb	r3, [r3, #0]
}
 800074e:	0018      	movs	r0, r3
 8000750:	46bd      	mov	sp, r7
 8000752:	b002      	add	sp, #8
 8000754:	bd80      	pop	{r7, pc}
 8000756:	46c0      	nop			; (mov r8, r8)
 8000758:	40022000 	.word	0x40022000

0800075c <HAL_InitTick>:
  *       implementation  in user file.
  * @param TickPriority Tick interrupt priority.
  * @retval HAL status
  */
__weak HAL_StatusTypeDef HAL_InitTick(uint32_t TickPriority)
{
 800075c:	b590      	push	{r4, r7, lr}
 800075e:	b083      	sub	sp, #12
 8000760:	af00      	add	r7, sp, #0
 8000762:	6078      	str	r0, [r7, #4]
  /* Configure the SysTick to have interrupt in 1ms time basis*/
  if (HAL_SYSTICK_Config(SystemCoreClock / (1000U / uwTickFreq)) > 0U)
 8000764:	4b14      	ldr	r3, [pc, #80]	; (80007b8 <HAL_InitTick+0x5c>)
 8000766:	681c      	ldr	r4, [r3, #0]
 8000768:	4b14      	ldr	r3, [pc, #80]	; (80007bc <HAL_InitTick+0x60>)
 800076a:	781b      	ldrb	r3, [r3, #0]
 800076c:	0019      	movs	r1, r3
 800076e:	23fa      	movs	r3, #250	; 0xfa
 8000770:	0098      	lsls	r0, r3, #2
 8000772:	f7ff fcc9 	bl	8000108 <__udivsi3>
 8000776:	0003      	movs	r3, r0
 8000778:	0019      	movs	r1, r3
 800077a:	0020      	movs	r0, r4
 800077c:	f7ff fcc4 	bl	8000108 <__udivsi3>
 8000780:	0003      	movs	r3, r0
 8000782:	0018      	movs	r0, r3
 8000784:	f000 f905 	bl	8000992 <HAL_SYSTICK_Config>
 8000788:	1e03      	subs	r3, r0, #0
 800078a:	d001      	beq.n	8000790 <HAL_InitTick+0x34>
  {
    return HAL_ERROR;
 800078c:	2301      	movs	r3, #1
 800078e:	e00f      	b.n	80007b0 <HAL_InitTick+0x54>
  }

  /* Configure the SysTick IRQ priority */
  if (TickPriority < (1UL << __NVIC_PRIO_BITS))
 8000790:	687b      	ldr	r3, [r7, #4]
 8000792:	2b03      	cmp	r3, #3
 8000794:	d80b      	bhi.n	80007ae <HAL_InitTick+0x52>
  {
    HAL_NVIC_SetPriority(SysTick_IRQn, TickPriority, 0U);
 8000796:	6879      	ldr	r1, [r7, #4]
 8000798:	2301      	movs	r3, #1
 800079a:	425b      	negs	r3, r3
 800079c:	2200      	movs	r2, #0
 800079e:	0018      	movs	r0, r3
 80007a0:	f000 f8e2 	bl	8000968 <HAL_NVIC_SetPriority>
    uwTickPrio = TickPriority;
 80007a4:	4b06      	ldr	r3, [pc, #24]	; (80007c0 <HAL_InitTick+0x64>)
 80007a6:	687a      	ldr	r2, [r7, #4]
 80007a8:	601a      	str	r2, [r3, #0]
  {
    return HAL_ERROR;
  }

  /* Return function status */
  return HAL_OK;
 80007aa:	2300      	movs	r3, #0
 80007ac:	e000      	b.n	80007b0 <HAL_InitTick+0x54>
    return HAL_ERROR;
 80007ae:	2301      	movs	r3, #1
}
 80007b0:	0018      	movs	r0, r3
 80007b2:	46bd      	mov	sp, r7
 80007b4:	b003      	add	sp, #12
 80007b6:	bd90      	pop	{r4, r7, pc}
 80007b8:	20000000 	.word	0x20000000
 80007bc:	20000008 	.word	0x20000008
 80007c0:	20000004 	.word	0x20000004

080007c4 <HAL_IncTick>:
 * @note This function is declared as __weak to be overwritten in case of other
  *      implementations in user file.
  * @retval None
  */
__weak void HAL_IncTick(void)
{
 80007c4:	b580      	push	{r7, lr}
 80007c6:	af00      	add	r7, sp, #0
  uwTick += uwTickFreq;
 80007c8:	4b05      	ldr	r3, [pc, #20]	; (80007e0 <HAL_IncTick+0x1c>)
 80007ca:	781b      	ldrb	r3, [r3, #0]
 80007cc:	001a      	movs	r2, r3
 80007ce:	4b05      	ldr	r3, [pc, #20]	; (80007e4 <HAL_IncTick+0x20>)
 80007d0:	681b      	ldr	r3, [r3, #0]
 80007d2:	18d2      	adds	r2, r2, r3
 80007d4:	4b03      	ldr	r3, [pc, #12]	; (80007e4 <HAL_IncTick+0x20>)
 80007d6:	601a      	str	r2, [r3, #0]
}
 80007d8:	46c0      	nop			; (mov r8, r8)
 80007da:	46bd      	mov	sp, r7
 80007dc:	bd80      	pop	{r7, pc}
 80007de:	46c0      	nop			; (mov r8, r8)
 80007e0:	20000008 	.word	0x20000008
 80007e4:	20000028 	.word	0x20000028

080007e8 <HAL_GetTick>:
  * @note This function is declared as __weak to be overwritten in case of other
  *       implementations in user file.
  * @retval tick value
  */
__weak uint32_t HAL_GetTick(void)
{
 80007e8:	b580      	push	{r7, lr}
 80007ea:	af00      	add	r7, sp, #0
  return uwTick;
 80007ec:	4b02      	ldr	r3, [pc, #8]	; (80007f8 <HAL_GetTick+0x10>)
 80007ee:	681b      	ldr	r3, [r3, #0]
}
 80007f0:	0018      	movs	r0, r3
 80007f2:	46bd      	mov	sp, r7
 80007f4:	bd80      	pop	{r7, pc}
 80007f6:	46c0      	nop			; (mov r8, r8)
 80007f8:	20000028 	.word	0x20000028

080007fc <HAL_Delay>:
  *       implementations in user file.
  * @param Delay specifies the delay time length, in milliseconds.
  * @retval None
  */
__weak void HAL_Delay(uint32_t Delay)
{
 80007fc:	b580      	push	{r7, lr}
 80007fe:	b084      	sub	sp, #16
 8000800:	af00      	add	r7, sp, #0
 8000802:	6078      	str	r0, [r7, #4]
  uint32_t tickstart = HAL_GetTick();
 8000804:	f7ff fff0 	bl	80007e8 <HAL_GetTick>
 8000808:	0003      	movs	r3, r0
 800080a:	60bb      	str	r3, [r7, #8]
  uint32_t wait = Delay;
 800080c:	687b      	ldr	r3, [r7, #4]
 800080e:	60fb      	str	r3, [r7, #12]

  /* Add a freq to guarantee minimum wait */
  if (wait < HAL_MAX_DELAY)
 8000810:	68fb      	ldr	r3, [r7, #12]
 8000812:	3301      	adds	r3, #1
 8000814:	d005      	beq.n	8000822 <HAL_Delay+0x26>
  {
    wait += (uint32_t)(uwTickFreq);
 8000816:	4b0a      	ldr	r3, [pc, #40]	; (8000840 <HAL_Delay+0x44>)
 8000818:	781b      	ldrb	r3, [r3, #0]
 800081a:	001a      	movs	r2, r3
 800081c:	68fb      	ldr	r3, [r7, #12]
 800081e:	189b      	adds	r3, r3, r2
 8000820:	60fb      	str	r3, [r7, #12]
  }

  while((HAL_GetTick() - tickstart) < wait)
 8000822:	46c0      	nop			; (mov r8, r8)
 8000824:	f7ff ffe0 	bl	80007e8 <HAL_GetTick>
 8000828:	0002      	movs	r2, r0
 800082a:	68bb      	ldr	r3, [r7, #8]
 800082c:	1ad3      	subs	r3, r2, r3
 800082e:	68fa      	ldr	r2, [r7, #12]
 8000830:	429a      	cmp	r2, r3
 8000832:	d8f7      	bhi.n	8000824 <HAL_Delay+0x28>
  {
  }
}
 8000834:	46c0      	nop			; (mov r8, r8)
 8000836:	46c0      	nop			; (mov r8, r8)
 8000838:	46bd      	mov	sp, r7
 800083a:	b004      	add	sp, #16
 800083c:	bd80      	pop	{r7, pc}
 800083e:	46c0      	nop			; (mov r8, r8)
 8000840:	20000008 	.word	0x20000008

08000844 <__NVIC_SetPriority>:
  \param [in]      IRQn  Interrupt number.
  \param [in]  priority  Priority to set.
  \note    The priority cannot be set for every processor exception.
 */
__STATIC_INLINE void __NVIC_SetPriority(IRQn_Type IRQn, uint32_t priority)
{
 8000844:	b590      	push	{r4, r7, lr}
 8000846:	b083      	sub	sp, #12
 8000848:	af00      	add	r7, sp, #0
 800084a:	0002      	movs	r2, r0
 800084c:	6039      	str	r1, [r7, #0]
 800084e:	1dfb      	adds	r3, r7, #7
 8000850:	701a      	strb	r2, [r3, #0]
  if ((int32_t)(IRQn) >= 0)
 8000852:	1dfb      	adds	r3, r7, #7
 8000854:	781b      	ldrb	r3, [r3, #0]
 8000856:	2b7f      	cmp	r3, #127	; 0x7f
 8000858:	d828      	bhi.n	80008ac <__NVIC_SetPriority+0x68>
  {
    NVIC->IP[_IP_IDX(IRQn)]  = ((uint32_t)(NVIC->IP[_IP_IDX(IRQn)]  & ~(0xFFUL << _BIT_SHIFT(IRQn))) |
 800085a:	4a2f      	ldr	r2, [pc, #188]	; (8000918 <__NVIC_SetPriority+0xd4>)
 800085c:	1dfb      	adds	r3, r7, #7
 800085e:	781b      	ldrb	r3, [r3, #0]
 8000860:	b25b      	sxtb	r3, r3
 8000862:	089b      	lsrs	r3, r3, #2
 8000864:	33c0      	adds	r3, #192	; 0xc0
 8000866:	009b      	lsls	r3, r3, #2
 8000868:	589b      	ldr	r3, [r3, r2]
 800086a:	1dfa      	adds	r2, r7, #7
 800086c:	7812      	ldrb	r2, [r2, #0]
 800086e:	0011      	movs	r1, r2
 8000870:	2203      	movs	r2, #3
 8000872:	400a      	ands	r2, r1
 8000874:	00d2      	lsls	r2, r2, #3
 8000876:	21ff      	movs	r1, #255	; 0xff
 8000878:	4091      	lsls	r1, r2
 800087a:	000a      	movs	r2, r1
 800087c:	43d2      	mvns	r2, r2
 800087e:	401a      	ands	r2, r3
 8000880:	0011      	movs	r1, r2
       (((priority << (8U - __NVIC_PRIO_BITS)) & (uint32_t)0xFFUL) << _BIT_SHIFT(IRQn)));
 8000882:	683b      	ldr	r3, [r7, #0]
 8000884:	019b      	lsls	r3, r3, #6
 8000886:	22ff      	movs	r2, #255	; 0xff
 8000888:	401a      	ands	r2, r3
 800088a:	1dfb      	adds	r3, r7, #7
 800088c:	781b      	ldrb	r3, [r3, #0]
 800088e:	0018      	movs	r0, r3
 8000890:	2303      	movs	r3, #3
 8000892:	4003      	ands	r3, r0
 8000894:	00db      	lsls	r3, r3, #3
 8000896:	409a      	lsls	r2, r3
    NVIC->IP[_IP_IDX(IRQn)]  = ((uint32_t)(NVIC->IP[_IP_IDX(IRQn)]  & ~(0xFFUL << _BIT_SHIFT(IRQn))) |
 8000898:	481f      	ldr	r0, [pc, #124]	; (8000918 <__NVIC_SetPriority+0xd4>)
 800089a:	1dfb      	adds	r3, r7, #7
 800089c:	781b      	ldrb	r3, [r3, #0]
 800089e:	b25b      	sxtb	r3, r3
 80008a0:	089b      	lsrs	r3, r3, #2
 80008a2:	430a      	orrs	r2, r1
 80008a4:	33c0      	adds	r3, #192	; 0xc0
 80008a6:	009b      	lsls	r3, r3, #2
 80008a8:	501a      	str	r2, [r3, r0]
  else
  {
    SCB->SHP[_SHP_IDX(IRQn)] = ((uint32_t)(SCB->SHP[_SHP_IDX(IRQn)] & ~(0xFFUL << _BIT_SHIFT(IRQn))) |
       (((priority << (8U - __NVIC_PRIO_BITS)) & (uint32_t)0xFFUL) << _BIT_SHIFT(IRQn)));
  }
}
 80008aa:	e031      	b.n	8000910 <__NVIC_SetPriority+0xcc>
    SCB->SHP[_SHP_IDX(IRQn)] = ((uint32_t)(SCB->SHP[_SHP_IDX(IRQn)] & ~(0xFFUL << _BIT_SHIFT(IRQn))) |
 80008ac:	4a1b      	ldr	r2, [pc, #108]	; (800091c <__NVIC_SetPriority+0xd8>)
 80008ae:	1dfb      	adds	r3, r7, #7
 80008b0:	781b      	ldrb	r3, [r3, #0]
 80008b2:	0019      	movs	r1, r3
 80008b4:	230f      	movs	r3, #15
 80008b6:	400b      	ands	r3, r1
 80008b8:	3b08      	subs	r3, #8
 80008ba:	089b      	lsrs	r3, r3, #2
 80008bc:	3306      	adds	r3, #6
 80008be:	009b      	lsls	r3, r3, #2
 80008c0:	18d3      	adds	r3, r2, r3
 80008c2:	3304      	adds	r3, #4
 80008c4:	681b      	ldr	r3, [r3, #0]
 80008c6:	1dfa      	adds	r2, r7, #7
 80008c8:	7812      	ldrb	r2, [r2, #0]
 80008ca:	0011      	movs	r1, r2
 80008cc:	2203      	movs	r2, #3
 80008ce:	400a      	ands	r2, r1
 80008d0:	00d2      	lsls	r2, r2, #3
 80008d2:	21ff      	movs	r1, #255	; 0xff
 80008d4:	4091      	lsls	r1, r2
 80008d6:	000a      	movs	r2, r1
 80008d8:	43d2      	mvns	r2, r2
 80008da:	401a      	ands	r2, r3
 80008dc:	0011      	movs	r1, r2
       (((priority << (8U - __NVIC_PRIO_BITS)) & (uint32_t)0xFFUL) << _BIT_SHIFT(IRQn)));
 80008de:	683b      	ldr	r3, [r7, #0]
 80008e0:	019b      	lsls	r3, r3, #6
 80008e2:	22ff      	movs	r2, #255	; 0xff
 80008e4:	401a      	ands	r2, r3
 80008e6:	1dfb      	adds	r3, r7, #7
 80008e8:	781b      	ldrb	r3, [r3, #0]
 80008ea:	0018      	movs	r0, r3
 80008ec:	2303      	movs	r3, #3
 80008ee:	4003      	ands	r3, r0
 80008f0:	00db      	lsls	r3, r3, #3
 80008f2:	409a      	lsls	r2, r3
    SCB->SHP[_SHP_IDX(IRQn)] = ((uint32_t)(SCB->SHP[_SHP_IDX(IRQn)] & ~(0xFFUL << _BIT_SHIFT(IRQn))) |
 80008f4:	4809      	ldr	r0, [pc, #36]	; (800091c <__NVIC_SetPriority+0xd8>)
 80008f6:	1dfb      	adds	r3, r7, #7
 80008f8:	781b      	ldrb	r3, [r3, #0]
 80008fa:	001c      	movs	r4, r3
 80008fc:	230f      	movs	r3, #15
 80008fe:	4023      	ands	r3, r4
 8000900:	3b08      	subs	r3, #8
 8000902:	089b      	lsrs	r3, r3, #2
 8000904:	430a      	orrs	r2, r1
 8000906:	3306      	adds	r3, #6
 8000908:	009b      	lsls	r3, r3, #2
 800090a:	18c3      	adds	r3, r0, r3
 800090c:	3304      	adds	r3, #4
 800090e:	601a      	str	r2, [r3, #0]
}
 8000910:	46c0      	nop			; (mov r8, r8)
 8000912:	46bd      	mov	sp, r7
 8000914:	b003      	add	sp, #12
 8000916:	bd90      	pop	{r4, r7, pc}
 8000918:	e000e100 	.word	0xe000e100
 800091c:	e000ed00 	.word	0xe000ed00

08000920 <SysTick_Config>:
  \note    When the variable <b>__Vendor_SysTickConfig</b> is set to 1, then the
           function <b>SysTick_Config</b> is not included. In this case, the file <b><i>device</i>.h</b>
           must contain a vendor-specific implementation of this function.
 */
__STATIC_INLINE uint32_t SysTick_Config(uint32_t ticks)
{
 8000920:	b580      	push	{r7, lr}
 8000922:	b082      	sub	sp, #8
 8000924:	af00      	add	r7, sp, #0
 8000926:	6078      	str	r0, [r7, #4]
  if ((ticks - 1UL) > SysTick_LOAD_RELOAD_Msk)
 8000928:	687b      	ldr	r3, [r7, #4]
 800092a:	1e5a      	subs	r2, r3, #1
 800092c:	2380      	movs	r3, #128	; 0x80
 800092e:	045b      	lsls	r3, r3, #17
 8000930:	429a      	cmp	r2, r3
 8000932:	d301      	bcc.n	8000938 <SysTick_Config+0x18>
  {
    return (1UL);                                                   /* Reload value impossible */
 8000934:	2301      	movs	r3, #1
 8000936:	e010      	b.n	800095a <SysTick_Config+0x3a>
  }

  SysTick->LOAD  = (uint32_t)(ticks - 1UL);                         /* set reload register */
 8000938:	4b0a      	ldr	r3, [pc, #40]	; (8000964 <SysTick_Config+0x44>)
 800093a:	687a      	ldr	r2, [r7, #4]
 800093c:	3a01      	subs	r2, #1
 800093e:	605a      	str	r2, [r3, #4]
  NVIC_SetPriority (SysTick_IRQn, (1UL << __NVIC_PRIO_BITS) - 1UL); /* set Priority for Systick Interrupt */
 8000940:	2301      	movs	r3, #1
 8000942:	425b      	negs	r3, r3
 8000944:	2103      	movs	r1, #3
 8000946:	0018      	movs	r0, r3
 8000948:	f7ff ff7c 	bl	8000844 <__NVIC_SetPriority>
  SysTick->VAL   = 0UL;                                             /* Load the SysTick Counter Value */
 800094c:	4b05      	ldr	r3, [pc, #20]	; (8000964 <SysTick_Config+0x44>)
 800094e:	2200      	movs	r2, #0
 8000950:	609a      	str	r2, [r3, #8]
  SysTick->CTRL  = SysTick_CTRL_CLKSOURCE_Msk |
 8000952:	4b04      	ldr	r3, [pc, #16]	; (8000964 <SysTick_Config+0x44>)
 8000954:	2207      	movs	r2, #7
 8000956:	601a      	str	r2, [r3, #0]
                   SysTick_CTRL_TICKINT_Msk   |
                   SysTick_CTRL_ENABLE_Msk;                         /* Enable SysTick IRQ and SysTick Timer */
  return (0UL);                                                     /* Function successful */
 8000958:	2300      	movs	r3, #0
}
 800095a:	0018      	movs	r0, r3
 800095c:	46bd      	mov	sp, r7
 800095e:	b002      	add	sp, #8
 8000960:	bd80      	pop	{r7, pc}
 8000962:	46c0      	nop			; (mov r8, r8)
 8000964:	e000e010 	.word	0xe000e010

08000968 <HAL_NVIC_SetPriority>:
  *         with stm32l0xx devices, this parameter is a dummy value and it is ignored, because 
  *         no subpriority supported in Cortex M0+ based products.   
  * @retval None
  */
void HAL_NVIC_SetPriority(IRQn_Type IRQn, uint32_t PreemptPriority, uint32_t SubPriority)
{ 
 8000968:	b580      	push	{r7, lr}
 800096a:	b084      	sub	sp, #16
 800096c:	af00      	add	r7, sp, #0
 800096e:	60b9      	str	r1, [r7, #8]
 8000970:	607a      	str	r2, [r7, #4]
 8000972:	210f      	movs	r1, #15
 8000974:	187b      	adds	r3, r7, r1
 8000976:	1c02      	adds	r2, r0, #0
 8000978:	701a      	strb	r2, [r3, #0]
    /* Check the parameters */
  assert_param(IS_NVIC_PREEMPTION_PRIORITY(PreemptPriority));
  NVIC_SetPriority(IRQn,PreemptPriority);
 800097a:	68ba      	ldr	r2, [r7, #8]
 800097c:	187b      	adds	r3, r7, r1
 800097e:	781b      	ldrb	r3, [r3, #0]
 8000980:	b25b      	sxtb	r3, r3
 8000982:	0011      	movs	r1, r2
 8000984:	0018      	movs	r0, r3
 8000986:	f7ff ff5d 	bl	8000844 <__NVIC_SetPriority>
}
 800098a:	46c0      	nop			; (mov r8, r8)
 800098c:	46bd      	mov	sp, r7
 800098e:	b004      	add	sp, #16
 8000990:	bd80      	pop	{r7, pc}

08000992 <HAL_SYSTICK_Config>:
  * @param  TicksNumb Specifies the ticks Number of ticks between two interrupts.
  * @retval status:  - 0  Function succeeded.
  *                  - 1  Function failed.
  */
uint32_t HAL_SYSTICK_Config(uint32_t TicksNumb)
{
 8000992:	b580      	push	{r7, lr}
 8000994:	b082      	sub	sp, #8
 8000996:	af00      	add	r7, sp, #0
 8000998:	6078      	str	r0, [r7, #4]
   return SysTick_Config(TicksNumb);
 800099a:	687b      	ldr	r3, [r7, #4]
 800099c:	0018      	movs	r0, r3
 800099e:	f7ff ffbf 	bl	8000920 <SysTick_Config>
 80009a2:	0003      	movs	r3, r0
}
 80009a4:	0018      	movs	r0, r3
 80009a6:	46bd      	mov	sp, r7
 80009a8:	b002      	add	sp, #8
 80009aa:	bd80      	pop	{r7, pc}

080009ac <HAL_GPIO_Init>:
  * @param  GPIO_Init pointer to a GPIO_InitTypeDef structure that contains
  *                    the configuration information for the specified GPIO peripheral.
  * @retval None
  */
void HAL_GPIO_Init(GPIO_TypeDef  *GPIOx, GPIO_InitTypeDef *GPIO_Init)
{
 80009ac:	b580      	push	{r7, lr}
 80009ae:	b086      	sub	sp, #24
 80009b0:	af00      	add	r7, sp, #0
 80009b2:	6078      	str	r0, [r7, #4]
 80009b4:	6039      	str	r1, [r7, #0]
  uint32_t position = 0x00U;
 80009b6:	2300      	movs	r3, #0
 80009b8:	617b      	str	r3, [r7, #20]
  uint32_t iocurrent = 0x00U;
 80009ba:	2300      	movs	r3, #0
 80009bc:	60fb      	str	r3, [r7, #12]
  uint32_t temp = 0x00U;
 80009be:	2300      	movs	r3, #0
 80009c0:	613b      	str	r3, [r7, #16]
  /* Check the parameters */
  assert_param(IS_GPIO_MODE(GPIO_Init->Mode));
  assert_param(IS_GPIO_PIN_AVAILABLE(GPIOx, (GPIO_Init->Pin)));

  /* Configure the port pins */
  while (((GPIO_Init->Pin) >> position) != 0)
 80009c2:	e155      	b.n	8000c70 <HAL_GPIO_Init+0x2c4>
  {
    /* Get the IO position */
    iocurrent = (GPIO_Init->Pin) & (1U << position);
 80009c4:	683b      	ldr	r3, [r7, #0]
 80009c6:	681b      	ldr	r3, [r3, #0]
 80009c8:	2101      	movs	r1, #1
 80009ca:	697a      	ldr	r2, [r7, #20]
 80009cc:	4091      	lsls	r1, r2
 80009ce:	000a      	movs	r2, r1
 80009d0:	4013      	ands	r3, r2
 80009d2:	60fb      	str	r3, [r7, #12]

    if (iocurrent)
 80009d4:	68fb      	ldr	r3, [r7, #12]
 80009d6:	2b00      	cmp	r3, #0
 80009d8:	d100      	bne.n	80009dc <HAL_GPIO_Init+0x30>
 80009da:	e146      	b.n	8000c6a <HAL_GPIO_Init+0x2be>
    {
      /*--------------------- GPIO Mode Configuration ------------------------*/
      /* In case of Output or Alternate function mode selection */
      if (((GPIO_Init->Mode & GPIO_MODE) == MODE_OUTPUT) ||
 80009dc:	683b      	ldr	r3, [r7, #0]
 80009de:	685b      	ldr	r3, [r3, #4]
 80009e0:	2203      	movs	r2, #3
 80009e2:	4013      	ands	r3, r2
 80009e4:	2b01      	cmp	r3, #1
 80009e6:	d005      	beq.n	80009f4 <HAL_GPIO_Init+0x48>
          ((GPIO_Init->Mode & GPIO_MODE) == MODE_AF))
 80009e8:	683b      	ldr	r3, [r7, #0]
 80009ea:	685b      	ldr	r3, [r3, #4]
 80009ec:	2203      	movs	r2, #3
 80009ee:	4013      	ands	r3, r2
      if (((GPIO_Init->Mode & GPIO_MODE) == MODE_OUTPUT) ||
 80009f0:	2b02      	cmp	r3, #2
 80009f2:	d130      	bne.n	8000a56 <HAL_GPIO_Init+0xaa>
      {
        /* Check the Speed parameter */
        assert_param(IS_GPIO_SPEED(GPIO_Init->Speed));
        /* Configure the IO Speed */
        temp = GPIOx->OSPEEDR;
 80009f4:	687b      	ldr	r3, [r7, #4]
 80009f6:	689b      	ldr	r3, [r3, #8]
 80009f8:	613b      	str	r3, [r7, #16]
        temp &= ~(GPIO_OSPEEDER_OSPEED0 << (position * 2U));
 80009fa:	697b      	ldr	r3, [r7, #20]
 80009fc:	005b      	lsls	r3, r3, #1
 80009fe:	2203      	movs	r2, #3
 8000a00:	409a      	lsls	r2, r3
 8000a02:	0013      	movs	r3, r2
 8000a04:	43da      	mvns	r2, r3
 8000a06:	693b      	ldr	r3, [r7, #16]
 8000a08:	4013      	ands	r3, r2
 8000a0a:	613b      	str	r3, [r7, #16]
        temp |= (GPIO_Init->Speed << (position * 2U));
 8000a0c:	683b      	ldr	r3, [r7, #0]
 8000a0e:	68da      	ldr	r2, [r3, #12]
 8000a10:	697b      	ldr	r3, [r7, #20]
 8000a12:	005b      	lsls	r3, r3, #1
 8000a14:	409a      	lsls	r2, r3
 8000a16:	0013      	movs	r3, r2
 8000a18:	693a      	ldr	r2, [r7, #16]
 8000a1a:	4313      	orrs	r3, r2
 8000a1c:	613b      	str	r3, [r7, #16]
        GPIOx->OSPEEDR = temp;
 8000a1e:	687b      	ldr	r3, [r7, #4]
 8000a20:	693a      	ldr	r2, [r7, #16]
 8000a22:	609a      	str	r2, [r3, #8]

        /* Configure the IO Output Type */
        temp = GPIOx->OTYPER;
 8000a24:	687b      	ldr	r3, [r7, #4]
 8000a26:	685b      	ldr	r3, [r3, #4]
 8000a28:	613b      	str	r3, [r7, #16]
        temp &= ~(GPIO_OTYPER_OT_0 << position) ;
 8000a2a:	2201      	movs	r2, #1
 8000a2c:	697b      	ldr	r3, [r7, #20]
 8000a2e:	409a      	lsls	r2, r3
 8000a30:	0013      	movs	r3, r2
 8000a32:	43da      	mvns	r2, r3
 8000a34:	693b      	ldr	r3, [r7, #16]
 8000a36:	4013      	ands	r3, r2
 8000a38:	613b      	str	r3, [r7, #16]
        temp |= (((GPIO_Init->Mode & OUTPUT_TYPE) >> OUTPUT_TYPE_Pos) << position);
 8000a3a:	683b      	ldr	r3, [r7, #0]
 8000a3c:	685b      	ldr	r3, [r3, #4]
 8000a3e:	091b      	lsrs	r3, r3, #4
 8000a40:	2201      	movs	r2, #1
 8000a42:	401a      	ands	r2, r3
 8000a44:	697b      	ldr	r3, [r7, #20]
 8000a46:	409a      	lsls	r2, r3
 8000a48:	0013      	movs	r3, r2
 8000a4a:	693a      	ldr	r2, [r7, #16]
 8000a4c:	4313      	orrs	r3, r2
 8000a4e:	613b      	str	r3, [r7, #16]
        GPIOx->OTYPER = temp;
 8000a50:	687b      	ldr	r3, [r7, #4]
 8000a52:	693a      	ldr	r2, [r7, #16]
 8000a54:	605a      	str	r2, [r3, #4]
      }

      if ((GPIO_Init->Mode & GPIO_MODE) != MODE_ANALOG)
 8000a56:	683b      	ldr	r3, [r7, #0]
 8000a58:	685b      	ldr	r3, [r3, #4]
 8000a5a:	2203      	movs	r2, #3
 8000a5c:	4013      	ands	r3, r2
 8000a5e:	2b03      	cmp	r3, #3
 8000a60:	d017      	beq.n	8000a92 <HAL_GPIO_Init+0xe6>
      {
        /* Check the Pull parameter */
        assert_param(IS_GPIO_PULL(GPIO_Init->Pull));

        /* Activate the Pull-up or Pull down resistor for the current IO */
        temp = GPIOx->PUPDR;
 8000a62:	687b      	ldr	r3, [r7, #4]
 8000a64:	68db      	ldr	r3, [r3, #12]
 8000a66:	613b      	str	r3, [r7, #16]
        temp &= ~(GPIO_PUPDR_PUPD0 << (position * 2U));
 8000a68:	697b      	ldr	r3, [r7, #20]
 8000a6a:	005b      	lsls	r3, r3, #1
 8000a6c:	2203      	movs	r2, #3
 8000a6e:	409a      	lsls	r2, r3
 8000a70:	0013      	movs	r3, r2
 8000a72:	43da      	mvns	r2, r3
 8000a74:	693b      	ldr	r3, [r7, #16]
 8000a76:	4013      	ands	r3, r2
 8000a78:	613b      	str	r3, [r7, #16]
        temp |= ((GPIO_Init->Pull) << (position * 2U));
 8000a7a:	683b      	ldr	r3, [r7, #0]
 8000a7c:	689a      	ldr	r2, [r3, #8]
 8000a7e:	697b      	ldr	r3, [r7, #20]
 8000a80:	005b      	lsls	r3, r3, #1
 8000a82:	409a      	lsls	r2, r3
 8000a84:	0013      	movs	r3, r2
 8000a86:	693a      	ldr	r2, [r7, #16]
 8000a88:	4313      	orrs	r3, r2
 8000a8a:	613b      	str	r3, [r7, #16]
        GPIOx->PUPDR = temp;
 8000a8c:	687b      	ldr	r3, [r7, #4]
 8000a8e:	693a      	ldr	r2, [r7, #16]
 8000a90:	60da      	str	r2, [r3, #12]
      }

      /* In case of Alternate function mode selection */
      if ((GPIO_Init->Mode & GPIO_MODE) == MODE_AF)
 8000a92:	683b      	ldr	r3, [r7, #0]
 8000a94:	685b      	ldr	r3, [r3, #4]
 8000a96:	2203      	movs	r2, #3
 8000a98:	4013      	ands	r3, r2
 8000a9a:	2b02      	cmp	r3, #2
 8000a9c:	d123      	bne.n	8000ae6 <HAL_GPIO_Init+0x13a>
        /* Check the Alternate function parameters */
        assert_param(IS_GPIO_AF_INSTANCE(GPIOx));
        assert_param(IS_GPIO_AF(GPIO_Init->Alternate));

        /* Configure Alternate function mapped with the current IO */
        temp = GPIOx->AFR[position >> 3U];
 8000a9e:	697b      	ldr	r3, [r7, #20]
 8000aa0:	08da      	lsrs	r2, r3, #3
 8000aa2:	687b      	ldr	r3, [r7, #4]
 8000aa4:	3208      	adds	r2, #8
 8000aa6:	0092      	lsls	r2, r2, #2
 8000aa8:	58d3      	ldr	r3, [r2, r3]
 8000aaa:	613b      	str	r3, [r7, #16]
        temp &= ~(0xFUL << ((uint32_t)(position & 0x07UL) * 4U));
 8000aac:	697b      	ldr	r3, [r7, #20]
 8000aae:	2207      	movs	r2, #7
 8000ab0:	4013      	ands	r3, r2
 8000ab2:	009b      	lsls	r3, r3, #2
 8000ab4:	220f      	movs	r2, #15
 8000ab6:	409a      	lsls	r2, r3
 8000ab8:	0013      	movs	r3, r2
 8000aba:	43da      	mvns	r2, r3
 8000abc:	693b      	ldr	r3, [r7, #16]
 8000abe:	4013      	ands	r3, r2
 8000ac0:	613b      	str	r3, [r7, #16]
        temp |= ((uint32_t)(GPIO_Init->Alternate) << (((uint32_t)position & (uint32_t)0x07U) * 4U));
 8000ac2:	683b      	ldr	r3, [r7, #0]
 8000ac4:	691a      	ldr	r2, [r3, #16]
 8000ac6:	697b      	ldr	r3, [r7, #20]
 8000ac8:	2107      	movs	r1, #7
 8000aca:	400b      	ands	r3, r1
 8000acc:	009b      	lsls	r3, r3, #2
 8000ace:	409a      	lsls	r2, r3
 8000ad0:	0013      	movs	r3, r2
 8000ad2:	693a      	ldr	r2, [r7, #16]
 8000ad4:	4313      	orrs	r3, r2
 8000ad6:	613b      	str	r3, [r7, #16]
        GPIOx->AFR[position >> 3U] = temp;
 8000ad8:	697b      	ldr	r3, [r7, #20]
 8000ada:	08da      	lsrs	r2, r3, #3
 8000adc:	687b      	ldr	r3, [r7, #4]
 8000ade:	3208      	adds	r2, #8
 8000ae0:	0092      	lsls	r2, r2, #2
 8000ae2:	6939      	ldr	r1, [r7, #16]
 8000ae4:	50d1      	str	r1, [r2, r3]
      }

      /* Configure IO Direction mode (Input, Output, Alternate or Analog) */
      temp = GPIOx->MODER;
 8000ae6:	687b      	ldr	r3, [r7, #4]
 8000ae8:	681b      	ldr	r3, [r3, #0]
 8000aea:	613b      	str	r3, [r7, #16]
      temp &= ~(GPIO_MODER_MODE0 << (position * 2U));
 8000aec:	697b      	ldr	r3, [r7, #20]
 8000aee:	005b      	lsls	r3, r3, #1
 8000af0:	2203      	movs	r2, #3
 8000af2:	409a      	lsls	r2, r3
 8000af4:	0013      	movs	r3, r2
 8000af6:	43da      	mvns	r2, r3
 8000af8:	693b      	ldr	r3, [r7, #16]
 8000afa:	4013      	ands	r3, r2
 8000afc:	613b      	str	r3, [r7, #16]
      temp |= ((GPIO_Init->Mode & GPIO_MODE) << (position * 2U));
 8000afe:	683b      	ldr	r3, [r7, #0]
 8000b00:	685b      	ldr	r3, [r3, #4]
 8000b02:	2203      	movs	r2, #3
 8000b04:	401a      	ands	r2, r3
 8000b06:	697b      	ldr	r3, [r7, #20]
 8000b08:	005b      	lsls	r3, r3, #1
 8000b0a:	409a      	lsls	r2, r3
 8000b0c:	0013      	movs	r3, r2
 8000b0e:	693a      	ldr	r2, [r7, #16]
 8000b10:	4313      	orrs	r3, r2
 8000b12:	613b      	str	r3, [r7, #16]
      GPIOx->MODER = temp;
 8000b14:	687b      	ldr	r3, [r7, #4]
 8000b16:	693a      	ldr	r2, [r7, #16]
 8000b18:	601a      	str	r2, [r3, #0]

      /*--------------------- EXTI Mode Configuration ------------------------*/
      /* Configure the External Interrupt or event for the current IO */
      if ((GPIO_Init->Mode & EXTI_MODE) != 0x00U)
 8000b1a:	683b      	ldr	r3, [r7, #0]
 8000b1c:	685a      	ldr	r2, [r3, #4]
 8000b1e:	23c0      	movs	r3, #192	; 0xc0
 8000b20:	029b      	lsls	r3, r3, #10
 8000b22:	4013      	ands	r3, r2
 8000b24:	d100      	bne.n	8000b28 <HAL_GPIO_Init+0x17c>
 8000b26:	e0a0      	b.n	8000c6a <HAL_GPIO_Init+0x2be>
      {
        /* Enable SYSCFG Clock */
        __HAL_RCC_SYSCFG_CLK_ENABLE();
 8000b28:	4b57      	ldr	r3, [pc, #348]	; (8000c88 <HAL_GPIO_Init+0x2dc>)
 8000b2a:	6b5a      	ldr	r2, [r3, #52]	; 0x34
 8000b2c:	4b56      	ldr	r3, [pc, #344]	; (8000c88 <HAL_GPIO_Init+0x2dc>)
 8000b2e:	2101      	movs	r1, #1
 8000b30:	430a      	orrs	r2, r1
 8000b32:	635a      	str	r2, [r3, #52]	; 0x34

        temp = SYSCFG->EXTICR[position >> 2U];
 8000b34:	4a55      	ldr	r2, [pc, #340]	; (8000c8c <HAL_GPIO_Init+0x2e0>)
 8000b36:	697b      	ldr	r3, [r7, #20]
 8000b38:	089b      	lsrs	r3, r3, #2
 8000b3a:	3302      	adds	r3, #2
 8000b3c:	009b      	lsls	r3, r3, #2
 8000b3e:	589b      	ldr	r3, [r3, r2]
 8000b40:	613b      	str	r3, [r7, #16]
        CLEAR_BIT(temp, (0x0FUL) << (4U * (position & 0x03U)));
 8000b42:	697b      	ldr	r3, [r7, #20]
 8000b44:	2203      	movs	r2, #3
 8000b46:	4013      	ands	r3, r2
 8000b48:	009b      	lsls	r3, r3, #2
 8000b4a:	220f      	movs	r2, #15
 8000b4c:	409a      	lsls	r2, r3
 8000b4e:	0013      	movs	r3, r2
 8000b50:	43da      	mvns	r2, r3
 8000b52:	693b      	ldr	r3, [r7, #16]
 8000b54:	4013      	ands	r3, r2
 8000b56:	613b      	str	r3, [r7, #16]
        SET_BIT(temp, (GPIO_GET_INDEX(GPIOx)) << (4 * (position & 0x03U)));
 8000b58:	687a      	ldr	r2, [r7, #4]
 8000b5a:	23a0      	movs	r3, #160	; 0xa0
 8000b5c:	05db      	lsls	r3, r3, #23
 8000b5e:	429a      	cmp	r2, r3
 8000b60:	d01f      	beq.n	8000ba2 <HAL_GPIO_Init+0x1f6>
 8000b62:	687b      	ldr	r3, [r7, #4]
 8000b64:	4a4a      	ldr	r2, [pc, #296]	; (8000c90 <HAL_GPIO_Init+0x2e4>)
 8000b66:	4293      	cmp	r3, r2
 8000b68:	d019      	beq.n	8000b9e <HAL_GPIO_Init+0x1f2>
 8000b6a:	687b      	ldr	r3, [r7, #4]
 8000b6c:	4a49      	ldr	r2, [pc, #292]	; (8000c94 <HAL_GPIO_Init+0x2e8>)
 8000b6e:	4293      	cmp	r3, r2
 8000b70:	d013      	beq.n	8000b9a <HAL_GPIO_Init+0x1ee>
 8000b72:	687b      	ldr	r3, [r7, #4]
 8000b74:	4a48      	ldr	r2, [pc, #288]	; (8000c98 <HAL_GPIO_Init+0x2ec>)
 8000b76:	4293      	cmp	r3, r2
 8000b78:	d00d      	beq.n	8000b96 <HAL_GPIO_Init+0x1ea>
 8000b7a:	687b      	ldr	r3, [r7, #4]
 8000b7c:	4a47      	ldr	r2, [pc, #284]	; (8000c9c <HAL_GPIO_Init+0x2f0>)
 8000b7e:	4293      	cmp	r3, r2
 8000b80:	d007      	beq.n	8000b92 <HAL_GPIO_Init+0x1e6>
 8000b82:	687b      	ldr	r3, [r7, #4]
 8000b84:	4a46      	ldr	r2, [pc, #280]	; (8000ca0 <HAL_GPIO_Init+0x2f4>)
 8000b86:	4293      	cmp	r3, r2
 8000b88:	d101      	bne.n	8000b8e <HAL_GPIO_Init+0x1e2>
 8000b8a:	2305      	movs	r3, #5
 8000b8c:	e00a      	b.n	8000ba4 <HAL_GPIO_Init+0x1f8>
 8000b8e:	2306      	movs	r3, #6
 8000b90:	e008      	b.n	8000ba4 <HAL_GPIO_Init+0x1f8>
 8000b92:	2304      	movs	r3, #4
 8000b94:	e006      	b.n	8000ba4 <HAL_GPIO_Init+0x1f8>
 8000b96:	2303      	movs	r3, #3
 8000b98:	e004      	b.n	8000ba4 <HAL_GPIO_Init+0x1f8>
 8000b9a:	2302      	movs	r3, #2
 8000b9c:	e002      	b.n	8000ba4 <HAL_GPIO_Init+0x1f8>
 8000b9e:	2301      	movs	r3, #1
 8000ba0:	e000      	b.n	8000ba4 <HAL_GPIO_Init+0x1f8>
 8000ba2:	2300      	movs	r3, #0
 8000ba4:	697a      	ldr	r2, [r7, #20]
 8000ba6:	2103      	movs	r1, #3
 8000ba8:	400a      	ands	r2, r1
 8000baa:	0092      	lsls	r2, r2, #2
 8000bac:	4093      	lsls	r3, r2
 8000bae:	693a      	ldr	r2, [r7, #16]
 8000bb0:	4313      	orrs	r3, r2
 8000bb2:	613b      	str	r3, [r7, #16]
        SYSCFG->EXTICR[position >> 2U] = temp;
 8000bb4:	4935      	ldr	r1, [pc, #212]	; (8000c8c <HAL_GPIO_Init+0x2e0>)
 8000bb6:	697b      	ldr	r3, [r7, #20]
 8000bb8:	089b      	lsrs	r3, r3, #2
 8000bba:	3302      	adds	r3, #2
 8000bbc:	009b      	lsls	r3, r3, #2
 8000bbe:	693a      	ldr	r2, [r7, #16]
 8000bc0:	505a      	str	r2, [r3, r1]

        /* Clear Rising Falling edge configuration */
        temp = EXTI->RTSR;
 8000bc2:	4b38      	ldr	r3, [pc, #224]	; (8000ca4 <HAL_GPIO_Init+0x2f8>)
 8000bc4:	689b      	ldr	r3, [r3, #8]
 8000bc6:	613b      	str	r3, [r7, #16]
        temp &= ~((uint32_t)iocurrent);
 8000bc8:	68fb      	ldr	r3, [r7, #12]
 8000bca:	43da      	mvns	r2, r3
 8000bcc:	693b      	ldr	r3, [r7, #16]
 8000bce:	4013      	ands	r3, r2
 8000bd0:	613b      	str	r3, [r7, #16]
        if ((GPIO_Init->Mode & TRIGGER_RISING) != 0x00U)
 8000bd2:	683b      	ldr	r3, [r7, #0]
 8000bd4:	685a      	ldr	r2, [r3, #4]
 8000bd6:	2380      	movs	r3, #128	; 0x80
 8000bd8:	035b      	lsls	r3, r3, #13
 8000bda:	4013      	ands	r3, r2
 8000bdc:	d003      	beq.n	8000be6 <HAL_GPIO_Init+0x23a>
        {
          temp |= iocurrent;
 8000bde:	693a      	ldr	r2, [r7, #16]
 8000be0:	68fb      	ldr	r3, [r7, #12]
 8000be2:	4313      	orrs	r3, r2
 8000be4:	613b      	str	r3, [r7, #16]
        }
        EXTI->RTSR = temp;
 8000be6:	4b2f      	ldr	r3, [pc, #188]	; (8000ca4 <HAL_GPIO_Init+0x2f8>)
 8000be8:	693a      	ldr	r2, [r7, #16]
 8000bea:	609a      	str	r2, [r3, #8]

        temp = EXTI->FTSR;
 8000bec:	4b2d      	ldr	r3, [pc, #180]	; (8000ca4 <HAL_GPIO_Init+0x2f8>)
 8000bee:	68db      	ldr	r3, [r3, #12]
 8000bf0:	613b      	str	r3, [r7, #16]
        temp &= ~((uint32_t)iocurrent);
 8000bf2:	68fb      	ldr	r3, [r7, #12]
 8000bf4:	43da      	mvns	r2, r3
 8000bf6:	693b      	ldr	r3, [r7, #16]
 8000bf8:	4013      	ands	r3, r2
 8000bfa:	613b      	str	r3, [r7, #16]
        if ((GPIO_Init->Mode & TRIGGER_FALLING) != 0x00U)
 8000bfc:	683b      	ldr	r3, [r7, #0]
 8000bfe:	685a      	ldr	r2, [r3, #4]
 8000c00:	2380      	movs	r3, #128	; 0x80
 8000c02:	039b      	lsls	r3, r3, #14
 8000c04:	4013      	ands	r3, r2
 8000c06:	d003      	beq.n	8000c10 <HAL_GPIO_Init+0x264>
        {
          temp |= iocurrent;
 8000c08:	693a      	ldr	r2, [r7, #16]
 8000c0a:	68fb      	ldr	r3, [r7, #12]
 8000c0c:	4313      	orrs	r3, r2
 8000c0e:	613b      	str	r3, [r7, #16]
        }
        EXTI->FTSR = temp;
 8000c10:	4b24      	ldr	r3, [pc, #144]	; (8000ca4 <HAL_GPIO_Init+0x2f8>)
 8000c12:	693a      	ldr	r2, [r7, #16]
 8000c14:	60da      	str	r2, [r3, #12]

        temp = EXTI->EMR;
 8000c16:	4b23      	ldr	r3, [pc, #140]	; (8000ca4 <HAL_GPIO_Init+0x2f8>)
 8000c18:	685b      	ldr	r3, [r3, #4]
 8000c1a:	613b      	str	r3, [r7, #16]
        temp &= ~((uint32_t)iocurrent);
 8000c1c:	68fb      	ldr	r3, [r7, #12]
 8000c1e:	43da      	mvns	r2, r3
 8000c20:	693b      	ldr	r3, [r7, #16]
 8000c22:	4013      	ands	r3, r2
 8000c24:	613b      	str	r3, [r7, #16]
        if ((GPIO_Init->Mode & EXTI_EVT) != 0x00U)
 8000c26:	683b      	ldr	r3, [r7, #0]
 8000c28:	685a      	ldr	r2, [r3, #4]
 8000c2a:	2380      	movs	r3, #128	; 0x80
 8000c2c:	029b      	lsls	r3, r3, #10
 8000c2e:	4013      	ands	r3, r2
 8000c30:	d003      	beq.n	8000c3a <HAL_GPIO_Init+0x28e>
        {
          temp |= iocurrent;
 8000c32:	693a      	ldr	r2, [r7, #16]
 8000c34:	68fb      	ldr	r3, [r7, #12]
 8000c36:	4313      	orrs	r3, r2
 8000c38:	613b      	str	r3, [r7, #16]
        }
        EXTI->EMR = temp;
 8000c3a:	4b1a      	ldr	r3, [pc, #104]	; (8000ca4 <HAL_GPIO_Init+0x2f8>)
 8000c3c:	693a      	ldr	r2, [r7, #16]
 8000c3e:	605a      	str	r2, [r3, #4]

        /* Clear EXTI line configuration */
        temp = EXTI->IMR;
 8000c40:	4b18      	ldr	r3, [pc, #96]	; (8000ca4 <HAL_GPIO_Init+0x2f8>)
 8000c42:	681b      	ldr	r3, [r3, #0]
 8000c44:	613b      	str	r3, [r7, #16]
        temp &= ~((uint32_t)iocurrent);
 8000c46:	68fb      	ldr	r3, [r7, #12]
 8000c48:	43da      	mvns	r2, r3
 8000c4a:	693b      	ldr	r3, [r7, #16]
 8000c4c:	4013      	ands	r3, r2
 8000c4e:	613b      	str	r3, [r7, #16]
        if ((GPIO_Init->Mode & EXTI_IT) != 0x00U)
 8000c50:	683b      	ldr	r3, [r7, #0]
 8000c52:	685a      	ldr	r2, [r3, #4]
 8000c54:	2380      	movs	r3, #128	; 0x80
 8000c56:	025b      	lsls	r3, r3, #9
 8000c58:	4013      	ands	r3, r2
 8000c5a:	d003      	beq.n	8000c64 <HAL_GPIO_Init+0x2b8>
        {
          temp |= iocurrent;
 8000c5c:	693a      	ldr	r2, [r7, #16]
 8000c5e:	68fb      	ldr	r3, [r7, #12]
 8000c60:	4313      	orrs	r3, r2
 8000c62:	613b      	str	r3, [r7, #16]
        }
        EXTI->IMR = temp;
 8000c64:	4b0f      	ldr	r3, [pc, #60]	; (8000ca4 <HAL_GPIO_Init+0x2f8>)
 8000c66:	693a      	ldr	r2, [r7, #16]
 8000c68:	601a      	str	r2, [r3, #0]
      }
    }
    position++;
 8000c6a:	697b      	ldr	r3, [r7, #20]
 8000c6c:	3301      	adds	r3, #1
 8000c6e:	617b      	str	r3, [r7, #20]
  while (((GPIO_Init->Pin) >> position) != 0)
 8000c70:	683b      	ldr	r3, [r7, #0]
 8000c72:	681a      	ldr	r2, [r3, #0]
 8000c74:	697b      	ldr	r3, [r7, #20]
 8000c76:	40da      	lsrs	r2, r3
 8000c78:	1e13      	subs	r3, r2, #0
 8000c7a:	d000      	beq.n	8000c7e <HAL_GPIO_Init+0x2d2>
 8000c7c:	e6a2      	b.n	80009c4 <HAL_GPIO_Init+0x18>
  }
}
 8000c7e:	46c0      	nop			; (mov r8, r8)
 8000c80:	46c0      	nop			; (mov r8, r8)
 8000c82:	46bd      	mov	sp, r7
 8000c84:	b006      	add	sp, #24
 8000c86:	bd80      	pop	{r7, pc}
 8000c88:	40021000 	.word	0x40021000
 8000c8c:	40010000 	.word	0x40010000
 8000c90:	50000400 	.word	0x50000400
 8000c94:	50000800 	.word	0x50000800
 8000c98:	50000c00 	.word	0x50000c00
 8000c9c:	50001000 	.word	0x50001000
 8000ca0:	50001c00 	.word	0x50001c00
 8000ca4:	40010400 	.word	0x40010400

08000ca8 <HAL_GPIO_WritePin>:
  *                        GPIO_PIN_RESET: to clear the port pin
  *                        GPIO_PIN_SET: to set the port pin
  * @retval None
  */
void HAL_GPIO_WritePin(GPIO_TypeDef *GPIOx, uint16_t GPIO_Pin, GPIO_PinState PinState)
{
 8000ca8:	b580      	push	{r7, lr}
 8000caa:	b082      	sub	sp, #8
 8000cac:	af00      	add	r7, sp, #0
 8000cae:	6078      	str	r0, [r7, #4]
 8000cb0:	0008      	movs	r0, r1
 8000cb2:	0011      	movs	r1, r2
 8000cb4:	1cbb      	adds	r3, r7, #2
 8000cb6:	1c02      	adds	r2, r0, #0
 8000cb8:	801a      	strh	r2, [r3, #0]
 8000cba:	1c7b      	adds	r3, r7, #1
 8000cbc:	1c0a      	adds	r2, r1, #0
 8000cbe:	701a      	strb	r2, [r3, #0]
  /* Check the parameters */
  assert_param(IS_GPIO_PIN_AVAILABLE(GPIOx, GPIO_Pin));
  assert_param(IS_GPIO_PIN_ACTION(PinState));

  if (PinState != GPIO_PIN_RESET)
 8000cc0:	1c7b      	adds	r3, r7, #1
 8000cc2:	781b      	ldrb	r3, [r3, #0]
 8000cc4:	2b00      	cmp	r3, #0
 8000cc6:	d004      	beq.n	8000cd2 <HAL_GPIO_WritePin+0x2a>
  {
    GPIOx->BSRR = GPIO_Pin;
 8000cc8:	1cbb      	adds	r3, r7, #2
 8000cca:	881a      	ldrh	r2, [r3, #0]
 8000ccc:	687b      	ldr	r3, [r7, #4]
 8000cce:	619a      	str	r2, [r3, #24]
  }
  else
  {
    GPIOx->BRR = GPIO_Pin ;
  }
}
 8000cd0:	e003      	b.n	8000cda <HAL_GPIO_WritePin+0x32>
    GPIOx->BRR = GPIO_Pin ;
 8000cd2:	1cbb      	adds	r3, r7, #2
 8000cd4:	881a      	ldrh	r2, [r3, #0]
 8000cd6:	687b      	ldr	r3, [r7, #4]
 8000cd8:	629a      	str	r2, [r3, #40]	; 0x28
}
 8000cda:	46c0      	nop			; (mov r8, r8)
 8000cdc:	46bd      	mov	sp, r7
 8000cde:	b002      	add	sp, #8
 8000ce0:	bd80      	pop	{r7, pc}
	...

08000ce4 <HAL_RCC_OscConfig>:
  *         supported by this macro. User should request a transition to HSE Off
  *         first and then HSE On or HSE Bypass.
  * @retval HAL status
  */
HAL_StatusTypeDef HAL_RCC_OscConfig(RCC_OscInitTypeDef  *RCC_OscInitStruct)
{
 8000ce4:	b5b0      	push	{r4, r5, r7, lr}
 8000ce6:	b08a      	sub	sp, #40	; 0x28
 8000ce8:	af00      	add	r7, sp, #0
 8000cea:	6078      	str	r0, [r7, #4]
  uint32_t hsi_state;
  HAL_StatusTypeDef status;
  uint32_t sysclk_source, pll_config;

  /* Check Null pointer */
  if(RCC_OscInitStruct == NULL)
 8000cec:	687b      	ldr	r3, [r7, #4]
 8000cee:	2b00      	cmp	r3, #0
 8000cf0:	d102      	bne.n	8000cf8 <HAL_RCC_OscConfig+0x14>
  {
    return HAL_ERROR;
 8000cf2:	2301      	movs	r3, #1
 8000cf4:	f000 fbbf 	bl	8001476 <HAL_RCC_OscConfig+0x792>
  }

  /* Check the parameters */
  assert_param(IS_RCC_OSCILLATORTYPE(RCC_OscInitStruct->OscillatorType));

  sysclk_source = __HAL_RCC_GET_SYSCLK_SOURCE();
 8000cf8:	4bc9      	ldr	r3, [pc, #804]	; (8001020 <HAL_RCC_OscConfig+0x33c>)
 8000cfa:	68db      	ldr	r3, [r3, #12]
 8000cfc:	220c      	movs	r2, #12
 8000cfe:	4013      	ands	r3, r2
 8000d00:	61fb      	str	r3, [r7, #28]
  pll_config = __HAL_RCC_GET_PLL_OSCSOURCE();
 8000d02:	4bc7      	ldr	r3, [pc, #796]	; (8001020 <HAL_RCC_OscConfig+0x33c>)
 8000d04:	68da      	ldr	r2, [r3, #12]
 8000d06:	2380      	movs	r3, #128	; 0x80
 8000d08:	025b      	lsls	r3, r3, #9
 8000d0a:	4013      	ands	r3, r2
 8000d0c:	61bb      	str	r3, [r7, #24]

  /*------------------------------- HSE Configuration ------------------------*/
  if(((RCC_OscInitStruct->OscillatorType) & RCC_OSCILLATORTYPE_HSE) == RCC_OSCILLATORTYPE_HSE)
 8000d0e:	687b      	ldr	r3, [r7, #4]
 8000d10:	681b      	ldr	r3, [r3, #0]
 8000d12:	2201      	movs	r2, #1
 8000d14:	4013      	ands	r3, r2
 8000d16:	d100      	bne.n	8000d1a <HAL_RCC_OscConfig+0x36>
 8000d18:	e07e      	b.n	8000e18 <HAL_RCC_OscConfig+0x134>
  {
    /* Check the parameters */
    assert_param(IS_RCC_HSE(RCC_OscInitStruct->HSEState));

    /* When the HSE is used as system clock or clock source for PLL in these cases it is not allowed to be disabled */
    if((sysclk_source == RCC_SYSCLKSOURCE_STATUS_HSE)
 8000d1a:	69fb      	ldr	r3, [r7, #28]
 8000d1c:	2b08      	cmp	r3, #8
 8000d1e:	d007      	beq.n	8000d30 <HAL_RCC_OscConfig+0x4c>
       || ((sysclk_source == RCC_SYSCLKSOURCE_STATUS_PLLCLK) && (pll_config == RCC_PLLSOURCE_HSE)))
 8000d20:	69fb      	ldr	r3, [r7, #28]
 8000d22:	2b0c      	cmp	r3, #12
 8000d24:	d112      	bne.n	8000d4c <HAL_RCC_OscConfig+0x68>
 8000d26:	69ba      	ldr	r2, [r7, #24]
 8000d28:	2380      	movs	r3, #128	; 0x80
 8000d2a:	025b      	lsls	r3, r3, #9
 8000d2c:	429a      	cmp	r2, r3
 8000d2e:	d10d      	bne.n	8000d4c <HAL_RCC_OscConfig+0x68>
    {
      if((__HAL_RCC_GET_FLAG(RCC_FLAG_HSERDY) != 0U) && (RCC_OscInitStruct->HSEState == RCC_HSE_OFF))
 8000d30:	4bbb      	ldr	r3, [pc, #748]	; (8001020 <HAL_RCC_OscConfig+0x33c>)
 8000d32:	681a      	ldr	r2, [r3, #0]
 8000d34:	2380      	movs	r3, #128	; 0x80
 8000d36:	029b      	lsls	r3, r3, #10
 8000d38:	4013      	ands	r3, r2
 8000d3a:	d100      	bne.n	8000d3e <HAL_RCC_OscConfig+0x5a>
 8000d3c:	e06b      	b.n	8000e16 <HAL_RCC_OscConfig+0x132>
 8000d3e:	687b      	ldr	r3, [r7, #4]
 8000d40:	685b      	ldr	r3, [r3, #4]
 8000d42:	2b00      	cmp	r3, #0
 8000d44:	d167      	bne.n	8000e16 <HAL_RCC_OscConfig+0x132>
      {
        return HAL_ERROR;
 8000d46:	2301      	movs	r3, #1
 8000d48:	f000 fb95 	bl	8001476 <HAL_RCC_OscConfig+0x792>
      }
    }
    else
    {
      /* Set the new HSE configuration ---------------------------------------*/
      __HAL_RCC_HSE_CONFIG(RCC_OscInitStruct->HSEState);
 8000d4c:	687b      	ldr	r3, [r7, #4]
 8000d4e:	685a      	ldr	r2, [r3, #4]
 8000d50:	2380      	movs	r3, #128	; 0x80
 8000d52:	025b      	lsls	r3, r3, #9
 8000d54:	429a      	cmp	r2, r3
 8000d56:	d107      	bne.n	8000d68 <HAL_RCC_OscConfig+0x84>
 8000d58:	4bb1      	ldr	r3, [pc, #708]	; (8001020 <HAL_RCC_OscConfig+0x33c>)
 8000d5a:	681a      	ldr	r2, [r3, #0]
 8000d5c:	4bb0      	ldr	r3, [pc, #704]	; (8001020 <HAL_RCC_OscConfig+0x33c>)
 8000d5e:	2180      	movs	r1, #128	; 0x80
 8000d60:	0249      	lsls	r1, r1, #9
 8000d62:	430a      	orrs	r2, r1
 8000d64:	601a      	str	r2, [r3, #0]
 8000d66:	e027      	b.n	8000db8 <HAL_RCC_OscConfig+0xd4>
 8000d68:	687b      	ldr	r3, [r7, #4]
 8000d6a:	685a      	ldr	r2, [r3, #4]
 8000d6c:	23a0      	movs	r3, #160	; 0xa0
 8000d6e:	02db      	lsls	r3, r3, #11
 8000d70:	429a      	cmp	r2, r3
 8000d72:	d10e      	bne.n	8000d92 <HAL_RCC_OscConfig+0xae>
 8000d74:	4baa      	ldr	r3, [pc, #680]	; (8001020 <HAL_RCC_OscConfig+0x33c>)
 8000d76:	681a      	ldr	r2, [r3, #0]
 8000d78:	4ba9      	ldr	r3, [pc, #676]	; (8001020 <HAL_RCC_OscConfig+0x33c>)
 8000d7a:	2180      	movs	r1, #128	; 0x80
 8000d7c:	02c9      	lsls	r1, r1, #11
 8000d7e:	430a      	orrs	r2, r1
 8000d80:	601a      	str	r2, [r3, #0]
 8000d82:	4ba7      	ldr	r3, [pc, #668]	; (8001020 <HAL_RCC_OscConfig+0x33c>)
 8000d84:	681a      	ldr	r2, [r3, #0]
 8000d86:	4ba6      	ldr	r3, [pc, #664]	; (8001020 <HAL_RCC_OscConfig+0x33c>)
 8000d88:	2180      	movs	r1, #128	; 0x80
 8000d8a:	0249      	lsls	r1, r1, #9
 8000d8c:	430a      	orrs	r2, r1
 8000d8e:	601a      	str	r2, [r3, #0]
 8000d90:	e012      	b.n	8000db8 <HAL_RCC_OscConfig+0xd4>
 8000d92:	4ba3      	ldr	r3, [pc, #652]	; (8001020 <HAL_RCC_OscConfig+0x33c>)
 8000d94:	681a      	ldr	r2, [r3, #0]
 8000d96:	4ba2      	ldr	r3, [pc, #648]	; (8001020 <HAL_RCC_OscConfig+0x33c>)
 8000d98:	49a2      	ldr	r1, [pc, #648]	; (8001024 <HAL_RCC_OscConfig+0x340>)
 8000d9a:	400a      	ands	r2, r1
 8000d9c:	601a      	str	r2, [r3, #0]
 8000d9e:	4ba0      	ldr	r3, [pc, #640]	; (8001020 <HAL_RCC_OscConfig+0x33c>)
 8000da0:	681a      	ldr	r2, [r3, #0]
 8000da2:	2380      	movs	r3, #128	; 0x80
 8000da4:	025b      	lsls	r3, r3, #9
 8000da6:	4013      	ands	r3, r2
 8000da8:	60fb      	str	r3, [r7, #12]
 8000daa:	68fb      	ldr	r3, [r7, #12]
 8000dac:	4b9c      	ldr	r3, [pc, #624]	; (8001020 <HAL_RCC_OscConfig+0x33c>)
 8000dae:	681a      	ldr	r2, [r3, #0]
 8000db0:	4b9b      	ldr	r3, [pc, #620]	; (8001020 <HAL_RCC_OscConfig+0x33c>)
 8000db2:	499d      	ldr	r1, [pc, #628]	; (8001028 <HAL_RCC_OscConfig+0x344>)
 8000db4:	400a      	ands	r2, r1
 8000db6:	601a      	str	r2, [r3, #0]

      /* Check the HSE State */
      if(RCC_OscInitStruct->HSEState != RCC_HSE_OFF)
 8000db8:	687b      	ldr	r3, [r7, #4]
 8000dba:	685b      	ldr	r3, [r3, #4]
 8000dbc:	2b00      	cmp	r3, #0
 8000dbe:	d015      	beq.n	8000dec <HAL_RCC_OscConfig+0x108>
      {
        /* Get Start Tick */
        tickstart = HAL_GetTick();
 8000dc0:	f7ff fd12 	bl	80007e8 <HAL_GetTick>
 8000dc4:	0003      	movs	r3, r0
 8000dc6:	617b      	str	r3, [r7, #20]

        /* Wait till HSE is ready */
        while(__HAL_RCC_GET_FLAG(RCC_FLAG_HSERDY) == 0U)
 8000dc8:	e009      	b.n	8000dde <HAL_RCC_OscConfig+0xfa>
        {
          if((HAL_GetTick() - tickstart ) > HSE_TIMEOUT_VALUE)
 8000dca:	f7ff fd0d 	bl	80007e8 <HAL_GetTick>
 8000dce:	0002      	movs	r2, r0
 8000dd0:	697b      	ldr	r3, [r7, #20]
 8000dd2:	1ad3      	subs	r3, r2, r3
 8000dd4:	2b64      	cmp	r3, #100	; 0x64
 8000dd6:	d902      	bls.n	8000dde <HAL_RCC_OscConfig+0xfa>
          {
            return HAL_TIMEOUT;
 8000dd8:	2303      	movs	r3, #3
 8000dda:	f000 fb4c 	bl	8001476 <HAL_RCC_OscConfig+0x792>
        while(__HAL_RCC_GET_FLAG(RCC_FLAG_HSERDY) == 0U)
 8000dde:	4b90      	ldr	r3, [pc, #576]	; (8001020 <HAL_RCC_OscConfig+0x33c>)
 8000de0:	681a      	ldr	r2, [r3, #0]
 8000de2:	2380      	movs	r3, #128	; 0x80
 8000de4:	029b      	lsls	r3, r3, #10
 8000de6:	4013      	ands	r3, r2
 8000de8:	d0ef      	beq.n	8000dca <HAL_RCC_OscConfig+0xe6>
 8000dea:	e015      	b.n	8000e18 <HAL_RCC_OscConfig+0x134>
        }
      }
      else
      {
        /* Get Start Tick */
        tickstart = HAL_GetTick();
 8000dec:	f7ff fcfc 	bl	80007e8 <HAL_GetTick>
 8000df0:	0003      	movs	r3, r0
 8000df2:	617b      	str	r3, [r7, #20]

        /* Wait till HSE is disabled */
        while(__HAL_RCC_GET_FLAG(RCC_FLAG_HSERDY) != 0U)
 8000df4:	e008      	b.n	8000e08 <HAL_RCC_OscConfig+0x124>
        {
           if((HAL_GetTick() - tickstart ) > HSE_TIMEOUT_VALUE)
 8000df6:	f7ff fcf7 	bl	80007e8 <HAL_GetTick>
 8000dfa:	0002      	movs	r2, r0
 8000dfc:	697b      	ldr	r3, [r7, #20]
 8000dfe:	1ad3      	subs	r3, r2, r3
 8000e00:	2b64      	cmp	r3, #100	; 0x64
 8000e02:	d901      	bls.n	8000e08 <HAL_RCC_OscConfig+0x124>
          {
            return HAL_TIMEOUT;
 8000e04:	2303      	movs	r3, #3
 8000e06:	e336      	b.n	8001476 <HAL_RCC_OscConfig+0x792>
        while(__HAL_RCC_GET_FLAG(RCC_FLAG_HSERDY) != 0U)
 8000e08:	4b85      	ldr	r3, [pc, #532]	; (8001020 <HAL_RCC_OscConfig+0x33c>)
 8000e0a:	681a      	ldr	r2, [r3, #0]
 8000e0c:	2380      	movs	r3, #128	; 0x80
 8000e0e:	029b      	lsls	r3, r3, #10
 8000e10:	4013      	ands	r3, r2
 8000e12:	d1f0      	bne.n	8000df6 <HAL_RCC_OscConfig+0x112>
 8000e14:	e000      	b.n	8000e18 <HAL_RCC_OscConfig+0x134>
      if((__HAL_RCC_GET_FLAG(RCC_FLAG_HSERDY) != 0U) && (RCC_OscInitStruct->HSEState == RCC_HSE_OFF))
 8000e16:	46c0      	nop			; (mov r8, r8)
        }
      }
    }
  }
  /*----------------------------- HSI Configuration --------------------------*/
  if(((RCC_OscInitStruct->OscillatorType) & RCC_OSCILLATORTYPE_HSI) == RCC_OSCILLATORTYPE_HSI)
 8000e18:	687b      	ldr	r3, [r7, #4]
 8000e1a:	681b      	ldr	r3, [r3, #0]
 8000e1c:	2202      	movs	r2, #2
 8000e1e:	4013      	ands	r3, r2
 8000e20:	d100      	bne.n	8000e24 <HAL_RCC_OscConfig+0x140>
 8000e22:	e099      	b.n	8000f58 <HAL_RCC_OscConfig+0x274>
  {
    /* Check the parameters */
    assert_param(IS_RCC_HSI(RCC_OscInitStruct->HSIState));
    assert_param(IS_RCC_CALIBRATION_VALUE(RCC_OscInitStruct->HSICalibrationValue));

    hsi_state = RCC_OscInitStruct->HSIState;
 8000e24:	687b      	ldr	r3, [r7, #4]
 8000e26:	68db      	ldr	r3, [r3, #12]
 8000e28:	627b      	str	r3, [r7, #36]	; 0x24

#if defined(RCC_CR_HSIOUTEN)
    if((hsi_state & RCC_HSI_OUTEN) != 0U)
 8000e2a:	6a7b      	ldr	r3, [r7, #36]	; 0x24
 8000e2c:	2220      	movs	r2, #32
 8000e2e:	4013      	ands	r3, r2
 8000e30:	d009      	beq.n	8000e46 <HAL_RCC_OscConfig+0x162>
    {
      /* HSI Output enable for timer requested */
      SET_BIT(RCC->CR, RCC_CR_HSIOUTEN);
 8000e32:	4b7b      	ldr	r3, [pc, #492]	; (8001020 <HAL_RCC_OscConfig+0x33c>)
 8000e34:	681a      	ldr	r2, [r3, #0]
 8000e36:	4b7a      	ldr	r3, [pc, #488]	; (8001020 <HAL_RCC_OscConfig+0x33c>)
 8000e38:	2120      	movs	r1, #32
 8000e3a:	430a      	orrs	r2, r1
 8000e3c:	601a      	str	r2, [r3, #0]

      hsi_state &= ~RCC_CR_HSIOUTEN;
 8000e3e:	6a7b      	ldr	r3, [r7, #36]	; 0x24
 8000e40:	2220      	movs	r2, #32
 8000e42:	4393      	bics	r3, r2
 8000e44:	627b      	str	r3, [r7, #36]	; 0x24
    }
#endif

    /* Check if HSI is used as system clock or as PLL source when PLL is selected as system clock */
    if((sysclk_source == RCC_SYSCLKSOURCE_STATUS_HSI)
 8000e46:	69fb      	ldr	r3, [r7, #28]
 8000e48:	2b04      	cmp	r3, #4
 8000e4a:	d005      	beq.n	8000e58 <HAL_RCC_OscConfig+0x174>
       || ((sysclk_source == RCC_SYSCLKSOURCE_STATUS_PLLCLK) && (pll_config == RCC_PLLSOURCE_HSI)))
 8000e4c:	69fb      	ldr	r3, [r7, #28]
 8000e4e:	2b0c      	cmp	r3, #12
 8000e50:	d13e      	bne.n	8000ed0 <HAL_RCC_OscConfig+0x1ec>
 8000e52:	69bb      	ldr	r3, [r7, #24]
 8000e54:	2b00      	cmp	r3, #0
 8000e56:	d13b      	bne.n	8000ed0 <HAL_RCC_OscConfig+0x1ec>
    {
      /* When HSI is used as system clock it will not disabled */
      if((__HAL_RCC_GET_FLAG(RCC_FLAG_HSIRDY) != 0U) && (hsi_state == RCC_HSI_OFF))
 8000e58:	4b71      	ldr	r3, [pc, #452]	; (8001020 <HAL_RCC_OscConfig+0x33c>)
 8000e5a:	681b      	ldr	r3, [r3, #0]
 8000e5c:	2204      	movs	r2, #4
 8000e5e:	4013      	ands	r3, r2
 8000e60:	d004      	beq.n	8000e6c <HAL_RCC_OscConfig+0x188>
 8000e62:	6a7b      	ldr	r3, [r7, #36]	; 0x24
 8000e64:	2b00      	cmp	r3, #0
 8000e66:	d101      	bne.n	8000e6c <HAL_RCC_OscConfig+0x188>
      {
        return HAL_ERROR;
 8000e68:	2301      	movs	r3, #1
 8000e6a:	e304      	b.n	8001476 <HAL_RCC_OscConfig+0x792>
      }
      /* Otherwise, just the calibration and HSI or HSIdiv4 are allowed */
      else
      {
        /* Adjusts the Internal High Speed oscillator (HSI) calibration value.*/
        __HAL_RCC_HSI_CALIBRATIONVALUE_ADJUST(RCC_OscInitStruct->HSICalibrationValue);
 8000e6c:	4b6c      	ldr	r3, [pc, #432]	; (8001020 <HAL_RCC_OscConfig+0x33c>)
 8000e6e:	685b      	ldr	r3, [r3, #4]
 8000e70:	4a6e      	ldr	r2, [pc, #440]	; (800102c <HAL_RCC_OscConfig+0x348>)
 8000e72:	4013      	ands	r3, r2
 8000e74:	0019      	movs	r1, r3
 8000e76:	687b      	ldr	r3, [r7, #4]
 8000e78:	691b      	ldr	r3, [r3, #16]
 8000e7a:	021a      	lsls	r2, r3, #8
 8000e7c:	4b68      	ldr	r3, [pc, #416]	; (8001020 <HAL_RCC_OscConfig+0x33c>)
 8000e7e:	430a      	orrs	r2, r1
 8000e80:	605a      	str	r2, [r3, #4]

        /* Enable the Internal High Speed oscillator (HSI or HSIdiv4) */
        __HAL_RCC_HSI_CONFIG(hsi_state);
 8000e82:	4b67      	ldr	r3, [pc, #412]	; (8001020 <HAL_RCC_OscConfig+0x33c>)
 8000e84:	681b      	ldr	r3, [r3, #0]
 8000e86:	2209      	movs	r2, #9
 8000e88:	4393      	bics	r3, r2
 8000e8a:	0019      	movs	r1, r3
 8000e8c:	4b64      	ldr	r3, [pc, #400]	; (8001020 <HAL_RCC_OscConfig+0x33c>)
 8000e8e:	6a7a      	ldr	r2, [r7, #36]	; 0x24
 8000e90:	430a      	orrs	r2, r1
 8000e92:	601a      	str	r2, [r3, #0]
      }

      /* Update the SystemCoreClock global variable */
      SystemCoreClock = HAL_RCC_GetSysClockFreq() >> AHBPrescTable[(RCC->CFGR & RCC_CFGR_HPRE)>> RCC_CFGR_HPRE_Pos];
 8000e94:	f000 fc42 	bl	800171c <HAL_RCC_GetSysClockFreq>
 8000e98:	0001      	movs	r1, r0
 8000e9a:	4b61      	ldr	r3, [pc, #388]	; (8001020 <HAL_RCC_OscConfig+0x33c>)
 8000e9c:	68db      	ldr	r3, [r3, #12]
 8000e9e:	091b      	lsrs	r3, r3, #4
 8000ea0:	220f      	movs	r2, #15
 8000ea2:	4013      	ands	r3, r2
 8000ea4:	4a62      	ldr	r2, [pc, #392]	; (8001030 <HAL_RCC_OscConfig+0x34c>)
 8000ea6:	5cd3      	ldrb	r3, [r2, r3]
 8000ea8:	000a      	movs	r2, r1
 8000eaa:	40da      	lsrs	r2, r3
 8000eac:	4b61      	ldr	r3, [pc, #388]	; (8001034 <HAL_RCC_OscConfig+0x350>)
 8000eae:	601a      	str	r2, [r3, #0]

      /* Configure the source of time base considering new system clocks settings*/
      status = HAL_InitTick (uwTickPrio);
 8000eb0:	4b61      	ldr	r3, [pc, #388]	; (8001038 <HAL_RCC_OscConfig+0x354>)
 8000eb2:	681b      	ldr	r3, [r3, #0]
 8000eb4:	2513      	movs	r5, #19
 8000eb6:	197c      	adds	r4, r7, r5
 8000eb8:	0018      	movs	r0, r3
 8000eba:	f7ff fc4f 	bl	800075c <HAL_InitTick>
 8000ebe:	0003      	movs	r3, r0
 8000ec0:	7023      	strb	r3, [r4, #0]
      if(status != HAL_OK)
 8000ec2:	197b      	adds	r3, r7, r5
 8000ec4:	781b      	ldrb	r3, [r3, #0]
 8000ec6:	2b00      	cmp	r3, #0
 8000ec8:	d046      	beq.n	8000f58 <HAL_RCC_OscConfig+0x274>
      {
        return status;
 8000eca:	197b      	adds	r3, r7, r5
 8000ecc:	781b      	ldrb	r3, [r3, #0]
 8000ece:	e2d2      	b.n	8001476 <HAL_RCC_OscConfig+0x792>
      }
    }
    else
    {
      /* Check the HSI State */
      if(hsi_state != RCC_HSI_OFF)
 8000ed0:	6a7b      	ldr	r3, [r7, #36]	; 0x24
 8000ed2:	2b00      	cmp	r3, #0
 8000ed4:	d027      	beq.n	8000f26 <HAL_RCC_OscConfig+0x242>
      {
        /* Enable the Internal High Speed oscillator (HSI or HSIdiv4) */
        __HAL_RCC_HSI_CONFIG(hsi_state);
 8000ed6:	4b52      	ldr	r3, [pc, #328]	; (8001020 <HAL_RCC_OscConfig+0x33c>)
 8000ed8:	681b      	ldr	r3, [r3, #0]
 8000eda:	2209      	movs	r2, #9
 8000edc:	4393      	bics	r3, r2
 8000ede:	0019      	movs	r1, r3
 8000ee0:	4b4f      	ldr	r3, [pc, #316]	; (8001020 <HAL_RCC_OscConfig+0x33c>)
 8000ee2:	6a7a      	ldr	r2, [r7, #36]	; 0x24
 8000ee4:	430a      	orrs	r2, r1
 8000ee6:	601a      	str	r2, [r3, #0]

        /* Get Start Tick */
        tickstart = HAL_GetTick();
 8000ee8:	f7ff fc7e 	bl	80007e8 <HAL_GetTick>
 8000eec:	0003      	movs	r3, r0
 8000eee:	617b      	str	r3, [r7, #20]

        /* Wait till HSI is ready */
        while(__HAL_RCC_GET_FLAG(RCC_FLAG_HSIRDY) == 0U)
 8000ef0:	e008      	b.n	8000f04 <HAL_RCC_OscConfig+0x220>
        {
          if((HAL_GetTick() - tickstart ) > HSI_TIMEOUT_VALUE)
 8000ef2:	f7ff fc79 	bl	80007e8 <HAL_GetTick>
 8000ef6:	0002      	movs	r2, r0
 8000ef8:	697b      	ldr	r3, [r7, #20]
 8000efa:	1ad3      	subs	r3, r2, r3
 8000efc:	2b02      	cmp	r3, #2
 8000efe:	d901      	bls.n	8000f04 <HAL_RCC_OscConfig+0x220>
          {
            return HAL_TIMEOUT;
 8000f00:	2303      	movs	r3, #3
 8000f02:	e2b8      	b.n	8001476 <HAL_RCC_OscConfig+0x792>
        while(__HAL_RCC_GET_FLAG(RCC_FLAG_HSIRDY) == 0U)
 8000f04:	4b46      	ldr	r3, [pc, #280]	; (8001020 <HAL_RCC_OscConfig+0x33c>)
 8000f06:	681b      	ldr	r3, [r3, #0]
 8000f08:	2204      	movs	r2, #4
 8000f0a:	4013      	ands	r3, r2
 8000f0c:	d0f1      	beq.n	8000ef2 <HAL_RCC_OscConfig+0x20e>
          }
        }

        /* Adjusts the Internal High Speed oscillator (HSI) calibration value.*/
        __HAL_RCC_HSI_CALIBRATIONVALUE_ADJUST(RCC_OscInitStruct->HSICalibrationValue);
 8000f0e:	4b44      	ldr	r3, [pc, #272]	; (8001020 <HAL_RCC_OscConfig+0x33c>)
 8000f10:	685b      	ldr	r3, [r3, #4]
 8000f12:	4a46      	ldr	r2, [pc, #280]	; (800102c <HAL_RCC_OscConfig+0x348>)
 8000f14:	4013      	ands	r3, r2
 8000f16:	0019      	movs	r1, r3
 8000f18:	687b      	ldr	r3, [r7, #4]
 8000f1a:	691b      	ldr	r3, [r3, #16]
 8000f1c:	021a      	lsls	r2, r3, #8
 8000f1e:	4b40      	ldr	r3, [pc, #256]	; (8001020 <HAL_RCC_OscConfig+0x33c>)
 8000f20:	430a      	orrs	r2, r1
 8000f22:	605a      	str	r2, [r3, #4]
 8000f24:	e018      	b.n	8000f58 <HAL_RCC_OscConfig+0x274>
      }
      else
      {
        /* Disable the Internal High Speed oscillator (HSI). */
        __HAL_RCC_HSI_DISABLE();
 8000f26:	4b3e      	ldr	r3, [pc, #248]	; (8001020 <HAL_RCC_OscConfig+0x33c>)
 8000f28:	681a      	ldr	r2, [r3, #0]
 8000f2a:	4b3d      	ldr	r3, [pc, #244]	; (8001020 <HAL_RCC_OscConfig+0x33c>)
 8000f2c:	2101      	movs	r1, #1
 8000f2e:	438a      	bics	r2, r1
 8000f30:	601a      	str	r2, [r3, #0]

        /* Get Start Tick */
        tickstart = HAL_GetTick();
 8000f32:	f7ff fc59 	bl	80007e8 <HAL_GetTick>
 8000f36:	0003      	movs	r3, r0
 8000f38:	617b      	str	r3, [r7, #20]

        /* Wait till HSI is disabled */
        while(__HAL_RCC_GET_FLAG(RCC_FLAG_HSIRDY) != 0U)
 8000f3a:	e008      	b.n	8000f4e <HAL_RCC_OscConfig+0x26a>
        {
          if((HAL_GetTick() - tickstart ) > HSI_TIMEOUT_VALUE)
 8000f3c:	f7ff fc54 	bl	80007e8 <HAL_GetTick>
 8000f40:	0002      	movs	r2, r0
 8000f42:	697b      	ldr	r3, [r7, #20]
 8000f44:	1ad3      	subs	r3, r2, r3
 8000f46:	2b02      	cmp	r3, #2
 8000f48:	d901      	bls.n	8000f4e <HAL_RCC_OscConfig+0x26a>
          {
            return HAL_TIMEOUT;
 8000f4a:	2303      	movs	r3, #3
 8000f4c:	e293      	b.n	8001476 <HAL_RCC_OscConfig+0x792>
        while(__HAL_RCC_GET_FLAG(RCC_FLAG_HSIRDY) != 0U)
 8000f4e:	4b34      	ldr	r3, [pc, #208]	; (8001020 <HAL_RCC_OscConfig+0x33c>)
 8000f50:	681b      	ldr	r3, [r3, #0]
 8000f52:	2204      	movs	r2, #4
 8000f54:	4013      	ands	r3, r2
 8000f56:	d1f1      	bne.n	8000f3c <HAL_RCC_OscConfig+0x258>
        }
      }
    }
  }
  /*----------------------------- MSI Configuration --------------------------*/
  if(((RCC_OscInitStruct->OscillatorType) & RCC_OSCILLATORTYPE_MSI) == RCC_OSCILLATORTYPE_MSI)
 8000f58:	687b      	ldr	r3, [r7, #4]
 8000f5a:	681b      	ldr	r3, [r3, #0]
 8000f5c:	2210      	movs	r2, #16
 8000f5e:	4013      	ands	r3, r2
 8000f60:	d100      	bne.n	8000f64 <HAL_RCC_OscConfig+0x280>
 8000f62:	e0a2      	b.n	80010aa <HAL_RCC_OscConfig+0x3c6>
  {
    /* When the MSI is used as system clock it will not be disabled */
    if(sysclk_source == RCC_CFGR_SWS_MSI)
 8000f64:	69fb      	ldr	r3, [r7, #28]
 8000f66:	2b00      	cmp	r3, #0
 8000f68:	d140      	bne.n	8000fec <HAL_RCC_OscConfig+0x308>
    {
      if((__HAL_RCC_GET_FLAG(RCC_FLAG_MSIRDY) != 0U) && (RCC_OscInitStruct->MSIState == RCC_MSI_OFF))
 8000f6a:	4b2d      	ldr	r3, [pc, #180]	; (8001020 <HAL_RCC_OscConfig+0x33c>)
 8000f6c:	681a      	ldr	r2, [r3, #0]
 8000f6e:	2380      	movs	r3, #128	; 0x80
 8000f70:	009b      	lsls	r3, r3, #2
 8000f72:	4013      	ands	r3, r2
 8000f74:	d005      	beq.n	8000f82 <HAL_RCC_OscConfig+0x29e>
 8000f76:	687b      	ldr	r3, [r7, #4]
 8000f78:	69db      	ldr	r3, [r3, #28]
 8000f7a:	2b00      	cmp	r3, #0
 8000f7c:	d101      	bne.n	8000f82 <HAL_RCC_OscConfig+0x29e>
      {
        return HAL_ERROR;
 8000f7e:	2301      	movs	r3, #1
 8000f80:	e279      	b.n	8001476 <HAL_RCC_OscConfig+0x792>
        /* Check MSICalibrationValue and MSIClockRange input parameters */
        assert_param(IS_RCC_MSICALIBRATION_VALUE(RCC_OscInitStruct->MSICalibrationValue));
        assert_param(IS_RCC_MSI_CLOCK_RANGE(RCC_OscInitStruct->MSIClockRange));

        /* Selects the Multiple Speed oscillator (MSI) clock range .*/
        __HAL_RCC_MSI_RANGE_CONFIG(RCC_OscInitStruct->MSIClockRange);
 8000f82:	4b27      	ldr	r3, [pc, #156]	; (8001020 <HAL_RCC_OscConfig+0x33c>)
 8000f84:	685b      	ldr	r3, [r3, #4]
 8000f86:	4a2d      	ldr	r2, [pc, #180]	; (800103c <HAL_RCC_OscConfig+0x358>)
 8000f88:	4013      	ands	r3, r2
 8000f8a:	0019      	movs	r1, r3
 8000f8c:	687b      	ldr	r3, [r7, #4]
 8000f8e:	6a5a      	ldr	r2, [r3, #36]	; 0x24
 8000f90:	4b23      	ldr	r3, [pc, #140]	; (8001020 <HAL_RCC_OscConfig+0x33c>)
 8000f92:	430a      	orrs	r2, r1
 8000f94:	605a      	str	r2, [r3, #4]
        /* Adjusts the Multiple Speed oscillator (MSI) calibration value.*/
        __HAL_RCC_MSI_CALIBRATIONVALUE_ADJUST(RCC_OscInitStruct->MSICalibrationValue);
 8000f96:	4b22      	ldr	r3, [pc, #136]	; (8001020 <HAL_RCC_OscConfig+0x33c>)
 8000f98:	685b      	ldr	r3, [r3, #4]
 8000f9a:	021b      	lsls	r3, r3, #8
 8000f9c:	0a19      	lsrs	r1, r3, #8
 8000f9e:	687b      	ldr	r3, [r7, #4]
 8000fa0:	6a1b      	ldr	r3, [r3, #32]
 8000fa2:	061a      	lsls	r2, r3, #24
 8000fa4:	4b1e      	ldr	r3, [pc, #120]	; (8001020 <HAL_RCC_OscConfig+0x33c>)
 8000fa6:	430a      	orrs	r2, r1
 8000fa8:	605a      	str	r2, [r3, #4]


        /* Update the SystemCoreClock global variable */
        SystemCoreClock =  (32768U * (1UL << ((RCC_OscInitStruct->MSIClockRange >> RCC_ICSCR_MSIRANGE_Pos) + 1U)))
 8000faa:	687b      	ldr	r3, [r7, #4]
 8000fac:	6a5b      	ldr	r3, [r3, #36]	; 0x24
 8000fae:	0b5b      	lsrs	r3, r3, #13
 8000fb0:	3301      	adds	r3, #1
 8000fb2:	2280      	movs	r2, #128	; 0x80
 8000fb4:	0212      	lsls	r2, r2, #8
 8000fb6:	409a      	lsls	r2, r3
                           >> AHBPrescTable[((RCC->CFGR & RCC_CFGR_HPRE) >> RCC_CFGR_HPRE_Pos)];
 8000fb8:	4b19      	ldr	r3, [pc, #100]	; (8001020 <HAL_RCC_OscConfig+0x33c>)
 8000fba:	68db      	ldr	r3, [r3, #12]
 8000fbc:	091b      	lsrs	r3, r3, #4
 8000fbe:	210f      	movs	r1, #15
 8000fc0:	400b      	ands	r3, r1
 8000fc2:	491b      	ldr	r1, [pc, #108]	; (8001030 <HAL_RCC_OscConfig+0x34c>)
 8000fc4:	5ccb      	ldrb	r3, [r1, r3]
 8000fc6:	40da      	lsrs	r2, r3
        SystemCoreClock =  (32768U * (1UL << ((RCC_OscInitStruct->MSIClockRange >> RCC_ICSCR_MSIRANGE_Pos) + 1U)))
 8000fc8:	4b1a      	ldr	r3, [pc, #104]	; (8001034 <HAL_RCC_OscConfig+0x350>)
 8000fca:	601a      	str	r2, [r3, #0]

        /* Configure the source of time base considering new system clocks settings*/
        status = HAL_InitTick (uwTickPrio);
 8000fcc:	4b1a      	ldr	r3, [pc, #104]	; (8001038 <HAL_RCC_OscConfig+0x354>)
 8000fce:	681b      	ldr	r3, [r3, #0]
 8000fd0:	2513      	movs	r5, #19
 8000fd2:	197c      	adds	r4, r7, r5
 8000fd4:	0018      	movs	r0, r3
 8000fd6:	f7ff fbc1 	bl	800075c <HAL_InitTick>
 8000fda:	0003      	movs	r3, r0
 8000fdc:	7023      	strb	r3, [r4, #0]
        if(status != HAL_OK)
 8000fde:	197b      	adds	r3, r7, r5
 8000fe0:	781b      	ldrb	r3, [r3, #0]
 8000fe2:	2b00      	cmp	r3, #0
 8000fe4:	d061      	beq.n	80010aa <HAL_RCC_OscConfig+0x3c6>
        {
          return status;
 8000fe6:	197b      	adds	r3, r7, r5
 8000fe8:	781b      	ldrb	r3, [r3, #0]
 8000fea:	e244      	b.n	8001476 <HAL_RCC_OscConfig+0x792>
    {
      /* Check MSI State */
      assert_param(IS_RCC_MSI(RCC_OscInitStruct->MSIState));

      /* Check the MSI State */
      if(RCC_OscInitStruct->MSIState != RCC_MSI_OFF)
 8000fec:	687b      	ldr	r3, [r7, #4]
 8000fee:	69db      	ldr	r3, [r3, #28]
 8000ff0:	2b00      	cmp	r3, #0
 8000ff2:	d040      	beq.n	8001076 <HAL_RCC_OscConfig+0x392>
      {
        /* Enable the Multi Speed oscillator (MSI). */
        __HAL_RCC_MSI_ENABLE();
 8000ff4:	4b0a      	ldr	r3, [pc, #40]	; (8001020 <HAL_RCC_OscConfig+0x33c>)
 8000ff6:	681a      	ldr	r2, [r3, #0]
 8000ff8:	4b09      	ldr	r3, [pc, #36]	; (8001020 <HAL_RCC_OscConfig+0x33c>)
 8000ffa:	2180      	movs	r1, #128	; 0x80
 8000ffc:	0049      	lsls	r1, r1, #1
 8000ffe:	430a      	orrs	r2, r1
 8001000:	601a      	str	r2, [r3, #0]

        /* Get Start Tick */
        tickstart = HAL_GetTick();
 8001002:	f7ff fbf1 	bl	80007e8 <HAL_GetTick>
 8001006:	0003      	movs	r3, r0
 8001008:	617b      	str	r3, [r7, #20]

        /* Wait till MSI is ready */
        while(__HAL_RCC_GET_FLAG(RCC_FLAG_MSIRDY) == 0U)
 800100a:	e019      	b.n	8001040 <HAL_RCC_OscConfig+0x35c>
        {
          if((HAL_GetTick() - tickstart) > MSI_TIMEOUT_VALUE)
 800100c:	f7ff fbec 	bl	80007e8 <HAL_GetTick>
 8001010:	0002      	movs	r2, r0
 8001012:	697b      	ldr	r3, [r7, #20]
 8001014:	1ad3      	subs	r3, r2, r3
 8001016:	2b02      	cmp	r3, #2
 8001018:	d912      	bls.n	8001040 <HAL_RCC_OscConfig+0x35c>
          {
            return HAL_TIMEOUT;
 800101a:	2303      	movs	r3, #3
 800101c:	e22b      	b.n	8001476 <HAL_RCC_OscConfig+0x792>
 800101e:	46c0      	nop			; (mov r8, r8)
 8001020:	40021000 	.word	0x40021000
 8001024:	fffeffff 	.word	0xfffeffff
 8001028:	fffbffff 	.word	0xfffbffff
 800102c:	ffffe0ff 	.word	0xffffe0ff
 8001030:	080018d8 	.word	0x080018d8
 8001034:	20000000 	.word	0x20000000
 8001038:	20000004 	.word	0x20000004
 800103c:	ffff1fff 	.word	0xffff1fff
        while(__HAL_RCC_GET_FLAG(RCC_FLAG_MSIRDY) == 0U)
 8001040:	4bca      	ldr	r3, [pc, #808]	; (800136c <HAL_RCC_OscConfig+0x688>)
 8001042:	681a      	ldr	r2, [r3, #0]
 8001044:	2380      	movs	r3, #128	; 0x80
 8001046:	009b      	lsls	r3, r3, #2
 8001048:	4013      	ands	r3, r2
 800104a:	d0df      	beq.n	800100c <HAL_RCC_OscConfig+0x328>
        /* Check MSICalibrationValue and MSIClockRange input parameters */
        assert_param(IS_RCC_MSICALIBRATION_VALUE(RCC_OscInitStruct->MSICalibrationValue));
        assert_param(IS_RCC_MSI_CLOCK_RANGE(RCC_OscInitStruct->MSIClockRange));

        /* Selects the Multiple Speed oscillator (MSI) clock range .*/
        __HAL_RCC_MSI_RANGE_CONFIG(RCC_OscInitStruct->MSIClockRange);
 800104c:	4bc7      	ldr	r3, [pc, #796]	; (800136c <HAL_RCC_OscConfig+0x688>)
 800104e:	685b      	ldr	r3, [r3, #4]
 8001050:	4ac7      	ldr	r2, [pc, #796]	; (8001370 <HAL_RCC_OscConfig+0x68c>)
 8001052:	4013      	ands	r3, r2
 8001054:	0019      	movs	r1, r3
 8001056:	687b      	ldr	r3, [r7, #4]
 8001058:	6a5a      	ldr	r2, [r3, #36]	; 0x24
 800105a:	4bc4      	ldr	r3, [pc, #784]	; (800136c <HAL_RCC_OscConfig+0x688>)
 800105c:	430a      	orrs	r2, r1
 800105e:	605a      	str	r2, [r3, #4]
         /* Adjusts the Multiple Speed oscillator (MSI) calibration value.*/
        __HAL_RCC_MSI_CALIBRATIONVALUE_ADJUST(RCC_OscInitStruct->MSICalibrationValue);
 8001060:	4bc2      	ldr	r3, [pc, #776]	; (800136c <HAL_RCC_OscConfig+0x688>)
 8001062:	685b      	ldr	r3, [r3, #4]
 8001064:	021b      	lsls	r3, r3, #8
 8001066:	0a19      	lsrs	r1, r3, #8
 8001068:	687b      	ldr	r3, [r7, #4]
 800106a:	6a1b      	ldr	r3, [r3, #32]
 800106c:	061a      	lsls	r2, r3, #24
 800106e:	4bbf      	ldr	r3, [pc, #764]	; (800136c <HAL_RCC_OscConfig+0x688>)
 8001070:	430a      	orrs	r2, r1
 8001072:	605a      	str	r2, [r3, #4]
 8001074:	e019      	b.n	80010aa <HAL_RCC_OscConfig+0x3c6>
      }
      else
      {
        /* Disable the Multi Speed oscillator (MSI). */
        __HAL_RCC_MSI_DISABLE();
 8001076:	4bbd      	ldr	r3, [pc, #756]	; (800136c <HAL_RCC_OscConfig+0x688>)
 8001078:	681a      	ldr	r2, [r3, #0]
 800107a:	4bbc      	ldr	r3, [pc, #752]	; (800136c <HAL_RCC_OscConfig+0x688>)
 800107c:	49bd      	ldr	r1, [pc, #756]	; (8001374 <HAL_RCC_OscConfig+0x690>)
 800107e:	400a      	ands	r2, r1
 8001080:	601a      	str	r2, [r3, #0]

        /* Get Start Tick */
        tickstart = HAL_GetTick();
 8001082:	f7ff fbb1 	bl	80007e8 <HAL_GetTick>
 8001086:	0003      	movs	r3, r0
 8001088:	617b      	str	r3, [r7, #20]

        /* Wait till MSI is ready */
        while(__HAL_RCC_GET_FLAG(RCC_FLAG_MSIRDY) != 0U)
 800108a:	e008      	b.n	800109e <HAL_RCC_OscConfig+0x3ba>
        {
          if((HAL_GetTick() - tickstart) > MSI_TIMEOUT_VALUE)
 800108c:	f7ff fbac 	bl	80007e8 <HAL_GetTick>
 8001090:	0002      	movs	r2, r0
 8001092:	697b      	ldr	r3, [r7, #20]
 8001094:	1ad3      	subs	r3, r2, r3
 8001096:	2b02      	cmp	r3, #2
 8001098:	d901      	bls.n	800109e <HAL_RCC_OscConfig+0x3ba>
          {
            return HAL_TIMEOUT;
 800109a:	2303      	movs	r3, #3
 800109c:	e1eb      	b.n	8001476 <HAL_RCC_OscConfig+0x792>
        while(__HAL_RCC_GET_FLAG(RCC_FLAG_MSIRDY) != 0U)
 800109e:	4bb3      	ldr	r3, [pc, #716]	; (800136c <HAL_RCC_OscConfig+0x688>)
 80010a0:	681a      	ldr	r2, [r3, #0]
 80010a2:	2380      	movs	r3, #128	; 0x80
 80010a4:	009b      	lsls	r3, r3, #2
 80010a6:	4013      	ands	r3, r2
 80010a8:	d1f0      	bne.n	800108c <HAL_RCC_OscConfig+0x3a8>
        }
      }
    }
  }
  /*------------------------------ LSI Configuration -------------------------*/
  if(((RCC_OscInitStruct->OscillatorType) & RCC_OSCILLATORTYPE_LSI) == RCC_OSCILLATORTYPE_LSI)
 80010aa:	687b      	ldr	r3, [r7, #4]
 80010ac:	681b      	ldr	r3, [r3, #0]
 80010ae:	2208      	movs	r2, #8
 80010b0:	4013      	ands	r3, r2
 80010b2:	d036      	beq.n	8001122 <HAL_RCC_OscConfig+0x43e>
  {
    /* Check the parameters */
    assert_param(IS_RCC_LSI(RCC_OscInitStruct->LSIState));

    /* Check the LSI State */
    if(RCC_OscInitStruct->LSIState != RCC_LSI_OFF)
 80010b4:	687b      	ldr	r3, [r7, #4]
 80010b6:	695b      	ldr	r3, [r3, #20]
 80010b8:	2b00      	cmp	r3, #0
 80010ba:	d019      	beq.n	80010f0 <HAL_RCC_OscConfig+0x40c>
    {
      /* Enable the Internal Low Speed oscillator (LSI). */
      __HAL_RCC_LSI_ENABLE();
 80010bc:	4bab      	ldr	r3, [pc, #684]	; (800136c <HAL_RCC_OscConfig+0x688>)
 80010be:	6d1a      	ldr	r2, [r3, #80]	; 0x50
 80010c0:	4baa      	ldr	r3, [pc, #680]	; (800136c <HAL_RCC_OscConfig+0x688>)
 80010c2:	2101      	movs	r1, #1
 80010c4:	430a      	orrs	r2, r1
 80010c6:	651a      	str	r2, [r3, #80]	; 0x50

      /* Get Start Tick */
      tickstart = HAL_GetTick();
 80010c8:	f7ff fb8e 	bl	80007e8 <HAL_GetTick>
 80010cc:	0003      	movs	r3, r0
 80010ce:	617b      	str	r3, [r7, #20]

      /* Wait till LSI is ready */
      while(__HAL_RCC_GET_FLAG(RCC_FLAG_LSIRDY) == 0U)
 80010d0:	e008      	b.n	80010e4 <HAL_RCC_OscConfig+0x400>
      {
        if((HAL_GetTick() - tickstart ) > LSI_TIMEOUT_VALUE)
 80010d2:	f7ff fb89 	bl	80007e8 <HAL_GetTick>
 80010d6:	0002      	movs	r2, r0
 80010d8:	697b      	ldr	r3, [r7, #20]
 80010da:	1ad3      	subs	r3, r2, r3
 80010dc:	2b02      	cmp	r3, #2
 80010de:	d901      	bls.n	80010e4 <HAL_RCC_OscConfig+0x400>
        {
          return HAL_TIMEOUT;
 80010e0:	2303      	movs	r3, #3
 80010e2:	e1c8      	b.n	8001476 <HAL_RCC_OscConfig+0x792>
      while(__HAL_RCC_GET_FLAG(RCC_FLAG_LSIRDY) == 0U)
 80010e4:	4ba1      	ldr	r3, [pc, #644]	; (800136c <HAL_RCC_OscConfig+0x688>)
 80010e6:	6d1b      	ldr	r3, [r3, #80]	; 0x50
 80010e8:	2202      	movs	r2, #2
 80010ea:	4013      	ands	r3, r2
 80010ec:	d0f1      	beq.n	80010d2 <HAL_RCC_OscConfig+0x3ee>
 80010ee:	e018      	b.n	8001122 <HAL_RCC_OscConfig+0x43e>
      }
    }
    else
    {
      /* Disable the Internal Low Speed oscillator (LSI). */
      __HAL_RCC_LSI_DISABLE();
 80010f0:	4b9e      	ldr	r3, [pc, #632]	; (800136c <HAL_RCC_OscConfig+0x688>)
 80010f2:	6d1a      	ldr	r2, [r3, #80]	; 0x50
 80010f4:	4b9d      	ldr	r3, [pc, #628]	; (800136c <HAL_RCC_OscConfig+0x688>)
 80010f6:	2101      	movs	r1, #1
 80010f8:	438a      	bics	r2, r1
 80010fa:	651a      	str	r2, [r3, #80]	; 0x50

      /* Get Start Tick */
      tickstart = HAL_GetTick();
 80010fc:	f7ff fb74 	bl	80007e8 <HAL_GetTick>
 8001100:	0003      	movs	r3, r0
 8001102:	617b      	str	r3, [r7, #20]

      /* Wait till LSI is disabled */
      while(__HAL_RCC_GET_FLAG(RCC_FLAG_LSIRDY) != 0U)
 8001104:	e008      	b.n	8001118 <HAL_RCC_OscConfig+0x434>
      {
        if((HAL_GetTick() - tickstart ) > LSI_TIMEOUT_VALUE)
 8001106:	f7ff fb6f 	bl	80007e8 <HAL_GetTick>
 800110a:	0002      	movs	r2, r0
 800110c:	697b      	ldr	r3, [r7, #20]
 800110e:	1ad3      	subs	r3, r2, r3
 8001110:	2b02      	cmp	r3, #2
 8001112:	d901      	bls.n	8001118 <HAL_RCC_OscConfig+0x434>
        {
          return HAL_TIMEOUT;
 8001114:	2303      	movs	r3, #3
 8001116:	e1ae      	b.n	8001476 <HAL_RCC_OscConfig+0x792>
      while(__HAL_RCC_GET_FLAG(RCC_FLAG_LSIRDY) != 0U)
 8001118:	4b94      	ldr	r3, [pc, #592]	; (800136c <HAL_RCC_OscConfig+0x688>)
 800111a:	6d1b      	ldr	r3, [r3, #80]	; 0x50
 800111c:	2202      	movs	r2, #2
 800111e:	4013      	ands	r3, r2
 8001120:	d1f1      	bne.n	8001106 <HAL_RCC_OscConfig+0x422>
        }
      }
    }
  }
  /*------------------------------ LSE Configuration -------------------------*/
  if(((RCC_OscInitStruct->OscillatorType) & RCC_OSCILLATORTYPE_LSE) == RCC_OSCILLATORTYPE_LSE)
 8001122:	687b      	ldr	r3, [r7, #4]
 8001124:	681b      	ldr	r3, [r3, #0]
 8001126:	2204      	movs	r2, #4
 8001128:	4013      	ands	r3, r2
 800112a:	d100      	bne.n	800112e <HAL_RCC_OscConfig+0x44a>
 800112c:	e0ae      	b.n	800128c <HAL_RCC_OscConfig+0x5a8>
  {
    FlagStatus       pwrclkchanged = RESET;
 800112e:	2023      	movs	r0, #35	; 0x23
 8001130:	183b      	adds	r3, r7, r0
 8001132:	2200      	movs	r2, #0
 8001134:	701a      	strb	r2, [r3, #0]
    /* Check the parameters */
    assert_param(IS_RCC_LSE(RCC_OscInitStruct->LSEState));

    /* Update LSE configuration in Backup Domain control register    */
    /* Requires to enable write access to Backup Domain of necessary */
    if(__HAL_RCC_PWR_IS_CLK_DISABLED())
 8001136:	4b8d      	ldr	r3, [pc, #564]	; (800136c <HAL_RCC_OscConfig+0x688>)
 8001138:	6b9a      	ldr	r2, [r3, #56]	; 0x38
 800113a:	2380      	movs	r3, #128	; 0x80
 800113c:	055b      	lsls	r3, r3, #21
 800113e:	4013      	ands	r3, r2
 8001140:	d109      	bne.n	8001156 <HAL_RCC_OscConfig+0x472>
    {
      __HAL_RCC_PWR_CLK_ENABLE();
 8001142:	4b8a      	ldr	r3, [pc, #552]	; (800136c <HAL_RCC_OscConfig+0x688>)
 8001144:	6b9a      	ldr	r2, [r3, #56]	; 0x38
 8001146:	4b89      	ldr	r3, [pc, #548]	; (800136c <HAL_RCC_OscConfig+0x688>)
 8001148:	2180      	movs	r1, #128	; 0x80
 800114a:	0549      	lsls	r1, r1, #21
 800114c:	430a      	orrs	r2, r1
 800114e:	639a      	str	r2, [r3, #56]	; 0x38
      pwrclkchanged = SET;
 8001150:	183b      	adds	r3, r7, r0
 8001152:	2201      	movs	r2, #1
 8001154:	701a      	strb	r2, [r3, #0]
    }

    if(HAL_IS_BIT_CLR(PWR->CR, PWR_CR_DBP))
 8001156:	4b88      	ldr	r3, [pc, #544]	; (8001378 <HAL_RCC_OscConfig+0x694>)
 8001158:	681a      	ldr	r2, [r3, #0]
 800115a:	2380      	movs	r3, #128	; 0x80
 800115c:	005b      	lsls	r3, r3, #1
 800115e:	4013      	ands	r3, r2
 8001160:	d11a      	bne.n	8001198 <HAL_RCC_OscConfig+0x4b4>
    {
      /* Enable write access to Backup domain */
      SET_BIT(PWR->CR, PWR_CR_DBP);
 8001162:	4b85      	ldr	r3, [pc, #532]	; (8001378 <HAL_RCC_OscConfig+0x694>)
 8001164:	681a      	ldr	r2, [r3, #0]
 8001166:	4b84      	ldr	r3, [pc, #528]	; (8001378 <HAL_RCC_OscConfig+0x694>)
 8001168:	2180      	movs	r1, #128	; 0x80
 800116a:	0049      	lsls	r1, r1, #1
 800116c:	430a      	orrs	r2, r1
 800116e:	601a      	str	r2, [r3, #0]

      /* Wait for Backup domain Write protection disable */
      tickstart = HAL_GetTick();
 8001170:	f7ff fb3a 	bl	80007e8 <HAL_GetTick>
 8001174:	0003      	movs	r3, r0
 8001176:	617b      	str	r3, [r7, #20]

      while(HAL_IS_BIT_CLR(PWR->CR, PWR_CR_DBP))
 8001178:	e008      	b.n	800118c <HAL_RCC_OscConfig+0x4a8>
      {
        if((HAL_GetTick() - tickstart) > RCC_DBP_TIMEOUT_VALUE)
 800117a:	f7ff fb35 	bl	80007e8 <HAL_GetTick>
 800117e:	0002      	movs	r2, r0
 8001180:	697b      	ldr	r3, [r7, #20]
 8001182:	1ad3      	subs	r3, r2, r3
 8001184:	2b64      	cmp	r3, #100	; 0x64
 8001186:	d901      	bls.n	800118c <HAL_RCC_OscConfig+0x4a8>
        {
          return HAL_TIMEOUT;
 8001188:	2303      	movs	r3, #3
 800118a:	e174      	b.n	8001476 <HAL_RCC_OscConfig+0x792>
      while(HAL_IS_BIT_CLR(PWR->CR, PWR_CR_DBP))
 800118c:	4b7a      	ldr	r3, [pc, #488]	; (8001378 <HAL_RCC_OscConfig+0x694>)
 800118e:	681a      	ldr	r2, [r3, #0]
 8001190:	2380      	movs	r3, #128	; 0x80
 8001192:	005b      	lsls	r3, r3, #1
 8001194:	4013      	ands	r3, r2
 8001196:	d0f0      	beq.n	800117a <HAL_RCC_OscConfig+0x496>
        }
      }
    }

    /* Set the new LSE configuration -----------------------------------------*/
    __HAL_RCC_LSE_CONFIG(RCC_OscInitStruct->LSEState);
 8001198:	687b      	ldr	r3, [r7, #4]
 800119a:	689a      	ldr	r2, [r3, #8]
 800119c:	2380      	movs	r3, #128	; 0x80
 800119e:	005b      	lsls	r3, r3, #1
 80011a0:	429a      	cmp	r2, r3
 80011a2:	d107      	bne.n	80011b4 <HAL_RCC_OscConfig+0x4d0>
 80011a4:	4b71      	ldr	r3, [pc, #452]	; (800136c <HAL_RCC_OscConfig+0x688>)
 80011a6:	6d1a      	ldr	r2, [r3, #80]	; 0x50
 80011a8:	4b70      	ldr	r3, [pc, #448]	; (800136c <HAL_RCC_OscConfig+0x688>)
 80011aa:	2180      	movs	r1, #128	; 0x80
 80011ac:	0049      	lsls	r1, r1, #1
 80011ae:	430a      	orrs	r2, r1
 80011b0:	651a      	str	r2, [r3, #80]	; 0x50
 80011b2:	e031      	b.n	8001218 <HAL_RCC_OscConfig+0x534>
 80011b4:	687b      	ldr	r3, [r7, #4]
 80011b6:	689b      	ldr	r3, [r3, #8]
 80011b8:	2b00      	cmp	r3, #0
 80011ba:	d10c      	bne.n	80011d6 <HAL_RCC_OscConfig+0x4f2>
 80011bc:	4b6b      	ldr	r3, [pc, #428]	; (800136c <HAL_RCC_OscConfig+0x688>)
 80011be:	6d1a      	ldr	r2, [r3, #80]	; 0x50
 80011c0:	4b6a      	ldr	r3, [pc, #424]	; (800136c <HAL_RCC_OscConfig+0x688>)
 80011c2:	496c      	ldr	r1, [pc, #432]	; (8001374 <HAL_RCC_OscConfig+0x690>)
 80011c4:	400a      	ands	r2, r1
 80011c6:	651a      	str	r2, [r3, #80]	; 0x50
 80011c8:	4b68      	ldr	r3, [pc, #416]	; (800136c <HAL_RCC_OscConfig+0x688>)
 80011ca:	6d1a      	ldr	r2, [r3, #80]	; 0x50
 80011cc:	4b67      	ldr	r3, [pc, #412]	; (800136c <HAL_RCC_OscConfig+0x688>)
 80011ce:	496b      	ldr	r1, [pc, #428]	; (800137c <HAL_RCC_OscConfig+0x698>)
 80011d0:	400a      	ands	r2, r1
 80011d2:	651a      	str	r2, [r3, #80]	; 0x50
 80011d4:	e020      	b.n	8001218 <HAL_RCC_OscConfig+0x534>
 80011d6:	687b      	ldr	r3, [r7, #4]
 80011d8:	689a      	ldr	r2, [r3, #8]
 80011da:	23a0      	movs	r3, #160	; 0xa0
 80011dc:	00db      	lsls	r3, r3, #3
 80011de:	429a      	cmp	r2, r3
 80011e0:	d10e      	bne.n	8001200 <HAL_RCC_OscConfig+0x51c>
 80011e2:	4b62      	ldr	r3, [pc, #392]	; (800136c <HAL_RCC_OscConfig+0x688>)
 80011e4:	6d1a      	ldr	r2, [r3, #80]	; 0x50
 80011e6:	4b61      	ldr	r3, [pc, #388]	; (800136c <HAL_RCC_OscConfig+0x688>)
 80011e8:	2180      	movs	r1, #128	; 0x80
 80011ea:	00c9      	lsls	r1, r1, #3
 80011ec:	430a      	orrs	r2, r1
 80011ee:	651a      	str	r2, [r3, #80]	; 0x50
 80011f0:	4b5e      	ldr	r3, [pc, #376]	; (800136c <HAL_RCC_OscConfig+0x688>)
 80011f2:	6d1a      	ldr	r2, [r3, #80]	; 0x50
 80011f4:	4b5d      	ldr	r3, [pc, #372]	; (800136c <HAL_RCC_OscConfig+0x688>)
 80011f6:	2180      	movs	r1, #128	; 0x80
 80011f8:	0049      	lsls	r1, r1, #1
 80011fa:	430a      	orrs	r2, r1
 80011fc:	651a      	str	r2, [r3, #80]	; 0x50
 80011fe:	e00b      	b.n	8001218 <HAL_RCC_OscConfig+0x534>
 8001200:	4b5a      	ldr	r3, [pc, #360]	; (800136c <HAL_RCC_OscConfig+0x688>)
 8001202:	6d1a      	ldr	r2, [r3, #80]	; 0x50
 8001204:	4b59      	ldr	r3, [pc, #356]	; (800136c <HAL_RCC_OscConfig+0x688>)
 8001206:	495b      	ldr	r1, [pc, #364]	; (8001374 <HAL_RCC_OscConfig+0x690>)
 8001208:	400a      	ands	r2, r1
 800120a:	651a      	str	r2, [r3, #80]	; 0x50
 800120c:	4b57      	ldr	r3, [pc, #348]	; (800136c <HAL_RCC_OscConfig+0x688>)
 800120e:	6d1a      	ldr	r2, [r3, #80]	; 0x50
 8001210:	4b56      	ldr	r3, [pc, #344]	; (800136c <HAL_RCC_OscConfig+0x688>)
 8001212:	495a      	ldr	r1, [pc, #360]	; (800137c <HAL_RCC_OscConfig+0x698>)
 8001214:	400a      	ands	r2, r1
 8001216:	651a      	str	r2, [r3, #80]	; 0x50

    /* Check the LSE State */
    if(RCC_OscInitStruct->LSEState != RCC_LSE_OFF)
 8001218:	687b      	ldr	r3, [r7, #4]
 800121a:	689b      	ldr	r3, [r3, #8]
 800121c:	2b00      	cmp	r3, #0
 800121e:	d015      	beq.n	800124c <HAL_RCC_OscConfig+0x568>
    {
      /* Get Start Tick */
      tickstart = HAL_GetTick();
 8001220:	f7ff fae2 	bl	80007e8 <HAL_GetTick>
 8001224:	0003      	movs	r3, r0
 8001226:	617b      	str	r3, [r7, #20]

      /* Wait till LSE is ready */
      while(__HAL_RCC_GET_FLAG(RCC_FLAG_LSERDY) == 0U)
 8001228:	e009      	b.n	800123e <HAL_RCC_OscConfig+0x55a>
      {
        if((HAL_GetTick() - tickstart ) > RCC_LSE_TIMEOUT_VALUE)
 800122a:	f7ff fadd 	bl	80007e8 <HAL_GetTick>
 800122e:	0002      	movs	r2, r0
 8001230:	697b      	ldr	r3, [r7, #20]
 8001232:	1ad3      	subs	r3, r2, r3
 8001234:	4a52      	ldr	r2, [pc, #328]	; (8001380 <HAL_RCC_OscConfig+0x69c>)
 8001236:	4293      	cmp	r3, r2
 8001238:	d901      	bls.n	800123e <HAL_RCC_OscConfig+0x55a>
        {
          return HAL_TIMEOUT;
 800123a:	2303      	movs	r3, #3
 800123c:	e11b      	b.n	8001476 <HAL_RCC_OscConfig+0x792>
      while(__HAL_RCC_GET_FLAG(RCC_FLAG_LSERDY) == 0U)
 800123e:	4b4b      	ldr	r3, [pc, #300]	; (800136c <HAL_RCC_OscConfig+0x688>)
 8001240:	6d1a      	ldr	r2, [r3, #80]	; 0x50
 8001242:	2380      	movs	r3, #128	; 0x80
 8001244:	009b      	lsls	r3, r3, #2
 8001246:	4013      	ands	r3, r2
 8001248:	d0ef      	beq.n	800122a <HAL_RCC_OscConfig+0x546>
 800124a:	e014      	b.n	8001276 <HAL_RCC_OscConfig+0x592>
      }
    }
    else
    {
      /* Get Start Tick */
      tickstart = HAL_GetTick();
 800124c:	f7ff facc 	bl	80007e8 <HAL_GetTick>
 8001250:	0003      	movs	r3, r0
 8001252:	617b      	str	r3, [r7, #20]

      /* Wait till LSE is disabled */
      while(__HAL_RCC_GET_FLAG(RCC_FLAG_LSERDY) != 0U)
 8001254:	e009      	b.n	800126a <HAL_RCC_OscConfig+0x586>
      {
        if((HAL_GetTick() - tickstart ) > RCC_LSE_TIMEOUT_VALUE)
 8001256:	f7ff fac7 	bl	80007e8 <HAL_GetTick>
 800125a:	0002      	movs	r2, r0
 800125c:	697b      	ldr	r3, [r7, #20]
 800125e:	1ad3      	subs	r3, r2, r3
 8001260:	4a47      	ldr	r2, [pc, #284]	; (8001380 <HAL_RCC_OscConfig+0x69c>)
 8001262:	4293      	cmp	r3, r2
 8001264:	d901      	bls.n	800126a <HAL_RCC_OscConfig+0x586>
        {
          return HAL_TIMEOUT;
 8001266:	2303      	movs	r3, #3
 8001268:	e105      	b.n	8001476 <HAL_RCC_OscConfig+0x792>
      while(__HAL_RCC_GET_FLAG(RCC_FLAG_LSERDY) != 0U)
 800126a:	4b40      	ldr	r3, [pc, #256]	; (800136c <HAL_RCC_OscConfig+0x688>)
 800126c:	6d1a      	ldr	r2, [r3, #80]	; 0x50
 800126e:	2380      	movs	r3, #128	; 0x80
 8001270:	009b      	lsls	r3, r3, #2
 8001272:	4013      	ands	r3, r2
 8001274:	d1ef      	bne.n	8001256 <HAL_RCC_OscConfig+0x572>
        }
      }
    }

    /* Require to disable power clock if necessary */
    if(pwrclkchanged == SET)
 8001276:	2323      	movs	r3, #35	; 0x23
 8001278:	18fb      	adds	r3, r7, r3
 800127a:	781b      	ldrb	r3, [r3, #0]
 800127c:	2b01      	cmp	r3, #1
 800127e:	d105      	bne.n	800128c <HAL_RCC_OscConfig+0x5a8>
    {
      __HAL_RCC_PWR_CLK_DISABLE();
 8001280:	4b3a      	ldr	r3, [pc, #232]	; (800136c <HAL_RCC_OscConfig+0x688>)
 8001282:	6b9a      	ldr	r2, [r3, #56]	; 0x38
 8001284:	4b39      	ldr	r3, [pc, #228]	; (800136c <HAL_RCC_OscConfig+0x688>)
 8001286:	493f      	ldr	r1, [pc, #252]	; (8001384 <HAL_RCC_OscConfig+0x6a0>)
 8001288:	400a      	ands	r2, r1
 800128a:	639a      	str	r2, [r3, #56]	; 0x38
    }
  }

#if defined(RCC_HSI48_SUPPORT)
  /*----------------------------- HSI48 Configuration --------------------------*/
  if(((RCC_OscInitStruct->OscillatorType) & RCC_OSCILLATORTYPE_HSI48) == RCC_OSCILLATORTYPE_HSI48)
 800128c:	687b      	ldr	r3, [r7, #4]
 800128e:	681b      	ldr	r3, [r3, #0]
 8001290:	2220      	movs	r2, #32
 8001292:	4013      	ands	r3, r2
 8001294:	d049      	beq.n	800132a <HAL_RCC_OscConfig+0x646>
  {
    /* Check the parameters */
    assert_param(IS_RCC_HSI48(RCC_OscInitStruct->HSI48State));

      /* Check the HSI48 State */
      if(RCC_OscInitStruct->HSI48State != RCC_HSI48_OFF)
 8001296:	687b      	ldr	r3, [r7, #4]
 8001298:	699b      	ldr	r3, [r3, #24]
 800129a:	2b00      	cmp	r3, #0
 800129c:	d026      	beq.n	80012ec <HAL_RCC_OscConfig+0x608>
      {
        /* Enable the Internal High Speed oscillator (HSI48). */
        __HAL_RCC_HSI48_ENABLE();
 800129e:	4b33      	ldr	r3, [pc, #204]	; (800136c <HAL_RCC_OscConfig+0x688>)
 80012a0:	689a      	ldr	r2, [r3, #8]
 80012a2:	4b32      	ldr	r3, [pc, #200]	; (800136c <HAL_RCC_OscConfig+0x688>)
 80012a4:	2101      	movs	r1, #1
 80012a6:	430a      	orrs	r2, r1
 80012a8:	609a      	str	r2, [r3, #8]
 80012aa:	4b30      	ldr	r3, [pc, #192]	; (800136c <HAL_RCC_OscConfig+0x688>)
 80012ac:	6b5a      	ldr	r2, [r3, #52]	; 0x34
 80012ae:	4b2f      	ldr	r3, [pc, #188]	; (800136c <HAL_RCC_OscConfig+0x688>)
 80012b0:	2101      	movs	r1, #1
 80012b2:	430a      	orrs	r2, r1
 80012b4:	635a      	str	r2, [r3, #52]	; 0x34
 80012b6:	4b34      	ldr	r3, [pc, #208]	; (8001388 <HAL_RCC_OscConfig+0x6a4>)
 80012b8:	6a1a      	ldr	r2, [r3, #32]
 80012ba:	4b33      	ldr	r3, [pc, #204]	; (8001388 <HAL_RCC_OscConfig+0x6a4>)
 80012bc:	2180      	movs	r1, #128	; 0x80
 80012be:	0189      	lsls	r1, r1, #6
 80012c0:	430a      	orrs	r2, r1
 80012c2:	621a      	str	r2, [r3, #32]

        /* Get Start Tick */
        tickstart = HAL_GetTick();
 80012c4:	f7ff fa90 	bl	80007e8 <HAL_GetTick>
 80012c8:	0003      	movs	r3, r0
 80012ca:	617b      	str	r3, [r7, #20]

        /* Wait till HSI48 is ready */
        while(__HAL_RCC_GET_FLAG(RCC_FLAG_HSI48RDY) == 0U)
 80012cc:	e008      	b.n	80012e0 <HAL_RCC_OscConfig+0x5fc>
        {
          if((HAL_GetTick() - tickstart) > HSI48_TIMEOUT_VALUE)
 80012ce:	f7ff fa8b 	bl	80007e8 <HAL_GetTick>
 80012d2:	0002      	movs	r2, r0
 80012d4:	697b      	ldr	r3, [r7, #20]
 80012d6:	1ad3      	subs	r3, r2, r3
 80012d8:	2b02      	cmp	r3, #2
 80012da:	d901      	bls.n	80012e0 <HAL_RCC_OscConfig+0x5fc>
          {
            return HAL_TIMEOUT;
 80012dc:	2303      	movs	r3, #3
 80012de:	e0ca      	b.n	8001476 <HAL_RCC_OscConfig+0x792>
        while(__HAL_RCC_GET_FLAG(RCC_FLAG_HSI48RDY) == 0U)
 80012e0:	4b22      	ldr	r3, [pc, #136]	; (800136c <HAL_RCC_OscConfig+0x688>)
 80012e2:	689b      	ldr	r3, [r3, #8]
 80012e4:	2202      	movs	r2, #2
 80012e6:	4013      	ands	r3, r2
 80012e8:	d0f1      	beq.n	80012ce <HAL_RCC_OscConfig+0x5ea>
 80012ea:	e01e      	b.n	800132a <HAL_RCC_OscConfig+0x646>
        }
      }
      else
      {
        /* Disable the Internal High Speed oscillator (HSI48). */
        __HAL_RCC_HSI48_DISABLE();
 80012ec:	4b1f      	ldr	r3, [pc, #124]	; (800136c <HAL_RCC_OscConfig+0x688>)
 80012ee:	689a      	ldr	r2, [r3, #8]
 80012f0:	4b1e      	ldr	r3, [pc, #120]	; (800136c <HAL_RCC_OscConfig+0x688>)
 80012f2:	2101      	movs	r1, #1
 80012f4:	438a      	bics	r2, r1
 80012f6:	609a      	str	r2, [r3, #8]
 80012f8:	4b23      	ldr	r3, [pc, #140]	; (8001388 <HAL_RCC_OscConfig+0x6a4>)
 80012fa:	6a1a      	ldr	r2, [r3, #32]
 80012fc:	4b22      	ldr	r3, [pc, #136]	; (8001388 <HAL_RCC_OscConfig+0x6a4>)
 80012fe:	4923      	ldr	r1, [pc, #140]	; (800138c <HAL_RCC_OscConfig+0x6a8>)
 8001300:	400a      	ands	r2, r1
 8001302:	621a      	str	r2, [r3, #32]

        /* Get Start Tick */
        tickstart = HAL_GetTick();
 8001304:	f7ff fa70 	bl	80007e8 <HAL_GetTick>
 8001308:	0003      	movs	r3, r0
 800130a:	617b      	str	r3, [r7, #20]

        /* Wait till HSI48 is ready */
        while(__HAL_RCC_GET_FLAG(RCC_FLAG_HSI48RDY) != 0U)
 800130c:	e008      	b.n	8001320 <HAL_RCC_OscConfig+0x63c>
        {
          if((HAL_GetTick() - tickstart) > HSI48_TIMEOUT_VALUE)
 800130e:	f7ff fa6b 	bl	80007e8 <HAL_GetTick>
 8001312:	0002      	movs	r2, r0
 8001314:	697b      	ldr	r3, [r7, #20]
 8001316:	1ad3      	subs	r3, r2, r3
 8001318:	2b02      	cmp	r3, #2
 800131a:	d901      	bls.n	8001320 <HAL_RCC_OscConfig+0x63c>
          {
            return HAL_TIMEOUT;
 800131c:	2303      	movs	r3, #3
 800131e:	e0aa      	b.n	8001476 <HAL_RCC_OscConfig+0x792>
        while(__HAL_RCC_GET_FLAG(RCC_FLAG_HSI48RDY) != 0U)
 8001320:	4b12      	ldr	r3, [pc, #72]	; (800136c <HAL_RCC_OscConfig+0x688>)
 8001322:	689b      	ldr	r3, [r3, #8]
 8001324:	2202      	movs	r2, #2
 8001326:	4013      	ands	r3, r2
 8001328:	d1f1      	bne.n	800130e <HAL_RCC_OscConfig+0x62a>
#endif /* RCC_HSI48_SUPPORT */

  /*-------------------------------- PLL Configuration -----------------------*/
  /* Check the parameters */
  assert_param(IS_RCC_PLL(RCC_OscInitStruct->PLL.PLLState));
  if ((RCC_OscInitStruct->PLL.PLLState) != RCC_PLL_NONE)
 800132a:	687b      	ldr	r3, [r7, #4]
 800132c:	6a9b      	ldr	r3, [r3, #40]	; 0x28
 800132e:	2b00      	cmp	r3, #0
 8001330:	d100      	bne.n	8001334 <HAL_RCC_OscConfig+0x650>
 8001332:	e09f      	b.n	8001474 <HAL_RCC_OscConfig+0x790>
  {
    /* Check if the PLL is used as system clock or not */
    if(sysclk_source != RCC_SYSCLKSOURCE_STATUS_PLLCLK)
 8001334:	69fb      	ldr	r3, [r7, #28]
 8001336:	2b0c      	cmp	r3, #12
 8001338:	d100      	bne.n	800133c <HAL_RCC_OscConfig+0x658>
 800133a:	e078      	b.n	800142e <HAL_RCC_OscConfig+0x74a>
    {
      if((RCC_OscInitStruct->PLL.PLLState) == RCC_PLL_ON)
 800133c:	687b      	ldr	r3, [r7, #4]
 800133e:	6a9b      	ldr	r3, [r3, #40]	; 0x28
 8001340:	2b02      	cmp	r3, #2
 8001342:	d159      	bne.n	80013f8 <HAL_RCC_OscConfig+0x714>
        assert_param(IS_RCC_PLLSOURCE(RCC_OscInitStruct->PLL.PLLSource));
        assert_param(IS_RCC_PLL_MUL(RCC_OscInitStruct->PLL.PLLMUL));
        assert_param(IS_RCC_PLL_DIV(RCC_OscInitStruct->PLL.PLLDIV));

        /* Disable the main PLL. */
        __HAL_RCC_PLL_DISABLE();
 8001344:	4b09      	ldr	r3, [pc, #36]	; (800136c <HAL_RCC_OscConfig+0x688>)
 8001346:	681a      	ldr	r2, [r3, #0]
 8001348:	4b08      	ldr	r3, [pc, #32]	; (800136c <HAL_RCC_OscConfig+0x688>)
 800134a:	4911      	ldr	r1, [pc, #68]	; (8001390 <HAL_RCC_OscConfig+0x6ac>)
 800134c:	400a      	ands	r2, r1
 800134e:	601a      	str	r2, [r3, #0]

        /* Get Start Tick */
        tickstart = HAL_GetTick();
 8001350:	f7ff fa4a 	bl	80007e8 <HAL_GetTick>
 8001354:	0003      	movs	r3, r0
 8001356:	617b      	str	r3, [r7, #20]

        /* Wait till PLL is ready */
        while(__HAL_RCC_GET_FLAG(RCC_FLAG_PLLRDY)  != 0U)
 8001358:	e01c      	b.n	8001394 <HAL_RCC_OscConfig+0x6b0>
        {
          if((HAL_GetTick() - tickstart ) > PLL_TIMEOUT_VALUE)
 800135a:	f7ff fa45 	bl	80007e8 <HAL_GetTick>
 800135e:	0002      	movs	r2, r0
 8001360:	697b      	ldr	r3, [r7, #20]
 8001362:	1ad3      	subs	r3, r2, r3
 8001364:	2b02      	cmp	r3, #2
 8001366:	d915      	bls.n	8001394 <HAL_RCC_OscConfig+0x6b0>
          {
            return HAL_TIMEOUT;
 8001368:	2303      	movs	r3, #3
 800136a:	e084      	b.n	8001476 <HAL_RCC_OscConfig+0x792>
 800136c:	40021000 	.word	0x40021000
 8001370:	ffff1fff 	.word	0xffff1fff
 8001374:	fffffeff 	.word	0xfffffeff
 8001378:	40007000 	.word	0x40007000
 800137c:	fffffbff 	.word	0xfffffbff
 8001380:	00001388 	.word	0x00001388
 8001384:	efffffff 	.word	0xefffffff
 8001388:	40010000 	.word	0x40010000
 800138c:	ffffdfff 	.word	0xffffdfff
 8001390:	feffffff 	.word	0xfeffffff
        while(__HAL_RCC_GET_FLAG(RCC_FLAG_PLLRDY)  != 0U)
 8001394:	4b3a      	ldr	r3, [pc, #232]	; (8001480 <HAL_RCC_OscConfig+0x79c>)
 8001396:	681a      	ldr	r2, [r3, #0]
 8001398:	2380      	movs	r3, #128	; 0x80
 800139a:	049b      	lsls	r3, r3, #18
 800139c:	4013      	ands	r3, r2
 800139e:	d1dc      	bne.n	800135a <HAL_RCC_OscConfig+0x676>
          }
        }

        /* Configure the main PLL clock source, multiplication and division factors. */
        __HAL_RCC_PLL_CONFIG(RCC_OscInitStruct->PLL.PLLSource,
 80013a0:	4b37      	ldr	r3, [pc, #220]	; (8001480 <HAL_RCC_OscConfig+0x79c>)
 80013a2:	68db      	ldr	r3, [r3, #12]
 80013a4:	4a37      	ldr	r2, [pc, #220]	; (8001484 <HAL_RCC_OscConfig+0x7a0>)
 80013a6:	4013      	ands	r3, r2
 80013a8:	0019      	movs	r1, r3
 80013aa:	687b      	ldr	r3, [r7, #4]
 80013ac:	6ada      	ldr	r2, [r3, #44]	; 0x2c
 80013ae:	687b      	ldr	r3, [r7, #4]
 80013b0:	6b1b      	ldr	r3, [r3, #48]	; 0x30
 80013b2:	431a      	orrs	r2, r3
 80013b4:	687b      	ldr	r3, [r7, #4]
 80013b6:	6b5b      	ldr	r3, [r3, #52]	; 0x34
 80013b8:	431a      	orrs	r2, r3
 80013ba:	4b31      	ldr	r3, [pc, #196]	; (8001480 <HAL_RCC_OscConfig+0x79c>)
 80013bc:	430a      	orrs	r2, r1
 80013be:	60da      	str	r2, [r3, #12]
                             RCC_OscInitStruct->PLL.PLLMUL,
                             RCC_OscInitStruct->PLL.PLLDIV);
        /* Enable the main PLL. */
        __HAL_RCC_PLL_ENABLE();
 80013c0:	4b2f      	ldr	r3, [pc, #188]	; (8001480 <HAL_RCC_OscConfig+0x79c>)
 80013c2:	681a      	ldr	r2, [r3, #0]
 80013c4:	4b2e      	ldr	r3, [pc, #184]	; (8001480 <HAL_RCC_OscConfig+0x79c>)
 80013c6:	2180      	movs	r1, #128	; 0x80
 80013c8:	0449      	lsls	r1, r1, #17
 80013ca:	430a      	orrs	r2, r1
 80013cc:	601a      	str	r2, [r3, #0]

        /* Get Start Tick */
        tickstart = HAL_GetTick();
 80013ce:	f7ff fa0b 	bl	80007e8 <HAL_GetTick>
 80013d2:	0003      	movs	r3, r0
 80013d4:	617b      	str	r3, [r7, #20]

        /* Wait till PLL is ready */
        while(__HAL_RCC_GET_FLAG(RCC_FLAG_PLLRDY)  == 0U)
 80013d6:	e008      	b.n	80013ea <HAL_RCC_OscConfig+0x706>
        {
          if((HAL_GetTick() - tickstart ) > PLL_TIMEOUT_VALUE)
 80013d8:	f7ff fa06 	bl	80007e8 <HAL_GetTick>
 80013dc:	0002      	movs	r2, r0
 80013de:	697b      	ldr	r3, [r7, #20]
 80013e0:	1ad3      	subs	r3, r2, r3
 80013e2:	2b02      	cmp	r3, #2
 80013e4:	d901      	bls.n	80013ea <HAL_RCC_OscConfig+0x706>
          {
            return HAL_TIMEOUT;
 80013e6:	2303      	movs	r3, #3
 80013e8:	e045      	b.n	8001476 <HAL_RCC_OscConfig+0x792>
        while(__HAL_RCC_GET_FLAG(RCC_FLAG_PLLRDY)  == 0U)
 80013ea:	4b25      	ldr	r3, [pc, #148]	; (8001480 <HAL_RCC_OscConfig+0x79c>)
 80013ec:	681a      	ldr	r2, [r3, #0]
 80013ee:	2380      	movs	r3, #128	; 0x80
 80013f0:	049b      	lsls	r3, r3, #18
 80013f2:	4013      	ands	r3, r2
 80013f4:	d0f0      	beq.n	80013d8 <HAL_RCC_OscConfig+0x6f4>
 80013f6:	e03d      	b.n	8001474 <HAL_RCC_OscConfig+0x790>
        }
      }
      else
      {
        /* Disable the main PLL. */
        __HAL_RCC_PLL_DISABLE();
 80013f8:	4b21      	ldr	r3, [pc, #132]	; (8001480 <HAL_RCC_OscConfig+0x79c>)
 80013fa:	681a      	ldr	r2, [r3, #0]
 80013fc:	4b20      	ldr	r3, [pc, #128]	; (8001480 <HAL_RCC_OscConfig+0x79c>)
 80013fe:	4922      	ldr	r1, [pc, #136]	; (8001488 <HAL_RCC_OscConfig+0x7a4>)
 8001400:	400a      	ands	r2, r1
 8001402:	601a      	str	r2, [r3, #0]

        /* Get Start Tick */
        tickstart = HAL_GetTick();
 8001404:	f7ff f9f0 	bl	80007e8 <HAL_GetTick>
 8001408:	0003      	movs	r3, r0
 800140a:	617b      	str	r3, [r7, #20]

        /* Wait till PLL is disabled */
        while(__HAL_RCC_GET_FLAG(RCC_FLAG_PLLRDY)  != 0U)
 800140c:	e008      	b.n	8001420 <HAL_RCC_OscConfig+0x73c>
        {
          if((HAL_GetTick() - tickstart ) > PLL_TIMEOUT_VALUE)
 800140e:	f7ff f9eb 	bl	80007e8 <HAL_GetTick>
 8001412:	0002      	movs	r2, r0
 8001414:	697b      	ldr	r3, [r7, #20]
 8001416:	1ad3      	subs	r3, r2, r3
 8001418:	2b02      	cmp	r3, #2
 800141a:	d901      	bls.n	8001420 <HAL_RCC_OscConfig+0x73c>
          {
            return HAL_TIMEOUT;
 800141c:	2303      	movs	r3, #3
 800141e:	e02a      	b.n	8001476 <HAL_RCC_OscConfig+0x792>
        while(__HAL_RCC_GET_FLAG(RCC_FLAG_PLLRDY)  != 0U)
 8001420:	4b17      	ldr	r3, [pc, #92]	; (8001480 <HAL_RCC_OscConfig+0x79c>)
 8001422:	681a      	ldr	r2, [r3, #0]
 8001424:	2380      	movs	r3, #128	; 0x80
 8001426:	049b      	lsls	r3, r3, #18
 8001428:	4013      	ands	r3, r2
 800142a:	d1f0      	bne.n	800140e <HAL_RCC_OscConfig+0x72a>
 800142c:	e022      	b.n	8001474 <HAL_RCC_OscConfig+0x790>
      }
    }
    else
    {
      /* Check if there is a request to disable the PLL used as System clock source */
      if((RCC_OscInitStruct->PLL.PLLState) == RCC_PLL_OFF)
 800142e:	687b      	ldr	r3, [r7, #4]
 8001430:	6a9b      	ldr	r3, [r3, #40]	; 0x28
 8001432:	2b01      	cmp	r3, #1
 8001434:	d101      	bne.n	800143a <HAL_RCC_OscConfig+0x756>
      {
        return HAL_ERROR;
 8001436:	2301      	movs	r3, #1
 8001438:	e01d      	b.n	8001476 <HAL_RCC_OscConfig+0x792>
      }
      else
      {
        /* Do not return HAL_ERROR if request repeats the current configuration */
        pll_config = RCC->CFGR;
 800143a:	4b11      	ldr	r3, [pc, #68]	; (8001480 <HAL_RCC_OscConfig+0x79c>)
 800143c:	68db      	ldr	r3, [r3, #12]
 800143e:	61bb      	str	r3, [r7, #24]
        if((READ_BIT(pll_config, RCC_CFGR_PLLSRC) != RCC_OscInitStruct->PLL.PLLSource) ||
 8001440:	69ba      	ldr	r2, [r7, #24]
 8001442:	2380      	movs	r3, #128	; 0x80
 8001444:	025b      	lsls	r3, r3, #9
 8001446:	401a      	ands	r2, r3
 8001448:	687b      	ldr	r3, [r7, #4]
 800144a:	6adb      	ldr	r3, [r3, #44]	; 0x2c
 800144c:	429a      	cmp	r2, r3
 800144e:	d10f      	bne.n	8001470 <HAL_RCC_OscConfig+0x78c>
           (READ_BIT(pll_config, RCC_CFGR_PLLMUL) != RCC_OscInitStruct->PLL.PLLMUL) ||
 8001450:	69ba      	ldr	r2, [r7, #24]
 8001452:	23f0      	movs	r3, #240	; 0xf0
 8001454:	039b      	lsls	r3, r3, #14
 8001456:	401a      	ands	r2, r3
 8001458:	687b      	ldr	r3, [r7, #4]
 800145a:	6b1b      	ldr	r3, [r3, #48]	; 0x30
        if((READ_BIT(pll_config, RCC_CFGR_PLLSRC) != RCC_OscInitStruct->PLL.PLLSource) ||
 800145c:	429a      	cmp	r2, r3
 800145e:	d107      	bne.n	8001470 <HAL_RCC_OscConfig+0x78c>
           (READ_BIT(pll_config, RCC_CFGR_PLLDIV) != RCC_OscInitStruct->PLL.PLLDIV))
 8001460:	69ba      	ldr	r2, [r7, #24]
 8001462:	23c0      	movs	r3, #192	; 0xc0
 8001464:	041b      	lsls	r3, r3, #16
 8001466:	401a      	ands	r2, r3
 8001468:	687b      	ldr	r3, [r7, #4]
 800146a:	6b5b      	ldr	r3, [r3, #52]	; 0x34
           (READ_BIT(pll_config, RCC_CFGR_PLLMUL) != RCC_OscInitStruct->PLL.PLLMUL) ||
 800146c:	429a      	cmp	r2, r3
 800146e:	d001      	beq.n	8001474 <HAL_RCC_OscConfig+0x790>
        {
          return HAL_ERROR;
 8001470:	2301      	movs	r3, #1
 8001472:	e000      	b.n	8001476 <HAL_RCC_OscConfig+0x792>
        }
      }
    }
  }
  return HAL_OK;
 8001474:	2300      	movs	r3, #0
}
 8001476:	0018      	movs	r0, r3
 8001478:	46bd      	mov	sp, r7
 800147a:	b00a      	add	sp, #40	; 0x28
 800147c:	bdb0      	pop	{r4, r5, r7, pc}
 800147e:	46c0      	nop			; (mov r8, r8)
 8001480:	40021000 	.word	0x40021000
 8001484:	ff02ffff 	.word	0xff02ffff
 8001488:	feffffff 	.word	0xfeffffff

0800148c <HAL_RCC_ClockConfig>:
  *         HPRE[3:0] bits to ensure that HCLK not exceed the maximum allowed frequency
  *         (for more details refer to section above "Initialization/de-initialization functions")
  * @retval HAL status
  */
HAL_StatusTypeDef HAL_RCC_ClockConfig(RCC_ClkInitTypeDef  *RCC_ClkInitStruct, uint32_t FLatency)
{
 800148c:	b5b0      	push	{r4, r5, r7, lr}
 800148e:	b084      	sub	sp, #16
 8001490:	af00      	add	r7, sp, #0
 8001492:	6078      	str	r0, [r7, #4]
 8001494:	6039      	str	r1, [r7, #0]
  uint32_t tickstart;
  HAL_StatusTypeDef status;

  /* Check Null pointer */
  if(RCC_ClkInitStruct == NULL)
 8001496:	687b      	ldr	r3, [r7, #4]
 8001498:	2b00      	cmp	r3, #0
 800149a:	d101      	bne.n	80014a0 <HAL_RCC_ClockConfig+0x14>
  {
    return HAL_ERROR;
 800149c:	2301      	movs	r3, #1
 800149e:	e128      	b.n	80016f2 <HAL_RCC_ClockConfig+0x266>
  /* To correctly read data from FLASH memory, the number of wait states (LATENCY)
  must be correctly programmed according to the frequency of the CPU clock
  (HCLK) and the supply voltage of the device. */

  /* Increasing the number of wait states because of higher CPU frequency */
  if(FLatency > __HAL_FLASH_GET_LATENCY())
 80014a0:	4b96      	ldr	r3, [pc, #600]	; (80016fc <HAL_RCC_ClockConfig+0x270>)
 80014a2:	681b      	ldr	r3, [r3, #0]
 80014a4:	2201      	movs	r2, #1
 80014a6:	4013      	ands	r3, r2
 80014a8:	683a      	ldr	r2, [r7, #0]
 80014aa:	429a      	cmp	r2, r3
 80014ac:	d91e      	bls.n	80014ec <HAL_RCC_ClockConfig+0x60>
  {
    /* Program the new number of wait states to the LATENCY bits in the FLASH_ACR register */
    __HAL_FLASH_SET_LATENCY(FLatency);
 80014ae:	4b93      	ldr	r3, [pc, #588]	; (80016fc <HAL_RCC_ClockConfig+0x270>)
 80014b0:	681b      	ldr	r3, [r3, #0]
 80014b2:	2201      	movs	r2, #1
 80014b4:	4393      	bics	r3, r2
 80014b6:	0019      	movs	r1, r3
 80014b8:	4b90      	ldr	r3, [pc, #576]	; (80016fc <HAL_RCC_ClockConfig+0x270>)
 80014ba:	683a      	ldr	r2, [r7, #0]
 80014bc:	430a      	orrs	r2, r1
 80014be:	601a      	str	r2, [r3, #0]

    /* Check that the new number of wait states is taken into account to access the Flash
    memory by polling the FLASH_ACR register */
    tickstart = HAL_GetTick();
 80014c0:	f7ff f992 	bl	80007e8 <HAL_GetTick>
 80014c4:	0003      	movs	r3, r0
 80014c6:	60fb      	str	r3, [r7, #12]

    while (__HAL_FLASH_GET_LATENCY() != FLatency)
 80014c8:	e009      	b.n	80014de <HAL_RCC_ClockConfig+0x52>
    {
      if ((HAL_GetTick() - tickstart) > CLOCKSWITCH_TIMEOUT_VALUE)
 80014ca:	f7ff f98d 	bl	80007e8 <HAL_GetTick>
 80014ce:	0002      	movs	r2, r0
 80014d0:	68fb      	ldr	r3, [r7, #12]
 80014d2:	1ad3      	subs	r3, r2, r3
 80014d4:	4a8a      	ldr	r2, [pc, #552]	; (8001700 <HAL_RCC_ClockConfig+0x274>)
 80014d6:	4293      	cmp	r3, r2
 80014d8:	d901      	bls.n	80014de <HAL_RCC_ClockConfig+0x52>
      {
        return HAL_TIMEOUT;
 80014da:	2303      	movs	r3, #3
 80014dc:	e109      	b.n	80016f2 <HAL_RCC_ClockConfig+0x266>
    while (__HAL_FLASH_GET_LATENCY() != FLatency)
 80014de:	4b87      	ldr	r3, [pc, #540]	; (80016fc <HAL_RCC_ClockConfig+0x270>)
 80014e0:	681b      	ldr	r3, [r3, #0]
 80014e2:	2201      	movs	r2, #1
 80014e4:	4013      	ands	r3, r2
 80014e6:	683a      	ldr	r2, [r7, #0]
 80014e8:	429a      	cmp	r2, r3
 80014ea:	d1ee      	bne.n	80014ca <HAL_RCC_ClockConfig+0x3e>
      }
    }
  }

  /*-------------------------- HCLK Configuration --------------------------*/
  if(((RCC_ClkInitStruct->ClockType) & RCC_CLOCKTYPE_HCLK) == RCC_CLOCKTYPE_HCLK)
 80014ec:	687b      	ldr	r3, [r7, #4]
 80014ee:	681b      	ldr	r3, [r3, #0]
 80014f0:	2202      	movs	r2, #2
 80014f2:	4013      	ands	r3, r2
 80014f4:	d009      	beq.n	800150a <HAL_RCC_ClockConfig+0x7e>
  {
    assert_param(IS_RCC_HCLK(RCC_ClkInitStruct->AHBCLKDivider));
    MODIFY_REG(RCC->CFGR, RCC_CFGR_HPRE, RCC_ClkInitStruct->AHBCLKDivider);
 80014f6:	4b83      	ldr	r3, [pc, #524]	; (8001704 <HAL_RCC_ClockConfig+0x278>)
 80014f8:	68db      	ldr	r3, [r3, #12]
 80014fa:	22f0      	movs	r2, #240	; 0xf0
 80014fc:	4393      	bics	r3, r2
 80014fe:	0019      	movs	r1, r3
 8001500:	687b      	ldr	r3, [r7, #4]
 8001502:	689a      	ldr	r2, [r3, #8]
 8001504:	4b7f      	ldr	r3, [pc, #508]	; (8001704 <HAL_RCC_ClockConfig+0x278>)
 8001506:	430a      	orrs	r2, r1
 8001508:	60da      	str	r2, [r3, #12]
  }

  /*------------------------- SYSCLK Configuration ---------------------------*/
  if(((RCC_ClkInitStruct->ClockType) & RCC_CLOCKTYPE_SYSCLK) == RCC_CLOCKTYPE_SYSCLK)
 800150a:	687b      	ldr	r3, [r7, #4]
 800150c:	681b      	ldr	r3, [r3, #0]
 800150e:	2201      	movs	r2, #1
 8001510:	4013      	ands	r3, r2
 8001512:	d100      	bne.n	8001516 <HAL_RCC_ClockConfig+0x8a>
 8001514:	e089      	b.n	800162a <HAL_RCC_ClockConfig+0x19e>
  {
    assert_param(IS_RCC_SYSCLKSOURCE(RCC_ClkInitStruct->SYSCLKSource));

    /* HSE is selected as System Clock Source */
    if(RCC_ClkInitStruct->SYSCLKSource == RCC_SYSCLKSOURCE_HSE)
 8001516:	687b      	ldr	r3, [r7, #4]
 8001518:	685b      	ldr	r3, [r3, #4]
 800151a:	2b02      	cmp	r3, #2
 800151c:	d107      	bne.n	800152e <HAL_RCC_ClockConfig+0xa2>
    {
      /* Check the HSE ready flag */
      if(__HAL_RCC_GET_FLAG(RCC_FLAG_HSERDY) == 0U)
 800151e:	4b79      	ldr	r3, [pc, #484]	; (8001704 <HAL_RCC_ClockConfig+0x278>)
 8001520:	681a      	ldr	r2, [r3, #0]
 8001522:	2380      	movs	r3, #128	; 0x80
 8001524:	029b      	lsls	r3, r3, #10
 8001526:	4013      	ands	r3, r2
 8001528:	d120      	bne.n	800156c <HAL_RCC_ClockConfig+0xe0>
      {
        return HAL_ERROR;
 800152a:	2301      	movs	r3, #1
 800152c:	e0e1      	b.n	80016f2 <HAL_RCC_ClockConfig+0x266>
      }
    }
    /* PLL is selected as System Clock Source */
    else if(RCC_ClkInitStruct->SYSCLKSource == RCC_SYSCLKSOURCE_PLLCLK)
 800152e:	687b      	ldr	r3, [r7, #4]
 8001530:	685b      	ldr	r3, [r3, #4]
 8001532:	2b03      	cmp	r3, #3
 8001534:	d107      	bne.n	8001546 <HAL_RCC_ClockConfig+0xba>
    {
      /* Check the PLL ready flag */
      if(__HAL_RCC_GET_FLAG(RCC_FLAG_PLLRDY) == 0U)
 8001536:	4b73      	ldr	r3, [pc, #460]	; (8001704 <HAL_RCC_ClockConfig+0x278>)
 8001538:	681a      	ldr	r2, [r3, #0]
 800153a:	2380      	movs	r3, #128	; 0x80
 800153c:	049b      	lsls	r3, r3, #18
 800153e:	4013      	ands	r3, r2
 8001540:	d114      	bne.n	800156c <HAL_RCC_ClockConfig+0xe0>
      {
        return HAL_ERROR;
 8001542:	2301      	movs	r3, #1
 8001544:	e0d5      	b.n	80016f2 <HAL_RCC_ClockConfig+0x266>
      }
    }
    /* HSI is selected as System Clock Source */
    else if(RCC_ClkInitStruct->SYSCLKSource == RCC_SYSCLKSOURCE_HSI)
 8001546:	687b      	ldr	r3, [r7, #4]
 8001548:	685b      	ldr	r3, [r3, #4]
 800154a:	2b01      	cmp	r3, #1
 800154c:	d106      	bne.n	800155c <HAL_RCC_ClockConfig+0xd0>
    {
      /* Check the HSI ready flag */
      if(__HAL_RCC_GET_FLAG(RCC_FLAG_HSIRDY) == 0U)
 800154e:	4b6d      	ldr	r3, [pc, #436]	; (8001704 <HAL_RCC_ClockConfig+0x278>)
 8001550:	681b      	ldr	r3, [r3, #0]
 8001552:	2204      	movs	r2, #4
 8001554:	4013      	ands	r3, r2
 8001556:	d109      	bne.n	800156c <HAL_RCC_ClockConfig+0xe0>
      {
        return HAL_ERROR;
 8001558:	2301      	movs	r3, #1
 800155a:	e0ca      	b.n	80016f2 <HAL_RCC_ClockConfig+0x266>
    }
    /* MSI is selected as System Clock Source */
    else
    {
      /* Check the MSI ready flag */
      if(__HAL_RCC_GET_FLAG(RCC_FLAG_MSIRDY) == 0U)
 800155c:	4b69      	ldr	r3, [pc, #420]	; (8001704 <HAL_RCC_ClockConfig+0x278>)
 800155e:	681a      	ldr	r2, [r3, #0]
 8001560:	2380      	movs	r3, #128	; 0x80
 8001562:	009b      	lsls	r3, r3, #2
 8001564:	4013      	ands	r3, r2
 8001566:	d101      	bne.n	800156c <HAL_RCC_ClockConfig+0xe0>
      {
        return HAL_ERROR;
 8001568:	2301      	movs	r3, #1
 800156a:	e0c2      	b.n	80016f2 <HAL_RCC_ClockConfig+0x266>
      }
    }
    __HAL_RCC_SYSCLK_CONFIG(RCC_ClkInitStruct->SYSCLKSource);
 800156c:	4b65      	ldr	r3, [pc, #404]	; (8001704 <HAL_RCC_ClockConfig+0x278>)
 800156e:	68db      	ldr	r3, [r3, #12]
 8001570:	2203      	movs	r2, #3
 8001572:	4393      	bics	r3, r2
 8001574:	0019      	movs	r1, r3
 8001576:	687b      	ldr	r3, [r7, #4]
 8001578:	685a      	ldr	r2, [r3, #4]
 800157a:	4b62      	ldr	r3, [pc, #392]	; (8001704 <HAL_RCC_ClockConfig+0x278>)
 800157c:	430a      	orrs	r2, r1
 800157e:	60da      	str	r2, [r3, #12]

    /* Get Start Tick */
    tickstart = HAL_GetTick();
 8001580:	f7ff f932 	bl	80007e8 <HAL_GetTick>
 8001584:	0003      	movs	r3, r0
 8001586:	60fb      	str	r3, [r7, #12]

    if(RCC_ClkInitStruct->SYSCLKSource == RCC_SYSCLKSOURCE_HSE)
 8001588:	687b      	ldr	r3, [r7, #4]
 800158a:	685b      	ldr	r3, [r3, #4]
 800158c:	2b02      	cmp	r3, #2
 800158e:	d111      	bne.n	80015b4 <HAL_RCC_ClockConfig+0x128>
    {
      while (__HAL_RCC_GET_SYSCLK_SOURCE() != RCC_SYSCLKSOURCE_STATUS_HSE)
 8001590:	e009      	b.n	80015a6 <HAL_RCC_ClockConfig+0x11a>
      {
        if((HAL_GetTick() - tickstart ) > CLOCKSWITCH_TIMEOUT_VALUE)
 8001592:	f7ff f929 	bl	80007e8 <HAL_GetTick>
 8001596:	0002      	movs	r2, r0
 8001598:	68fb      	ldr	r3, [r7, #12]
 800159a:	1ad3      	subs	r3, r2, r3
 800159c:	4a58      	ldr	r2, [pc, #352]	; (8001700 <HAL_RCC_ClockConfig+0x274>)
 800159e:	4293      	cmp	r3, r2
 80015a0:	d901      	bls.n	80015a6 <HAL_RCC_ClockConfig+0x11a>
        {
          return HAL_TIMEOUT;
 80015a2:	2303      	movs	r3, #3
 80015a4:	e0a5      	b.n	80016f2 <HAL_RCC_ClockConfig+0x266>
      while (__HAL_RCC_GET_SYSCLK_SOURCE() != RCC_SYSCLKSOURCE_STATUS_HSE)
 80015a6:	4b57      	ldr	r3, [pc, #348]	; (8001704 <HAL_RCC_ClockConfig+0x278>)
 80015a8:	68db      	ldr	r3, [r3, #12]
 80015aa:	220c      	movs	r2, #12
 80015ac:	4013      	ands	r3, r2
 80015ae:	2b08      	cmp	r3, #8
 80015b0:	d1ef      	bne.n	8001592 <HAL_RCC_ClockConfig+0x106>
 80015b2:	e03a      	b.n	800162a <HAL_RCC_ClockConfig+0x19e>
        }
      }
    }
    else if(RCC_ClkInitStruct->SYSCLKSource == RCC_SYSCLKSOURCE_PLLCLK)
 80015b4:	687b      	ldr	r3, [r7, #4]
 80015b6:	685b      	ldr	r3, [r3, #4]
 80015b8:	2b03      	cmp	r3, #3
 80015ba:	d111      	bne.n	80015e0 <HAL_RCC_ClockConfig+0x154>
    {
      while (__HAL_RCC_GET_SYSCLK_SOURCE() != RCC_SYSCLKSOURCE_STATUS_PLLCLK)
 80015bc:	e009      	b.n	80015d2 <HAL_RCC_ClockConfig+0x146>
      {
        if((HAL_GetTick() - tickstart ) > CLOCKSWITCH_TIMEOUT_VALUE)
 80015be:	f7ff f913 	bl	80007e8 <HAL_GetTick>
 80015c2:	0002      	movs	r2, r0
 80015c4:	68fb      	ldr	r3, [r7, #12]
 80015c6:	1ad3      	subs	r3, r2, r3
 80015c8:	4a4d      	ldr	r2, [pc, #308]	; (8001700 <HAL_RCC_ClockConfig+0x274>)
 80015ca:	4293      	cmp	r3, r2
 80015cc:	d901      	bls.n	80015d2 <HAL_RCC_ClockConfig+0x146>
        {
          return HAL_TIMEOUT;
 80015ce:	2303      	movs	r3, #3
 80015d0:	e08f      	b.n	80016f2 <HAL_RCC_ClockConfig+0x266>
      while (__HAL_RCC_GET_SYSCLK_SOURCE() != RCC_SYSCLKSOURCE_STATUS_PLLCLK)
 80015d2:	4b4c      	ldr	r3, [pc, #304]	; (8001704 <HAL_RCC_ClockConfig+0x278>)
 80015d4:	68db      	ldr	r3, [r3, #12]
 80015d6:	220c      	movs	r2, #12
 80015d8:	4013      	ands	r3, r2
 80015da:	2b0c      	cmp	r3, #12
 80015dc:	d1ef      	bne.n	80015be <HAL_RCC_ClockConfig+0x132>
 80015de:	e024      	b.n	800162a <HAL_RCC_ClockConfig+0x19e>
        }
      }
    }
    else if(RCC_ClkInitStruct->SYSCLKSource == RCC_SYSCLKSOURCE_HSI)
 80015e0:	687b      	ldr	r3, [r7, #4]
 80015e2:	685b      	ldr	r3, [r3, #4]
 80015e4:	2b01      	cmp	r3, #1
 80015e6:	d11b      	bne.n	8001620 <HAL_RCC_ClockConfig+0x194>
    {
      while (__HAL_RCC_GET_SYSCLK_SOURCE() != RCC_SYSCLKSOURCE_STATUS_HSI)
 80015e8:	e009      	b.n	80015fe <HAL_RCC_ClockConfig+0x172>
      {
        if((HAL_GetTick() - tickstart ) > CLOCKSWITCH_TIMEOUT_VALUE)
 80015ea:	f7ff f8fd 	bl	80007e8 <HAL_GetTick>
 80015ee:	0002      	movs	r2, r0
 80015f0:	68fb      	ldr	r3, [r7, #12]
 80015f2:	1ad3      	subs	r3, r2, r3
 80015f4:	4a42      	ldr	r2, [pc, #264]	; (8001700 <HAL_RCC_ClockConfig+0x274>)
 80015f6:	4293      	cmp	r3, r2
 80015f8:	d901      	bls.n	80015fe <HAL_RCC_ClockConfig+0x172>
        {
          return HAL_TIMEOUT;
 80015fa:	2303      	movs	r3, #3
 80015fc:	e079      	b.n	80016f2 <HAL_RCC_ClockConfig+0x266>
      while (__HAL_RCC_GET_SYSCLK_SOURCE() != RCC_SYSCLKSOURCE_STATUS_HSI)
 80015fe:	4b41      	ldr	r3, [pc, #260]	; (8001704 <HAL_RCC_ClockConfig+0x278>)
 8001600:	68db      	ldr	r3, [r3, #12]
 8001602:	220c      	movs	r2, #12
 8001604:	4013      	ands	r3, r2
 8001606:	2b04      	cmp	r3, #4
 8001608:	d1ef      	bne.n	80015ea <HAL_RCC_ClockConfig+0x15e>
 800160a:	e00e      	b.n	800162a <HAL_RCC_ClockConfig+0x19e>
    }
    else
    {
      while(__HAL_RCC_GET_SYSCLK_SOURCE() != RCC_SYSCLKSOURCE_STATUS_MSI)
      {
        if((HAL_GetTick() - tickstart ) > CLOCKSWITCH_TIMEOUT_VALUE)
 800160c:	f7ff f8ec 	bl	80007e8 <HAL_GetTick>
 8001610:	0002      	movs	r2, r0
 8001612:	68fb      	ldr	r3, [r7, #12]
 8001614:	1ad3      	subs	r3, r2, r3
 8001616:	4a3a      	ldr	r2, [pc, #232]	; (8001700 <HAL_RCC_ClockConfig+0x274>)
 8001618:	4293      	cmp	r3, r2
 800161a:	d901      	bls.n	8001620 <HAL_RCC_ClockConfig+0x194>
        {
          return HAL_TIMEOUT;
 800161c:	2303      	movs	r3, #3
 800161e:	e068      	b.n	80016f2 <HAL_RCC_ClockConfig+0x266>
      while(__HAL_RCC_GET_SYSCLK_SOURCE() != RCC_SYSCLKSOURCE_STATUS_MSI)
 8001620:	4b38      	ldr	r3, [pc, #224]	; (8001704 <HAL_RCC_ClockConfig+0x278>)
 8001622:	68db      	ldr	r3, [r3, #12]
 8001624:	220c      	movs	r2, #12
 8001626:	4013      	ands	r3, r2
 8001628:	d1f0      	bne.n	800160c <HAL_RCC_ClockConfig+0x180>
        }
      }
    }
  }
  /* Decreasing the number of wait states because of lower CPU frequency */
  if(FLatency < __HAL_FLASH_GET_LATENCY())
 800162a:	4b34      	ldr	r3, [pc, #208]	; (80016fc <HAL_RCC_ClockConfig+0x270>)
 800162c:	681b      	ldr	r3, [r3, #0]
 800162e:	2201      	movs	r2, #1
 8001630:	4013      	ands	r3, r2
 8001632:	683a      	ldr	r2, [r7, #0]
 8001634:	429a      	cmp	r2, r3
 8001636:	d21e      	bcs.n	8001676 <HAL_RCC_ClockConfig+0x1ea>
  {
    /* Program the new number of wait states to the LATENCY bits in the FLASH_ACR register */
    __HAL_FLASH_SET_LATENCY(FLatency);
 8001638:	4b30      	ldr	r3, [pc, #192]	; (80016fc <HAL_RCC_ClockConfig+0x270>)
 800163a:	681b      	ldr	r3, [r3, #0]
 800163c:	2201      	movs	r2, #1
 800163e:	4393      	bics	r3, r2
 8001640:	0019      	movs	r1, r3
 8001642:	4b2e      	ldr	r3, [pc, #184]	; (80016fc <HAL_RCC_ClockConfig+0x270>)
 8001644:	683a      	ldr	r2, [r7, #0]
 8001646:	430a      	orrs	r2, r1
 8001648:	601a      	str	r2, [r3, #0]

    /* Check that the new number of wait states is taken into account to access the Flash
    memory by polling the FLASH_ACR register */
    tickstart = HAL_GetTick();
 800164a:	f7ff f8cd 	bl	80007e8 <HAL_GetTick>
 800164e:	0003      	movs	r3, r0
 8001650:	60fb      	str	r3, [r7, #12]

    while (__HAL_FLASH_GET_LATENCY() != FLatency)
 8001652:	e009      	b.n	8001668 <HAL_RCC_ClockConfig+0x1dc>
    {
      if ((HAL_GetTick() - tickstart) > CLOCKSWITCH_TIMEOUT_VALUE)
 8001654:	f7ff f8c8 	bl	80007e8 <HAL_GetTick>
 8001658:	0002      	movs	r2, r0
 800165a:	68fb      	ldr	r3, [r7, #12]
 800165c:	1ad3      	subs	r3, r2, r3
 800165e:	4a28      	ldr	r2, [pc, #160]	; (8001700 <HAL_RCC_ClockConfig+0x274>)
 8001660:	4293      	cmp	r3, r2
 8001662:	d901      	bls.n	8001668 <HAL_RCC_ClockConfig+0x1dc>
      {
        return HAL_TIMEOUT;
 8001664:	2303      	movs	r3, #3
 8001666:	e044      	b.n	80016f2 <HAL_RCC_ClockConfig+0x266>
    while (__HAL_FLASH_GET_LATENCY() != FLatency)
 8001668:	4b24      	ldr	r3, [pc, #144]	; (80016fc <HAL_RCC_ClockConfig+0x270>)
 800166a:	681b      	ldr	r3, [r3, #0]
 800166c:	2201      	movs	r2, #1
 800166e:	4013      	ands	r3, r2
 8001670:	683a      	ldr	r2, [r7, #0]
 8001672:	429a      	cmp	r2, r3
 8001674:	d1ee      	bne.n	8001654 <HAL_RCC_ClockConfig+0x1c8>
      }
    }
  }

  /*-------------------------- PCLK1 Configuration ---------------------------*/
  if(((RCC_ClkInitStruct->ClockType) & RCC_CLOCKTYPE_PCLK1) == RCC_CLOCKTYPE_PCLK1)
 8001676:	687b      	ldr	r3, [r7, #4]
 8001678:	681b      	ldr	r3, [r3, #0]
 800167a:	2204      	movs	r2, #4
 800167c:	4013      	ands	r3, r2
 800167e:	d009      	beq.n	8001694 <HAL_RCC_ClockConfig+0x208>
  {
    assert_param(IS_RCC_PCLK(RCC_ClkInitStruct->APB1CLKDivider));
    MODIFY_REG(RCC->CFGR, RCC_CFGR_PPRE1, RCC_ClkInitStruct->APB1CLKDivider);
 8001680:	4b20      	ldr	r3, [pc, #128]	; (8001704 <HAL_RCC_ClockConfig+0x278>)
 8001682:	68db      	ldr	r3, [r3, #12]
 8001684:	4a20      	ldr	r2, [pc, #128]	; (8001708 <HAL_RCC_ClockConfig+0x27c>)
 8001686:	4013      	ands	r3, r2
 8001688:	0019      	movs	r1, r3
 800168a:	687b      	ldr	r3, [r7, #4]
 800168c:	68da      	ldr	r2, [r3, #12]
 800168e:	4b1d      	ldr	r3, [pc, #116]	; (8001704 <HAL_RCC_ClockConfig+0x278>)
 8001690:	430a      	orrs	r2, r1
 8001692:	60da      	str	r2, [r3, #12]
  }

  /*-------------------------- PCLK2 Configuration ---------------------------*/
  if(((RCC_ClkInitStruct->ClockType) & RCC_CLOCKTYPE_PCLK2) == RCC_CLOCKTYPE_PCLK2)
 8001694:	687b      	ldr	r3, [r7, #4]
 8001696:	681b      	ldr	r3, [r3, #0]
 8001698:	2208      	movs	r2, #8
 800169a:	4013      	ands	r3, r2
 800169c:	d00a      	beq.n	80016b4 <HAL_RCC_ClockConfig+0x228>
  {
    assert_param(IS_RCC_PCLK(RCC_ClkInitStruct->APB2CLKDivider));
    MODIFY_REG(RCC->CFGR, RCC_CFGR_PPRE2, ((RCC_ClkInitStruct->APB2CLKDivider) << 3));
 800169e:	4b19      	ldr	r3, [pc, #100]	; (8001704 <HAL_RCC_ClockConfig+0x278>)
 80016a0:	68db      	ldr	r3, [r3, #12]
 80016a2:	4a1a      	ldr	r2, [pc, #104]	; (800170c <HAL_RCC_ClockConfig+0x280>)
 80016a4:	4013      	ands	r3, r2
 80016a6:	0019      	movs	r1, r3
 80016a8:	687b      	ldr	r3, [r7, #4]
 80016aa:	691b      	ldr	r3, [r3, #16]
 80016ac:	00da      	lsls	r2, r3, #3
 80016ae:	4b15      	ldr	r3, [pc, #84]	; (8001704 <HAL_RCC_ClockConfig+0x278>)
 80016b0:	430a      	orrs	r2, r1
 80016b2:	60da      	str	r2, [r3, #12]
  }

  /* Update the SystemCoreClock global variable */
  SystemCoreClock = HAL_RCC_GetSysClockFreq() >> AHBPrescTable[(RCC->CFGR & RCC_CFGR_HPRE)>> RCC_CFGR_HPRE_Pos];
 80016b4:	f000 f832 	bl	800171c <HAL_RCC_GetSysClockFreq>
 80016b8:	0001      	movs	r1, r0
 80016ba:	4b12      	ldr	r3, [pc, #72]	; (8001704 <HAL_RCC_ClockConfig+0x278>)
 80016bc:	68db      	ldr	r3, [r3, #12]
 80016be:	091b      	lsrs	r3, r3, #4
 80016c0:	220f      	movs	r2, #15
 80016c2:	4013      	ands	r3, r2
 80016c4:	4a12      	ldr	r2, [pc, #72]	; (8001710 <HAL_RCC_ClockConfig+0x284>)
 80016c6:	5cd3      	ldrb	r3, [r2, r3]
 80016c8:	000a      	movs	r2, r1
 80016ca:	40da      	lsrs	r2, r3
 80016cc:	4b11      	ldr	r3, [pc, #68]	; (8001714 <HAL_RCC_ClockConfig+0x288>)
 80016ce:	601a      	str	r2, [r3, #0]

  /* Configure the source of time base considering new system clocks settings*/
  status = HAL_InitTick(uwTickPrio);
 80016d0:	4b11      	ldr	r3, [pc, #68]	; (8001718 <HAL_RCC_ClockConfig+0x28c>)
 80016d2:	681b      	ldr	r3, [r3, #0]
 80016d4:	250b      	movs	r5, #11
 80016d6:	197c      	adds	r4, r7, r5
 80016d8:	0018      	movs	r0, r3
 80016da:	f7ff f83f 	bl	800075c <HAL_InitTick>
 80016de:	0003      	movs	r3, r0
 80016e0:	7023      	strb	r3, [r4, #0]
  if(status != HAL_OK)
 80016e2:	197b      	adds	r3, r7, r5
 80016e4:	781b      	ldrb	r3, [r3, #0]
 80016e6:	2b00      	cmp	r3, #0
 80016e8:	d002      	beq.n	80016f0 <HAL_RCC_ClockConfig+0x264>
  {
    return status;
 80016ea:	197b      	adds	r3, r7, r5
 80016ec:	781b      	ldrb	r3, [r3, #0]
 80016ee:	e000      	b.n	80016f2 <HAL_RCC_ClockConfig+0x266>
  }

  return HAL_OK;
 80016f0:	2300      	movs	r3, #0
}
 80016f2:	0018      	movs	r0, r3
 80016f4:	46bd      	mov	sp, r7
 80016f6:	b004      	add	sp, #16
 80016f8:	bdb0      	pop	{r4, r5, r7, pc}
 80016fa:	46c0      	nop			; (mov r8, r8)
 80016fc:	40022000 	.word	0x40022000
 8001700:	00001388 	.word	0x00001388
 8001704:	40021000 	.word	0x40021000
 8001708:	fffff8ff 	.word	0xfffff8ff
 800170c:	ffffc7ff 	.word	0xffffc7ff
 8001710:	080018d8 	.word	0x080018d8
 8001714:	20000000 	.word	0x20000000
 8001718:	20000004 	.word	0x20000004

0800171c <HAL_RCC_GetSysClockFreq>:
  *         right SYSCLK value. Otherwise, any configuration based on this function will be incorrect.
  *
  * @retval SYSCLK frequency
  */
uint32_t HAL_RCC_GetSysClockFreq(void)
{
 800171c:	b5b0      	push	{r4, r5, r7, lr}
 800171e:	b08e      	sub	sp, #56	; 0x38
 8001720:	af00      	add	r7, sp, #0
  uint32_t tmpreg, pllm, plld, pllvco, msiclkrange;    /* no init needed */
  uint32_t sysclockfreq;

  tmpreg = RCC->CFGR;
 8001722:	4b4c      	ldr	r3, [pc, #304]	; (8001854 <HAL_RCC_GetSysClockFreq+0x138>)
 8001724:	68db      	ldr	r3, [r3, #12]
 8001726:	62fb      	str	r3, [r7, #44]	; 0x2c

  /* Get SYSCLK source -------------------------------------------------------*/
  switch (tmpreg & RCC_CFGR_SWS)
 8001728:	6afa      	ldr	r2, [r7, #44]	; 0x2c
 800172a:	230c      	movs	r3, #12
 800172c:	4013      	ands	r3, r2
 800172e:	2b0c      	cmp	r3, #12
 8001730:	d014      	beq.n	800175c <HAL_RCC_GetSysClockFreq+0x40>
 8001732:	d900      	bls.n	8001736 <HAL_RCC_GetSysClockFreq+0x1a>
 8001734:	e07b      	b.n	800182e <HAL_RCC_GetSysClockFreq+0x112>
 8001736:	2b04      	cmp	r3, #4
 8001738:	d002      	beq.n	8001740 <HAL_RCC_GetSysClockFreq+0x24>
 800173a:	2b08      	cmp	r3, #8
 800173c:	d00b      	beq.n	8001756 <HAL_RCC_GetSysClockFreq+0x3a>
 800173e:	e076      	b.n	800182e <HAL_RCC_GetSysClockFreq+0x112>
  {
    case RCC_SYSCLKSOURCE_STATUS_HSI:  /* HSI used as system clock source */
    {
      if ((RCC->CR & RCC_CR_HSIDIVF) != 0U)
 8001740:	4b44      	ldr	r3, [pc, #272]	; (8001854 <HAL_RCC_GetSysClockFreq+0x138>)
 8001742:	681b      	ldr	r3, [r3, #0]
 8001744:	2210      	movs	r2, #16
 8001746:	4013      	ands	r3, r2
 8001748:	d002      	beq.n	8001750 <HAL_RCC_GetSysClockFreq+0x34>
      {
        sysclockfreq =  (HSI_VALUE >> 2);
 800174a:	4b43      	ldr	r3, [pc, #268]	; (8001858 <HAL_RCC_GetSysClockFreq+0x13c>)
 800174c:	633b      	str	r3, [r7, #48]	; 0x30
      }
      else
      {
        sysclockfreq =  HSI_VALUE;
      }
      break;
 800174e:	e07c      	b.n	800184a <HAL_RCC_GetSysClockFreq+0x12e>
        sysclockfreq =  HSI_VALUE;
 8001750:	4b42      	ldr	r3, [pc, #264]	; (800185c <HAL_RCC_GetSysClockFreq+0x140>)
 8001752:	633b      	str	r3, [r7, #48]	; 0x30
      break;
 8001754:	e079      	b.n	800184a <HAL_RCC_GetSysClockFreq+0x12e>
    }
    case RCC_SYSCLKSOURCE_STATUS_HSE:  /* HSE used as system clock */
    {
      sysclockfreq = HSE_VALUE;
 8001756:	4b42      	ldr	r3, [pc, #264]	; (8001860 <HAL_RCC_GetSysClockFreq+0x144>)
 8001758:	633b      	str	r3, [r7, #48]	; 0x30
      break;
 800175a:	e076      	b.n	800184a <HAL_RCC_GetSysClockFreq+0x12e>
    }
    case RCC_SYSCLKSOURCE_STATUS_PLLCLK:  /* PLL used as system clock */
    {
      pllm = PLLMulTable[(uint32_t)(tmpreg & RCC_CFGR_PLLMUL) >> RCC_CFGR_PLLMUL_Pos];
 800175c:	6afb      	ldr	r3, [r7, #44]	; 0x2c
 800175e:	0c9a      	lsrs	r2, r3, #18
 8001760:	230f      	movs	r3, #15
 8001762:	401a      	ands	r2, r3
 8001764:	4b3f      	ldr	r3, [pc, #252]	; (8001864 <HAL_RCC_GetSysClockFreq+0x148>)
 8001766:	5c9b      	ldrb	r3, [r3, r2]
 8001768:	62bb      	str	r3, [r7, #40]	; 0x28
      plld = ((uint32_t)(tmpreg & RCC_CFGR_PLLDIV) >> RCC_CFGR_PLLDIV_Pos) + 1U;
 800176a:	6afb      	ldr	r3, [r7, #44]	; 0x2c
 800176c:	0d9a      	lsrs	r2, r3, #22
 800176e:	2303      	movs	r3, #3
 8001770:	4013      	ands	r3, r2
 8001772:	3301      	adds	r3, #1
 8001774:	627b      	str	r3, [r7, #36]	; 0x24
      if (__HAL_RCC_GET_PLL_OSCSOURCE() != RCC_PLLSOURCE_HSI)
 8001776:	4b37      	ldr	r3, [pc, #220]	; (8001854 <HAL_RCC_GetSysClockFreq+0x138>)
 8001778:	68da      	ldr	r2, [r3, #12]
 800177a:	2380      	movs	r3, #128	; 0x80
 800177c:	025b      	lsls	r3, r3, #9
 800177e:	4013      	ands	r3, r2
 8001780:	d01a      	beq.n	80017b8 <HAL_RCC_GetSysClockFreq+0x9c>
      {
        /* HSE used as PLL clock source */
        pllvco = (uint32_t)(((uint64_t)HSE_VALUE * (uint64_t)pllm) / (uint64_t)plld);
 8001782:	6abb      	ldr	r3, [r7, #40]	; 0x28
 8001784:	61bb      	str	r3, [r7, #24]
 8001786:	2300      	movs	r3, #0
 8001788:	61fb      	str	r3, [r7, #28]
 800178a:	4a35      	ldr	r2, [pc, #212]	; (8001860 <HAL_RCC_GetSysClockFreq+0x144>)
 800178c:	2300      	movs	r3, #0
 800178e:	69b8      	ldr	r0, [r7, #24]
 8001790:	69f9      	ldr	r1, [r7, #28]
 8001792:	f7fe fd65 	bl	8000260 <__aeabi_lmul>
 8001796:	0002      	movs	r2, r0
 8001798:	000b      	movs	r3, r1
 800179a:	0010      	movs	r0, r2
 800179c:	0019      	movs	r1, r3
 800179e:	6a7b      	ldr	r3, [r7, #36]	; 0x24
 80017a0:	613b      	str	r3, [r7, #16]
 80017a2:	2300      	movs	r3, #0
 80017a4:	617b      	str	r3, [r7, #20]
 80017a6:	693a      	ldr	r2, [r7, #16]
 80017a8:	697b      	ldr	r3, [r7, #20]
 80017aa:	f7fe fd39 	bl	8000220 <__aeabi_uldivmod>
 80017ae:	0002      	movs	r2, r0
 80017b0:	000b      	movs	r3, r1
 80017b2:	0013      	movs	r3, r2
 80017b4:	637b      	str	r3, [r7, #52]	; 0x34
 80017b6:	e037      	b.n	8001828 <HAL_RCC_GetSysClockFreq+0x10c>
      }
      else
      {
        if ((RCC->CR & RCC_CR_HSIDIVF) != 0U)
 80017b8:	4b26      	ldr	r3, [pc, #152]	; (8001854 <HAL_RCC_GetSysClockFreq+0x138>)
 80017ba:	681b      	ldr	r3, [r3, #0]
 80017bc:	2210      	movs	r2, #16
 80017be:	4013      	ands	r3, r2
 80017c0:	d01a      	beq.n	80017f8 <HAL_RCC_GetSysClockFreq+0xdc>
        {
          pllvco = (uint32_t)((((uint64_t)(HSI_VALUE >> 2)) * (uint64_t)pllm) / (uint64_t)plld);
 80017c2:	6abb      	ldr	r3, [r7, #40]	; 0x28
 80017c4:	60bb      	str	r3, [r7, #8]
 80017c6:	2300      	movs	r3, #0
 80017c8:	60fb      	str	r3, [r7, #12]
 80017ca:	4a23      	ldr	r2, [pc, #140]	; (8001858 <HAL_RCC_GetSysClockFreq+0x13c>)
 80017cc:	2300      	movs	r3, #0
 80017ce:	68b8      	ldr	r0, [r7, #8]
 80017d0:	68f9      	ldr	r1, [r7, #12]
 80017d2:	f7fe fd45 	bl	8000260 <__aeabi_lmul>
 80017d6:	0002      	movs	r2, r0
 80017d8:	000b      	movs	r3, r1
 80017da:	0010      	movs	r0, r2
 80017dc:	0019      	movs	r1, r3
 80017de:	6a7b      	ldr	r3, [r7, #36]	; 0x24
 80017e0:	603b      	str	r3, [r7, #0]
 80017e2:	2300      	movs	r3, #0
 80017e4:	607b      	str	r3, [r7, #4]
 80017e6:	683a      	ldr	r2, [r7, #0]
 80017e8:	687b      	ldr	r3, [r7, #4]
 80017ea:	f7fe fd19 	bl	8000220 <__aeabi_uldivmod>
 80017ee:	0002      	movs	r2, r0
 80017f0:	000b      	movs	r3, r1
 80017f2:	0013      	movs	r3, r2
 80017f4:	637b      	str	r3, [r7, #52]	; 0x34
 80017f6:	e017      	b.n	8001828 <HAL_RCC_GetSysClockFreq+0x10c>
        }
        else
        {
         pllvco = (uint32_t)(((uint64_t)HSI_VALUE * (uint64_t)pllm) / (uint64_t)plld);
 80017f8:	6abb      	ldr	r3, [r7, #40]	; 0x28
 80017fa:	0018      	movs	r0, r3
 80017fc:	2300      	movs	r3, #0
 80017fe:	0019      	movs	r1, r3
 8001800:	4a16      	ldr	r2, [pc, #88]	; (800185c <HAL_RCC_GetSysClockFreq+0x140>)
 8001802:	2300      	movs	r3, #0
 8001804:	f7fe fd2c 	bl	8000260 <__aeabi_lmul>
 8001808:	0002      	movs	r2, r0
 800180a:	000b      	movs	r3, r1
 800180c:	0010      	movs	r0, r2
 800180e:	0019      	movs	r1, r3
 8001810:	6a7b      	ldr	r3, [r7, #36]	; 0x24
 8001812:	001c      	movs	r4, r3
 8001814:	2300      	movs	r3, #0
 8001816:	001d      	movs	r5, r3
 8001818:	0022      	movs	r2, r4
 800181a:	002b      	movs	r3, r5
 800181c:	f7fe fd00 	bl	8000220 <__aeabi_uldivmod>
 8001820:	0002      	movs	r2, r0
 8001822:	000b      	movs	r3, r1
 8001824:	0013      	movs	r3, r2
 8001826:	637b      	str	r3, [r7, #52]	; 0x34
        }
      }
      sysclockfreq = pllvco;
 8001828:	6b7b      	ldr	r3, [r7, #52]	; 0x34
 800182a:	633b      	str	r3, [r7, #48]	; 0x30
      break;
 800182c:	e00d      	b.n	800184a <HAL_RCC_GetSysClockFreq+0x12e>
    }
    case RCC_SYSCLKSOURCE_STATUS_MSI:  /* MSI used as system clock source */
    default: /* MSI used as system clock */
    {
      msiclkrange = (RCC->ICSCR & RCC_ICSCR_MSIRANGE ) >> RCC_ICSCR_MSIRANGE_Pos;
 800182e:	4b09      	ldr	r3, [pc, #36]	; (8001854 <HAL_RCC_GetSysClockFreq+0x138>)
 8001830:	685b      	ldr	r3, [r3, #4]
 8001832:	0b5b      	lsrs	r3, r3, #13
 8001834:	2207      	movs	r2, #7
 8001836:	4013      	ands	r3, r2
 8001838:	623b      	str	r3, [r7, #32]
      sysclockfreq = (32768U * (1UL << (msiclkrange + 1U)));
 800183a:	6a3b      	ldr	r3, [r7, #32]
 800183c:	3301      	adds	r3, #1
 800183e:	2280      	movs	r2, #128	; 0x80
 8001840:	0212      	lsls	r2, r2, #8
 8001842:	409a      	lsls	r2, r3
 8001844:	0013      	movs	r3, r2
 8001846:	633b      	str	r3, [r7, #48]	; 0x30
      break;
 8001848:	46c0      	nop			; (mov r8, r8)
    }
  }
  return sysclockfreq;
 800184a:	6b3b      	ldr	r3, [r7, #48]	; 0x30
}
 800184c:	0018      	movs	r0, r3
 800184e:	46bd      	mov	sp, r7
 8001850:	b00e      	add	sp, #56	; 0x38
 8001852:	bdb0      	pop	{r4, r5, r7, pc}
 8001854:	40021000 	.word	0x40021000
 8001858:	003d0900 	.word	0x003d0900
 800185c:	00f42400 	.word	0x00f42400
 8001860:	007a1200 	.word	0x007a1200
 8001864:	080018e8 	.word	0x080018e8

08001868 <__libc_init_array>:
 8001868:	b570      	push	{r4, r5, r6, lr}
 800186a:	2600      	movs	r6, #0
 800186c:	4d0c      	ldr	r5, [pc, #48]	; (80018a0 <__libc_init_array+0x38>)
 800186e:	4c0d      	ldr	r4, [pc, #52]	; (80018a4 <__libc_init_array+0x3c>)
 8001870:	1b64      	subs	r4, r4, r5
 8001872:	10a4      	asrs	r4, r4, #2
 8001874:	42a6      	cmp	r6, r4
 8001876:	d109      	bne.n	800188c <__libc_init_array+0x24>
 8001878:	2600      	movs	r6, #0
 800187a:	f000 f821 	bl	80018c0 <_init>
 800187e:	4d0a      	ldr	r5, [pc, #40]	; (80018a8 <__libc_init_array+0x40>)
 8001880:	4c0a      	ldr	r4, [pc, #40]	; (80018ac <__libc_init_array+0x44>)
 8001882:	1b64      	subs	r4, r4, r5
 8001884:	10a4      	asrs	r4, r4, #2
 8001886:	42a6      	cmp	r6, r4
 8001888:	d105      	bne.n	8001896 <__libc_init_array+0x2e>
 800188a:	bd70      	pop	{r4, r5, r6, pc}
 800188c:	00b3      	lsls	r3, r6, #2
 800188e:	58eb      	ldr	r3, [r5, r3]
 8001890:	4798      	blx	r3
 8001892:	3601      	adds	r6, #1
 8001894:	e7ee      	b.n	8001874 <__libc_init_array+0xc>
 8001896:	00b3      	lsls	r3, r6, #2
 8001898:	58eb      	ldr	r3, [r5, r3]
 800189a:	4798      	blx	r3
 800189c:	3601      	adds	r6, #1
 800189e:	e7f2      	b.n	8001886 <__libc_init_array+0x1e>
 80018a0:	080018fc 	.word	0x080018fc
 80018a4:	080018fc 	.word	0x080018fc
 80018a8:	080018fc 	.word	0x080018fc
 80018ac:	08001900 	.word	0x08001900

080018b0 <memset>:
 80018b0:	0003      	movs	r3, r0
 80018b2:	1882      	adds	r2, r0, r2
 80018b4:	4293      	cmp	r3, r2
 80018b6:	d100      	bne.n	80018ba <memset+0xa>
 80018b8:	4770      	bx	lr
 80018ba:	7019      	strb	r1, [r3, #0]
 80018bc:	3301      	adds	r3, #1
 80018be:	e7f9      	b.n	80018b4 <memset+0x4>

080018c0 <_init>:
 80018c0:	b5f8      	push	{r3, r4, r5, r6, r7, lr}
 80018c2:	46c0      	nop			; (mov r8, r8)
 80018c4:	bcf8      	pop	{r3, r4, r5, r6, r7}
 80018c6:	bc08      	pop	{r3}
 80018c8:	469e      	mov	lr, r3
 80018ca:	4770      	bx	lr

080018cc <_fini>:
 80018cc:	b5f8      	push	{r3, r4, r5, r6, r7, lr}
 80018ce:	46c0      	nop			; (mov r8, r8)
 80018d0:	bcf8      	pop	{r3, r4, r5, r6, r7}
 80018d2:	bc08      	pop	{r3}
 80018d4:	469e      	mov	lr, r3
 80018d6:	4770      	bx	lr
